:020000040800F2
:1000000000000120C1780008DB330008DD33000860
:10001000DF330008E1330008E3330008000000008C
:10002000000000000000000000000000E5330008B0
:10003000E733000800000000E9330008EB33000854
:100040001179000811790008ED33000811790008D2
:100050001179000811790008F93300080D340008FF
:1000600011790008133400081179000819340008C8
:10007000253400083134000811790008117900088E
:100080003D34000841340008117900081179000856
:1000900000000000117900084D34000811790008B3
:1000A0001179000811790008117900081179000808
:1000B00011790008117900081179000811790008F8
:1000C00011790008117900085134000811790008ED
:1000D000117900085D3400081179000811790008D1
:1000E00011790008117900086934000811790008B5
:1000F00011790008000000000000000011790008DC
:100100001179000811790008753400081179000888
:100110001179000811790008117900081179000897
:100120001179000811790008117900081179000887
:080130001179000811790008A3
:1001400010B5054C237833B9044B13B10448AFF311
:1001500000800123237010BDF8060020000000007D
:10016000441E030808B5034B1BB103490348AFF312
:10017000008008BD00000000FC060020441E0308AB
:1001800014214160704714207047406A7047000096
:1001900081010008870100088B010008A101000807
:1001A00010B5044604F1100000F05CFCC4F8F8003F
:1001B0000148C4F87C0110BD90010008F8B5E6B014
:1001C00004460D4616461F460A4906A800F0CAFE18
:1001D00070996F9A05910492009733466E996D9AC3
:1001E000039102922A466C990191214600F060F831
:1001F00067B0F0BD9C010008F8B5E6B004460D46B6
:1002000016461F46094906A800F0ACFE6F996E9A83
:100210000491039200976D996C9A02910192334672
:100220002A46214600F087F867B0F0BD9C0100081F
:1002300038B500281CBF01680029184A23D1184B83
:100240001C684FF6F0710C404CF24025AC421FBFC9
:100250001B6819404CF27024A14212D1114D29683B
:1002600079B911490B68C3F30B03B3F58A6F1FBF4C
:100270000968C1F30B0140F28343994204BF012195
:10028000117028B905E0094B994204BF0121117092
:100290004068BDE8324002F073BC00BF1407002084
:1002A00000ED00E0002004E00010005C0000374892
:1002B0002DE9F04104460D46216816464A681F465E
:1002C00090478046B8F5403F2ED122680A9993683E
:1002D000204698478046B8F5403F25D12368089AC4
:1002E0000799D3F80CC02046E0478046B8F5403F58
:1002F0001AD12368069A39461F692046B8478046B6
:10030000B8F5403F10D1236829465D693246204642
:10031000A8478046B8F5403F06D123680B9A099953
:100320009D692046A847804621680A682046904774
:100330004046BDE8F0812DE9F04104460D462168B4
:1003400016464A681F4690478046B8F5403F2ED172
:1003500022680A999368204698478046B8F5403F3E
:1003600025D12368089A0799D3F80CC02046E047A6
:100370008046B8F5403F1AD12368069A39461F696E
:100380002046B8478046B8F5403F10D1236829463B
:100390005D6932462046A8478046B8F5403F06D101
:1003A00023680999DD6900222046A8478046216814
:1003B0000A68204690474046BDE8F0814FF440303F
:1003C00070470000F0B50C4685B0114600281A466B
:1003D0001CBF0568002D0B4B11D082B104B971B957
:1003E0000D9860B10F9E0E9F0A9B02900496039792
:1003F0000B980C9E009001962046A847034618468D
:1004000005B0F0BD020003002DE9F04F0646D0B064
:100410000868F56DD6F860E0726EB76EF36E00BADC
:1004200000906C46486800BA60600DF1400888682A
:1004300000BAA060C86800BAE060086900BA20612C
:10044000486900BA6061886900BAA061C86900BAE9
:10045000E061086A00BA2062486A00BA6062886A8D
:1004600000BAA062C86A00BAE062086B00BA2063F2
:10047000486B00BA6063886B00BAA063C86B00BAAF
:10048000E063402058F80C1C58F820CC58F838ACE1
:100490008CEA010158F840CC8AEA01018CEA010992
:1004A0004FEAF979401E48F8049BEBD187EA020035
:1004B00000EA0E00784010EBF5610098DFF824C4E4
:1004C00041186144C81882EABE032B404FEAF0612C
:1004D00053405918636859186144CF194FEAB5035E
:1004E00083EABE01014081EABE0111EBF765A16814
:1004F0004D196544A91883EAB0023A404FEAF16504
:100500005A405519E26855194FEAB70282EAB00716
:1005100065440F4005EBBE0E97EAB00717EBFE658A
:1005200027697D194FEAB10782EA0701654401EAAC
:100530000E01EB18514011EBF36561694D194FEA5B
:10054000BE0187EA010E65440EEA030E15EBB0000A
:100550008EEA070E0EEBF065D4F818E0754465449A
:10056000AA1881EAB30505404FEAF26E4D40AE4449
:10057000E569AE44E64477444FEAB00080EAB30E42
:100580000EEA020E8EEAB30E0EEBF765D4F820E009
:1005900075446544691880EAB2053D404FEAF16E42
:1005A0004540AE44656AAE44E6440EEBB3034FEA01
:1005B000B70787EAB20E0EEA010E8EEAB20E0EEB14
:1005C000F365D4F828E075446544281887EAB10536
:1005D0001D404FEAF06E7D40AE44E56AAE44E6440D
:1005E0000EEBB2024FEAB30383EAB10E0EEA000E3D
:1005F0008EEAB10E0EEBF265D4F830E07544654436
:10060000EF1983EAB00515404FEAF76E5D40AE443E
:10061000656BAE44E6440EEBB1014FEAB20282EAEA
:10062000B00E0EEA070E8EEAB00E0EEBF165D4F8AE
:1006300038E075446544EB1882EAB7050D404FEA8F
:10064000F36E5540AE44E56BAE44E6440EEBB000AD
:100650004FEAB10181EAB70E0EEA030E8EEAB70E39
:100660000EEBF065D4F840E07544654481EAB30EC2
:10067000AA180EEA000E4FEAF2658EEA010E7544E2
:10068000DDF844E04FEAB000754480EAB30E6544FB
:100690000EEA020E15EBB7078EEAB30E0EEBF76506
:1006A000DDF848E04FEAB202754480EA020E654484
:1006B0000EEA070E69188EEA000E0EEBF165DDF802
:1006C0004CE07544654405EBB3034FEAB70E1427BD
:1006D0000DF1500CDFF810528EEA010B82EA0B0B81
:1006E0000BEBF36A5CF804BBDA44AA44504483EA97
:1006F000B10B4FEAF06A8EEA0B0BDA445CF804BBEC
:10070000DA44AA44524480EAB30B4FEAF26A8BEA15
:10071000B10BDA445CF804BBDA444FEAB000AA44F7
:1007200080EA020BD6448BEAB30B0BEBFE6A5CF853
:1007300004BBDA444FEAB202AA4482EA0E0B0AEB87
:10074000B10180EA0B0B0BEBF16A5CF804BBDA44F5
:100750007F1DAA44282F0AEBB3034FEABE0EBBD37A
:100760003C2F61D3502F4DD204EB870CC7F15407B7
:100770005E4CA7FB04A504465D4FA8088EEA010A5B
:1007800082EA0A0A5CF804BB0AEBF3655D447D1952
:100790002C1983EAB10A4FEAF4658EEA0A0A554435
:1007A0005CF804AB5CF804BB55447D19AA1884EAD4
:1007B000B30A4FEAF2658AEAB10A55445D444FEA4A
:1007C000B4047D1984EA020AAE448AEAB30A0AEB49
:1007D000FE655CF804AB55444FEAB2027D1982EA2B
:1007E0000E0A15EBB10184EA0A0A5CF804BB0AEBB5
:1007F000F1655D447D1915EBB303401E4FEABE0E53
:10080000BCD12046F46D1B19F365336EC9183166EF
:10081000716E71447166B36ED218B266F16E401893
:10082000F06650B0BDE8F08F4EEA010B0EEA010A07
:100830000BEA020B4BEA0A0A0AEBF36554F827A00D
:10084000DFF8B0C0554443EAB10B654403EAB10A8E
:100850000BEA0E0B28184BEA0A0A7F1C0AEBF0651C
:1008600054F827A0554440EAB30B654400EAB30AA4
:100870000BEAB10BAA184BEA0A0A7F1C0AEBF265D5
:1008800054F827A055444FEAB00040EA020B6544F3
:1008900000EA020A0BEAB30BAE444BEA0A0A7F1CD9
:1008A0000AEBFE6554F827A055444FEAB20242EA2B
:1008B0000E0B654402EA0E0A0BEA000B15EBB101C0
:1008C0004BEA0A0A7F1C0AEBF16554F827A055444D
:1008D0007F1C65443C2F05EBB3034FEABE0EA3D348
:1008E00040E700BF9979825AA1EBD96ECDCCCCCC30
:1008F000D6C162CADCBC1B8F00B581B00168074A53
:10090000914200D110B9064801B000BD7C212EF003
:1009100006F84FF4003001B000BD00BF040A000823
:10092000030002002DE9F0410B4A92E8F85188B02B
:10093000694681E8F8510268084B9A4200D118B91B
:10094000074808B0BDE8F0811422083000F04FFBE2
:1009500008B0BDE8F08100BFE4090008040A0008FF
:1009600003000200152904D20268044B9A4200D108
:1009700008B903487047083000F048BB040A000873
:100980000300020010B481B013460268074CA24273
:1009900000D118B901B010BC0548704701B000F192
:1009A000240210BC083000F035BB00BF040A000868
:1009B0000300020010B481B013460268074CA24243
:1009C00000D118B901B010BC054870470A4601B003
:1009D00000F1240110BC083000F070BB040A0008CC
:1009E000030002000123456789ABCDEFFEDCBA9816
:1009F00076543210F0E1D2C3000000000000000085
:100A000000000000F9080008250900086509000831
:100A100085090008B509000809040008810F0008CD
:100A2000CD0F0008890F0008F0B5A3B004460B48AD
:100A300002900D4616461F46094B0822402104A885
:100A400000F0D1FA28980190009733462A462146B3
:100A500002A800F01BF823B0F0BD00BF040A000894
:100A6000180A000810B5040008BF002408D0054883
:100A7000054B20600822402104F1080000F0B3FA81
:100A8000204610BD040A0008180A00082DE9F041AC
:100A900004460E46216817464A681D469047804620
:100AA000B8F5003F19D12268069993682046984707
:100AB0008046B8F5003F10D123683146DE683A46DB
:100AC0002046B0478046B8F5003F06D12368079A14
:100AD00029461D692046A847804621680A682046A5
:100AE00090474046BDE8F08110B500F033FA4FF46E
:100AF000403400280EBF034C4FF4C0712DF00FFF9F
:100B0000204610BD0200030010B5044600F022FA92
:100B100008B9054810BD0021A160D0F87C211168FA
:100B200088474FF4403010BD0200030070B5044602
:100B30000D4600F00FFA064E40B1D0F87C01416836
:100B40008847A84224BF65604FF44036304670BDE8
:100B5000020003002DE9FF4715000C4600D02CB120
:100B6000064600F0F7F95FEA000801D16448C3E0E7
:100B7000D8F8F80001684A689047B0F5003F17D1EF
:100B8000D8F87C118A68404690478146B9F1810FB8
:100B900080F09E80A94508F1FC0A17D2D8F8F80029
:100BA0000368D3F80CC02A462146E047B0F5003F61
:100BB00040F08E80D8F8F8000368D3F810C06A4679
:100BC0005146E047B0F5003F76D10AE0002004E04E
:100BD000215C0AF800100098401C00900098A84280
:100BE000F6D34FF0000C4749474A484B01AC0098F8
:100BF000844558D2D3E9007001ADC5E90070107882
:100C000000281ABF042086464FF0000E085854F8FA
:100C10000E5028443E4D05600127D0F800E0876063
:100C2000019D4F681AF80C007D408EEA050585F09D
:100C3000040E65680F687D4085F0FC05754485F0FD
:100C4000A30568400AF80C000CF1010CCFE7D3E9CA
:100C5000004501A8C0E9004510782E4D002814BFBA
:100C60004FF0040E4FF0000E01A8744651F80EE04C
:100C70000459A6440127CEF80050DEF80040CEF813
:100C800008704D68019F40687D406C400D68684069
:100C900084F0040480F0FC00041984F057040AF87E
:100CA0000C400CF1010CCC45D1D3D8F8F800016808
:100CB0004A689047B0F5003F0AD1D8F8F8000368B9
:100CC000D3F80C804A465146C047B0F5003F01D0EA
:100CD000114811E0002006E05AF8201081F06A3136
:100CE0004AF82010401CB0EB990FF5D3B06840F0E3
:100CF0000100B0604FF4403004B0BDE8F08700BFA1
:100D000002000300845F0308140700202C0F000872
:100D1000ADBE4ED70DBE75A10100030038B50C461F
:100D2000017A1546CA0702D500F014F908B9084837
:100D300032BDD0F8F80003682146DC682A46A04797
:100D4000B0F5003F01D0034832BD4FF4403032BD12
:100D500002000300010003002DE9F84191B00546AF
:100D60000E461746402101A82DF0D9FD297AC80763
:100D700004D5284600F0EEF8040002D1DFF8A48084
:100D80004BE0D4F8F800DFF8A0800368D3F810C077
:100D90006A4601A9E047B0F5003F3ED1D4F8F8001B
:100DA00001684A689047B0F5003F36D1D4F87C110D
:100DB0008A6820469047D4F8F830024618461B68E7
:100DC000D3F80CC004F1FC01E047B0F5003F24D19A
:100DD000D4F87C0141688847D4F8F83002461846B8
:100DE0001B68D3F80CC001A9E047B0F5003F14D14F
:100DF000D4F8F8000268696893689847B0F5003F36
:100E00000BD1D4F8F80003681C693A463146A04774
:100E1000B0F5003F08BF4FF44038404612B0BDE87F
:100E2000F08100BF02000300010003002DE9F8413A
:100E3000A5B0074688461646402115A82DF06FFD3F
:100E400000220492402105A82DF069FD387AC107DF
:100E50005ED5384600F07EF8050059D0D5F8F80088
:100E60002D4C0368D3F810C06A4605A9E047B0F5D9
:100E7000003F3CD1D5F8F80001684A689047B0F5CA
:100E8000003F34D1D5F87C118A6828469047D5F8C0
:100E9000F830024618461B68D3F80CC005F1FC0177
:100EA000E047B0F5003F22D1D5F87C014168884782
:100EB000D5F8F830024618461B68D3F80CC005A9CF
:100EC000E047B0F5003F12D1D5F8F8000268796824
:100ED00093689847B0F5003F09D1D5F8F80003684A
:100EE0001D6904AA15A9A847B0F5003F01D0204606
:100EF0000FE00A4B0A490B4A0396029101924046C1
:100F00001C68049B009415AA796800F0E5F900E0DC
:100F1000054826B0BDE8F081010003008C5F03089E
:100F2000936E030026C703000200030004B0010112
:100F300000170145E90A0008090B00082D0B0008FD
:100F4000BD030008550B00081D0D0008590D0008D1
:100F50002D0E00080168024A914218BF0020704718
:100F6000340F000810B5040008BF002404D0034863
:100F70002060204609688847204610BD340F0008CD
:100F800020225C302DF0C7BCF0B58468A308002295
:100F900004F0030407E000F15C0555F8226035BA5F
:100FA00041F82250521C9A42F5D300220BE000F186
:100FB0005C0502EB830755F82360D500C5F11805E1
:100FC000EE40CE55521CA242F1D3F0BD30B5C468FC
:100FD00003690022E31AD5188C5C0544521C082AC8
:100FE0002C77F8D330BD0360C1600261704738B51B
:100FF000044615460022626023685A689047002024
:101000006061A061A5604FF4003032BD81604FF493
:10101000003070472DE9F84304462079D4F80C805D
:10102000450748BF244845D466691D46A8F101001C
:1010300000EAD60306EBC506B6EBC50F666102D221
:10104000A669761CA6611746A66906EB5576A661C9
:101050000E46E918884225D2A8EB03094A463146D4
:10106000F8182DF058FC2268136839460FE0424604
:1010700038462DF050FC23681A68394620469047C0
:1010800007E0311811F00300F1D1226813682046FF
:101090009847484600EB0809A9F10101A942F0D39D
:1010A000002300E000202A1A3118F8182DF033FC34
:1010B0004FF40030BDE8F283040002002DE9FC4F3C
:1010C000024685B0D0681369DFF86CC1DFF86C8127
:1010D000A0EB030A506840F004005060002703A80A
:1010E00002900DF10C0ED8E9003403A8544DC0E96C
:1010F00000342878534D00280CBF00230423994660
:101100005CF803305EF80940234401261D601C682A
:101110009E60DCF80430039DDCF80090DEF804608B
:101120005D406540484C654089EA0606474C66408C
:101130007519474C6540D8E9006B03AC0028C4E939
:10114000006B0EBF002404200424029E5CF8000003
:10115000345920183F4C04600126046886600398C7
:10116000029E43406340384C7068634089EA000047
:10117000364C6040034438484340280018BF0120E3
:101180005B1E9B41042F2CBFC0B2D80F02F1140389
:1011900053F8200007F00303C3F10303DB00D8403A
:1011A0000DF807007F1C082F9DD315460C466A6971
:1011B000AB69E868D20842EA4372401E00EA0207BF
:1011C000002302409B420AD8524508D28020E055B5
:1011D0007F1C574516D2AAEB0701E01910E08020CA
:1011E000E05500E0E355E8687F1C8742FAD32A689F
:1011F000136828469847BAF1000F03D0514620469D
:101200002DF08DFB2A68069E059F93686946284647
:1012100098472A68D2F8009021462846C8472B688C
:10122000DA683946284690470EB1A86830604FF416
:10123000003007B0BDE8F08F845F03085C1200083F
:10124000140700205FC5109304850012FC68017A22
:10125000C0F524FF24AF33D426AF698B04B001015D
:1012600000170145F8B501240094002300240DE087
:10127000009D065D0F5D7E40F643761CF60F86F0FE
:10128000010635400095641C009DEB189442EFD395
:101290001846F2BDF8B5002301240094002A11E09D
:1012A000009C85188F1815F8016C17F8015C6E40CA
:1012B000F643761CF60F86F0010634400094009C3D
:1012C000E318521EECD11846F2BD0000651200086A
:1012D00095120008010000002DE9F84F1D46DDF8C9
:1012E00028900B9F0D9C4FF0FF3300930E469246C3
:1012F000D9F800B0804632465146D847834664B399
:10130000D9F8043032465146404698476FEA0B02FE
:10131000521C42EA0B0200996FEAD2735B1C19401F
:10132000C2430091521C024300996FEAD2735B1CC6
:101330001940009186F05531484087EA000181F05C
:101340005531216080F05531C943491C0843009A4A
:101350006FEAD070401C82430092D9F8080001283F
:1013600009D17540E943491C0D4300986FEAD572D5
:10137000521C90430AE0F11C85EA9102D243521CB0
:10138000154300986FEAD5735B1C984386F0AA3624
:10139000009086EA0B0686F0AA33F243DB430C98F2
:1013A000C2F3C0725B1C42EAD3720099D243521C52
:1013B00091430091774000998843009987F0AA37BC
:1013C0000F403843BDE8F28F00000000000000002D
:1013D00001F0FF01102A2BDB10F0070F08D010F8E6
:1013E000013B013A8B422DD010F0070F42B3F6D1EA
:1013F000F0B441EA012141EA014122F007047FF003
:1014000000070023F0E80256083C85EA010586EA59
:10141000010685FA47F5A3FA87F586FA47F6A5FA95
:1014200087F68EB9EED1F0BC01F0FF0102F00702A1
:1014300032B110F8013B013A83EA010313B1F8D14C
:101440000020704701387047002D06BF354603382D
:10145000073815F0010F07D1013015F4807F02BF66
:10146000013015F4C03F0130F0BC0138704700BFB7
:10147000034613F8012B002AFBD1181A01387047D4
:1014800081F0004102E000BF83F0004330B54FEA35
:1014900041044FEA430594EA050F08BF90EA020FA2
:1014A0001FBF54EA000C55EA020C7FEA645C7FEA35
:1014B000655C00F0E2804FEA5454D4EB5555B8BF58
:1014C0006D420CDD2C4480EA020281EA030382EAC9
:1014D000000083EA010180EA020281EA0303362D5B
:1014E00088BF30BD11F0004F4FEA01314FF4801C2E
:1014F0004CEA113102D0404261EB410113F0004F40
:101500004FEA03334CEA133302D0524263EB4303F6
:1015100094EA050F00F0A780A4F10104D5F1200E94
:101520000DDB02FA0EFC22FA05F2801841F10001EF
:1015300003FA0EF2801843FA05F359410EE0A5F1C3
:1015400020050EF1200E012A03FA0EFC28BF4CF0F4
:10155000020C43FA05F3C01851EBE37101F00045AA
:1015600007D54FF0000EDCF1000C7EEB00006EEBB7
:101570000101B1F5801F1BD3B1F5001F0CD3490841
:101580005FEA30004FEA3C0C04F101044FEA445298
:1015900012F5800F80F09A80BCF1004F08BF5FEA1F
:1015A000500C50F1000041EB045141EA050130BDFF
:1015B0005FEA4C0C404141EB0101013C28BFB1F511
:1015C000801FE9D291F0000F04BF01460020B1FA5C
:1015D00081F308BF2033A3F10B03B3F120020CDA2F
:1015E0000C3208DD02F1140CC2F10C0201FA0CF00D
:1015F00021FA02F10CE002F11402D8BFC2F1200C72
:1016000001FA02F120FA0CFCDCBF41EA0C01904027
:10161000E41AA2BF01EB0451294330BD6FEA040470
:101620001F3C1CDA0C340EDC04F11404C4F120025B
:1016300020FA04F001FA02F340EA030021FA04F36D
:1016400045EA030130BDC4F10C04C4F1200220FAC4
:1016500002F001FA04F340EA0300294630BD21FA02
:1016600004F0294630BD94F0000F83F4801306BFC8
:1016700081F480110134013D4EE77FEA645C18BFBC
:101680007FEA655C29D094EA050F08BF90EA020F53
:1016900005D054EA000C04BF1946104630BD91EA4B
:1016A000030F1EBF0021002030BD5FEA545C05D14E
:1016B0004000494128BF41F0004130BD14F580048D
:1016C0003CBF01F5801130BD01F0004545F0FE4101
:1016D00041F470014FF0000030BD7FEA645C1ABF36
:1016E000194610467FEA655C1CBF0B46024650EA6D
:1016F000013406BF52EA033591EA030F41F4002199
:1017000030BD00BF90F0000F04BF0021704730B51E
:101710004FF4806404F132044FF000054FF00001F3
:1017200050E700BF90F0000F04BF0021704730B5B4
:101730004FF4806404F1320410F0004548BF404289
:101740004FF000013EE700BF42004FEAE2014FEADE
:1017500031014FEA02701FBF12F07F4393F07F4FB9
:1017600081F06051704732F07F4208BF704793F0BC
:101770007F4F04BF41F40021704730B54FF46074CF
:1017800001F0004521F000411CE700BF50EA0102D2
:1017900008BF704730B54FF000050AE050EA01027B
:1017A00008BF704730B511F0004502D5404261EBEB
:1017B00041014FF4806404F132045FEA915C3FF42C
:1017C000D8AE4FF003025FEADC0C18BF03325FEAC9
:1017D000DC0C18BF033202EBDC02C2F1200300FA7A
:1017E00003FC20FA02F001FA03FE40EA0E0021FA9F
:1017F00002F11444BDE600BF70B54FF0FF0C4CF48D
:10180000E06C1CEA11541DBF1CEA135594EA0C0F3E
:1018100095EA0C0F00F0DEF82C4481EA030621EA79
:101820004C5123EA4C5350EA013518BF52EA0335B4
:1018300041F4801143F4801338D0A0FB02CE4FF066
:101840000005E1FB02E506F00042E0FB03E54FF096
:101850000006E1FB03569CF0000F18BF4EF0010E8E
:10186000A4F1FF04B6F5007F64F5407404D25FEA8A
:101870004E0E6D4146EB060642EAC62141EA55513D
:101880004FEAC52040EA5E504FEACE2EB4F1FD0C7F
:1018900088BFBCF5E06F1ED8BEF1004F08BF5FEAFD
:1018A000500E50F1000041EB045170BD06F00046AF
:1018B00046EA010140EA020081EA0301B4EB5C045C
:1018C000C2BFD4EB0C0541EA045170BD41F4801154
:1018D0004FF0000E013C00F3AB8014F1360FDEBF79
:1018E000002001F0004170BDC4F10004203C35DA55
:1018F0000C341BDC04F11404C4F1200500FA05F3D8
:1019000020FA04F001FA05F240EA020001F0004278
:1019100021F0004110EBD37021FA04F642EB0601EE
:101920005EEA430E08BF20EAD37070BDC4F10C0418
:10193000C4F1200500FA04F320FA05F001FA04F2DC
:1019400040EA020001F0004110EBD37041F10001C8
:101950005EEA430E08BF20EAD37070BDC4F12005D3
:1019600000FA05F24EEA020E20FA04F301FA05F23B
:1019700043EA020321FA04F001F0004121FA04F2E3
:1019800020EA020000EBD3705EEA430E08BF20EAB3
:10199000D37070BD94F0000F0FD101F000464000ED
:1019A00041EB010111F4801F08BF013CF7D041EA6F
:1019B000060195F0000F18BF704703F00046520073
:1019C00043EB030313F4801F08BF013DF7D043EA44
:1019D0000603704794EA0C0F0CEA135518BF95EAFA
:1019E0000C0F0CD050EA410618BF52EA4306D1D181
:1019F00081EA030101F000414FF0000070BD50EAA0
:101A0000410606BF1046194652EA430619D094EA29
:101A10000C0F02D150EA013613D195EA0C0F05D113
:101A200052EA03361CBF104619460AD181EA030167
:101A300001F0004141F0FE4141F470014FF000001F
:101A400070BD41F0FE4141F4780170BD70B54FF0BA
:101A5000FF0C4CF4E06C1CEA11541DBF1CEA13553A
:101A600094EA0C0F95EA0C0F00F0A7F8A4EB05041C
:101A700081EA030E52EA03354FEA013100F0888013
:101A80004FEA03334FF0805545EA131343EA1263DC
:101A90004FEA022245EA111545EA10654FEA002691
:101AA0000EF000419D4208BF964244F1FD0404F54A
:101AB000407402D25B084FEA3202B61A65EB0305A6
:101AC0005B084FEA32024FF480104FF4002CB6EB63
:101AD000020E75EB030E22BFB61A754640EA0C00E3
:101AE0005B084FEA3202B6EB020E75EB030E22BF23
:101AF000B61A754640EA5C005B084FEA3202B6EB64
:101B0000020E75EB030E22BFB61A754640EA9C0022
:101B10005B084FEA3202B6EB020E75EB030E22BFF2
:101B2000B61A754640EADC0055EA060E18D04FEAB0
:101B3000051545EA16754FEA06164FEAC30343EA50
:101B400052734FEAC2025FEA1C1CC0D111F4801F1D
:101B50000BD141EA00014FF000004FF0004CB6E716
:101B600011F4801F04BF01430020B4F1FD0C88BFB5
:101B7000BCF5E06F3FF6AFAEB5EB030C04BFB6EBC0
:101B8000020C5FEA500C50F1000041EB045170BDB3
:101B90000EF0004E4EEA113114EB5C04C2BFD4EBE0
:101BA0000C0541EA045170BD41F480114FF0000E64
:101BB000013C90E645EA060E8DE60CEA135594EAE0
:101BC0000C0F08BF95EA0C0F3FF43BAF94EA0C0FE3
:101BD0000AD150EA01347FF434AF95EA0C0F7FF458
:101BE00025AF104619462CE795EA0C0F06D152EAAC
:101BF00003353FF4FDAE1046194622E750EA410690
:101C000018BF52EA43067FF4C5AE50EA41047FF4A0
:101C10000DAF52EA43057FF4EBAE12E74FF0FF3C05
:101C200006E000BF4FF0010C02E000BF4FF0010CD6
:101C30004DF804CD4FEA410C7FEA6C5C4FEA430C4F
:101C400018BF7FEA6C5C1BD001B050EA410C0CBF9E
:101C500052EA430C91EA030F02BF90EA020F002000
:101C6000704710F1000F91EA030F58BF994208BF67
:101C700090422CBFD8176FEAE37040F00100704724
:101C80004FEA410C7FEA6C5C02D150EA013C07D17B
:101C90004FEA430C7FEA6C5CD6D152EA033CD3D0C6
:101CA0005DF8040B704700BF8446104662468C46C0
:101CB0001946634600E000BF01B5FFF7B7FF0028F3
:101CC00048BF10F1000F01BD4DF808EDFFF7F4FF1C
:101CD0000CBF012000205DF808FB00BF4DF808EDA7
:101CE000FFF7EAFF34BF012000205DF808FB00BFCA
:101CF0004DF808EDFFF7E0FF94BF012000205DF8EC
:101D000008FB00BF4DF808EDFFF7CEFF94BF0120A0
:101D100000205DF808FB00BF4DF808EDFFF7C4FF99
:101D200034BF012000205DF808FB00BF4FEA410CE2
:101D30007FEA6C5C02D150EA013C0AD14FEA430CC5
:101D40007FEA6C5C02D152EA033C02D14FF0000002
:101D500070474FF0010070474FEA410212F5001240
:101D600015D211D56FF47873B3EB625212D94FEAE2
:101D7000C12343F0004343EA505311F0004F23FACC
:101D800002F018BF404270474FF00000704750EA21
:101D9000013005D111F0004008BF6FF000407047DE
:101DA0004FF00000704700BF4FEA4102B2F1E0433C
:101DB00024BFB3F5001CDCF1FE5C0DD901F0004C32
:101DC0004FEAC0024CEA5070B2F1004F40EB830082
:101DD00008BF20F00100704711F0804F21D113F1AE
:101DE0003872BCBF01F00040704741F480114FEAE7
:101DF0005252C2F11802C2F1200C10FA0CF320FA70
:101E000002F018BF40F001004FEAC1234FEAD3238C
:101E100003FA0CFC40EA0C0023FA02F34FEA4303F6
:101E2000CCE77FEA625307D150EA01331EBF4FF07F
:101E3000FE4040F44000704701F0004040F0FE409A
:101E400040F40000704700BF80F0004002E000BF97
:101E500081F0004142001FBF5FEA410392EA030F95
:101E60007FEA226C7FEA236C6AD04FEA1262D2EBDF
:101E70001363C1BFD218414048404140B8BF5B42E4
:101E8000192B88BF704710F0004F40F4000020F07D
:101E90007F4018BF404211F0004F41F4000121F093
:101EA0007F4118BF494292EA030F3FD0A2F10102DD
:101EB00041FA03FC10EB0C00C3F1200301FA03F11B
:101EC00000F0004302D5494260EB4000B0F5000F3E
:101ED00013D3B0F1807F06D340084FEA310102F1FD
:101EE0000102FE2A51D2B1F1004F40EBC25008BFAF
:101EF00020F0010040EA03007047490040EB000079
:101F0000013A28BFB0F5000FEDD2B0FA80FCACF179
:101F1000080CB2EB0C0200FA0CF0AABF00EBC250A6
:101F200052421843BCBFD0401843704792F0000F94
:101F300081F4000106BF80F400000132013BB5E7E7
:101F40004FEA41037FEA226C18BF7FEA236C21D05D
:101F500092EA030F04D092F0000F08BF08467047C2
:101F600090EA010F1CBF0020704712F07F4F04D190
:101F7000400028BF40F00040704712F100723CBFA3
:101F800000F50000704700F0004343F0FE4040F4CD
:101F9000000070477FEA226216BF08467FEA23638B
:101FA0000146420206BF5FEA412390EA010F40F476
:101FB000800070474FF0000304E000BF10F00043C2
:101FC00048BF40425FEA000C08BF704743F09643A9
:101FD00001464FF000001CE050EA010208BF7047C4
:101FE0004FF000030AE000BF50EA010208BF70474B
:101FF00011F0004302D5404261EB41015FEA010C60
:1020000002BF84460146002043F0B64308BFA3F157
:102010008053A3F50003BCFA8CF2083AA3EBC25339
:1020200010DB01FA02FC634400FA02FCC2F1200258
:10203000BCF1004F20FA02F243EB020008BF20F08F
:102040000100704702F1200201FA02FCC2F12002F5
:1020500050EA4C0021FA02F243EB020008BF20EAEA
:10206000DC7070474FF0FF0C1CEAD0521EBF1CEA18
:10207000D15392EA0C0F93EA0C0F6FD01A4480EA06
:10208000010C400218BF5FEA41211ED04FF00063EF
:1020900043EA501043EA5111A0FB01310CF000401B
:1020A000B1F5000F3EBF490041EAD3715B0040EA41
:1020B000010062F17F02FD2A1DD8B3F1004F40EB11
:1020C000C25008BF20F00100704790F0000F0CF0E4
:1020D000004C08BF49024CEA502040EA51207F3AA8
:1020E000C2BFD2F1FF0340EAC250704740F4000083
:1020F0004FF00003013A5DDC12F1190FDCBF00F074
:1021000000407047C2F10002410021FA02F1C2F121
:10211000200200FA02FC5FEA310040F1000053EABD
:102120004C0308BF20EADC70704792F0000F00F00B
:10213000004C02BF400010F4000F013AF9D040EA11
:102140000C0093F0000F01F0004C02BF490011F4A5
:10215000000F013BF9D041EA0C018FE70CEAD153A3
:1021600092EA0C0F18BF93EA0C0F0AD030F0004C23
:1021700018BF31F0004CD8D180EA010000F00040D7
:10218000704790F0000F17BF90F0004F084691F095
:10219000000F91F0004F14D092EA0C0F01D14202CF
:1021A0000FD193EA0C0F03D14B0218BF084608D198
:1021B00080EA010000F0004040F0FE4040F40000E2
:1021C000704740F0FE4040F4400070474FF0FF0C75
:1021D0001CEAD0521EBF1CEAD15392EA0C0F93EABC
:1021E0000C0F69D0A2EB030280EA010C49024FEA0E
:1021F000402037D04FF0805343EA111143EA1013C7
:102200000CF000408B4238BF5B0042F17D024FF47E
:10221000000C8B4224BF5B1A40EA0C00B3EB510F59
:1022200024BFA3EB510340EA5C00B3EB910F24BF42
:10223000A3EB910340EA9C00B3EBD10F24BFA3EBC7
:10224000D10340EADC001B0118BF5FEA1C1CE0D18F
:10225000FD2A3FF650AF8B4240EBC25008BF20F042
:10226000010070470CF0004C4CEA50207F32C2BF96
:10227000D2F1FF0340EAC250704740F400004FF033
:102280000003013A37E792F0000F00F0004C02BF64
:10229000400010F4000F013AF9D040EA0C0093F02E
:1022A000000F01F0004C02BF490011F4000F013B88
:1022B000F9D041EA0C0195E70CEAD15392EA0C0FF0
:1022C00008D142027FF47DAF93EA0C0F7FF470AF28
:1022D000084676E793EA0C0F04D14B023FF44CAF6B
:1022E00008466EE730F0004C18BF31F0004CCAD100
:1022F00030F000427FF45CAF31F000437FF43CAF3C
:102300005FE700BF4FF0FF3C06E000BF4FF0010C5D
:1023100002E000BF4FF0010C4DF804CD4FEA40023F
:102320004FEA41037FEA226C18BF7FEA236C11D089
:1023300001B052EA530C18BF90EA010F58BFB2EB3C
:10234000030088BFC81738BF6FEAE17018BF40F0BC
:10235000010070477FEA226C02D15FEA402C05D170
:102360007FEA236CE4D15FEA412CE1D05DF8040BF5
:10237000704700BF844608466146FFE70FB5FFF788
:10238000C9FF002848BF10F1000F0FBD4DF808ED40
:10239000FFF7F4FF0CBF012000205DF808FB00BF31
:1023A0004DF808EDFFF7EAFF34BF012000205DF88B
:1023B00008FB00BF4DF808EDFFF7E0FF94BF0120D8
:1023C00000205DF808FB00BF4DF808EDFFF7D2FFD5
:1023D00094BF012000205DF808FB00BF4DF808ED18
:1023E000FFF7C8FF34BF012000205DF808FB00BFE5
:1023F0004FEA40024FEA41037FEA226C02D15FEAD2
:10240000402C08D17FEA236C02D15FEA412C02D133
:102410004FF0000070474FF0010070474FEA400254
:10242000B2F1FE4F0FD34FF09E03B3EB12620DD902
:102430004FEA002343F0004310F0004F23FA02F06C
:1024400018BF404270474FF00000704712F1610F13
:1024500001D1420205D110F0004008BF6FF00040EA
:1024600070474FF00000704742000ED2B2F1FE4FAD
:102470000BD34FF09E03B3EB126209D44FEA002353
:1024800043F0004323FA02F070474FF0000070471A
:1024900012F1610F01D1420202D14FF0FF307047BB
:1024A0004FF00000704700BF53B94AB9002908BF78
:1024B00000281CBF4FF0FF314FF0FF3000F06AB929
:1024C000ADF1080C6DE904CE00F006F8DDF804E08B
:1024D000DDE9022304B070472DE9F047089D0C4662
:1024E000002B4ED194468C458646B2FA82F262D9D0
:1024F0004AB1C2F12003914020FA03F30CFA02FC26
:10250000194300FA02FE4FEA1C471FFA8CF6B1FB92
:10251000F7F44FEA1E4307FB141143EA014304FB9F
:1025200006F199420AD91CEB030304F1FF3080F055
:102530001281994240F20F81023C6344591A1FFAFA
:102540008EF3B1FBF7F007FB101143EA014300FBE8
:1025500006F69E420AD91CEB030300F1FF3180F01E
:10256000FC809E4240F2F980634402389B1B40EAA3
:10257000044000211DB1D3400022C5E90032BDE86E
:10258000F0878B4205D90DB1C5E90001002108464D
:10259000F5E7B3FA83F1002946D1A34202D3904272
:1025A000C0F0F080861A64EB03030120002DE6D012
:1025B000C5E90063E3E7002A40F09080A1EB0C043A
:1025C0004FEA1C481FFA8CF70121B4FBF8F64FEADA
:1025D0001E4308FB164443EA044307FB06F09842F7
:1025E00008D91CEB030306F1FF3402D2984200F233
:1025F000CD8026461C1A1FFA8EF3B4FBF8F008FBB8
:10260000104443EA044300FB07F79F4208D91CEB40
:10261000030300F1FF3402D29F4200F2B080204653
:10262000DB1B40EA0640A5E7C1F120068B4022FAF9
:1026300006F71F4320FA06FC04FA01F343EA0C03F1
:10264000F44000FA01F8380C4FEA1349B4FBF0FEED
:102650001FFA87FC00FB1E4449EA04440EFB0CF9F8
:10266000A14502FA01F20AD93C190EF1FF3A80F0B5
:102670008480A14540F28180AEF1020E3C44A4EB7F
:1026800009041FFA83F9B4FBF0F300FB134449EA91
:10269000044403FB0CFCA44507D93C1903F1FF30AB
:1026A00067D2A44565D9023B3C4443EA0E40A0FBF7
:1026B0000293A4EB0C049C42CE469C4651D34ED0D0
:1026C00055B1B8EB0E0364EB0C0404FA06F6CB40EC
:1026D0001E43CC40C5E90064002150E7C2F120034D
:1026E00020FA03F10CFA02FC24FA03F394400C43A1
:1026F0004FEA1C4800FA02FE1FFA8CF7B3FBF8F011
:1027000008FB1031230C43EA014300FB07F1994217
:1027100008D91CEB030300F1FF362CD299422AD9C9
:10272000023863445B1AA4B2B3FBF8F108FB11331F
:1027300044EA034401FB07F3A34208D91CEB040459
:1027400001F1FF3613D2A34211D902396444E41ACD
:1027500041EA004139E70446F0E6084606E7C84585
:10276000AED2B9EB020E63EB070C0138A8E7314695
:10277000EDE7034699E73046D4E7D6467FE7634462
:1027800002384DE70646234608460FE7023E6344FB
:1027900030E700BF704700BF00487047001BB74BD1
:1027A00070B50C4601F030FB104E0546082130464E
:1027B00006F0AAF9012804D001F026FB431BA3422E
:1027C00007D30821094806F09FF9431E5842584193
:1027D00070BD72B60821304606F096F9012800D087
:1027E00030BF62B6BFF36F8FE0E700BF0004004860
:1027F00008B5002210214FF0904006F08BF90548F3
:102800000022202106F086F9BDE80840022001F0F0
:1028100003BB00BF0004004810B50C4C012210217E
:10282000204606F077F9052001F0F6FA204601224D
:10283000202106F06FF94FF090400122102106F0A0
:1028400069F9BDE81040022001F0E6BA0004004832
:1028500070B54FF090400C46164610210022144DE2
:1028600006F058F900232B701248B3B222462146D5
:1028700007F044FBD8B901F0C7FA41F287360446A5
:102880002B783BB1BDE87040012210214FF0904001
:1028900006F040B901F0B8FA031BB342F2D872B6A1
:1028A0002B7803B930BF62B6BFF36F8FE8E770BD16
:1028B0001507002078080020014B01221A7070478C
:1028C0001507002000487047905F030813B5114BAF
:1028D0000446186800909B88ADF804300120FFF78B
:1028E0009BFF062269460120FFF7B2FF0120FFF798
:1028F0007FFF9DF80430112B08D19DF80520122A86
:1029000004D101202370627002B010BD00231A466A
:102910001846F7E7601E03080CB4F0B5ADB032AB53
:1029200006AF53F8042B059305460E46384696210C
:102930002BF044FF9528C1BF42F62E63ADF8AA30B4
:102940002E23ADF8AC3000F037F83C24042D4FF4C2
:102950007A7E1449B0FBFEFCB0FBF1F14EF6602329
:10296000B0FBF3F3B3FBF4F204FB1232BCFBF4F361
:1029700004FB13C30EFB1C049ABF0B48405D3F20B1
:10298000CDE90040CDE9026708482BF097FE084BDF
:102990001B6898682BF0BCFD2DB0BDE8F04002B07C
:1029A000704700BF80EE3600EE5F0308CC5F03087F
:1029B0002405002001F030BA01F026BA1348144A69
:1029C00008B54FF00043C0E9002304224261012210
:1029D0000023C2614FF480510722C0E90233C0E9ED
:1029E0000933C0E90C1203610383837680F8203039
:1029F00080F82C30826380F83C30C36404F0DCFF44
:102A000018B1BDE8084000F08FBB08BD18070020D2
:102A1000002401400268084B9A4282B00AD14FF06C
:102A2000B0431A6E42F400721A661B6E03F4007310
:102A30000193019B02B07047002401400268054BDE
:102A40009A4201BF4FF0B042136E23F40073136635
:102A5000704700BF0024014030B585B00024054612
:102A6000CDE901440394FFF7A9FF144805F038FBB2
:102A700008B100F059FB1148039401A9CDE90154B4
:102A800005F0F8F808B100F04FFB0C4805F052FAD9
:102A900008B100F049FB4FF0FF31084805F08CF811
:102AA000064805F0FFFA054805F0E0F8044603483B
:102AB00005F0A2FA204605B030BD00BF180700207F
:102AC000014B024A1A607047180700200024014099
:102AD00008B50948FFF7C0FF68B1084BB3F8AA3042
:102AE0004FF6FF72934216BF40F6E442044B534345
:102AF000B3FBF0F398B208BD002000B40075FF1FCF
:102B0000D8084C0013B50023ADF80630FFF7E0FFFE
:102B100004461948FFF7A0FF184BB3F8C820B3F8D4
:102B2000A8108A4204FB00F018D040F6E443B0FB42
:102B3000F3F364205B1A4343521A93FBF2F31E3300
:102B40001BB2ADF80630BDF806305BB21B02ADF823
:102B50000630BDF8060000B202B010BD4FF47A7224
:102B600040F6FF73B0FBF3F35343A3F53923A3F50A
:102B70000C6340F6C412E0E7001000B00075FF1FC0
:102B80004FF0B04382B09A6A22F480529A629A6CF3
:102B900042F480529A649B6C03F480530193019B2E
:102BA000002002B070474FF0B04307B59A6C42F076
:102BB00004029A649A6C02F004020192019A9A6CDF
:102BC00042F001029A649B6C002203F0010311465B
:102BD00000930B20009B05F021FB0B2005F050FB20
:102BE000002211460C2005F019FB0C2005F048FBD3
:102BF000002211460D2005F011FB0D2005F040FBD1
:102C0000002202210F2005F009FB0F2005F038FB00
:102C100000221146102005F001FB102005F030FBCA
:102C200000221146112005F0F9FA112003B05DF8D9
:102C300004EB05F025BB000008B505F065FD10B1FB
:102C40006FF0040008BD064B9A6942F040429A6159
:102C50004CF2FA321A6105F069FD0028F2D0EFE774
:102C600000400058F0B585B000230D46009306469D
:102C7000A8B3FFF7E1FF044670BB05F045FD88BB34
:102C80001A481B4A02230193D0F8E01506F1784355
:102C900002EA8121B3FBF1F701FB1733DB0A029350
:102CA000D0F8E00505F178410139314402EA80228B
:102CB000B1FBF2F002FB1011C3EBD12301336946E3
:102CC00001A8039305F0B2FD20B1022814BF6FF0F4
:102CD0000104012405F02AFD204605B0F0BD6FF087
:102CE0000504F9E76FF00404F6E700BF0070FF1F6A
:102CF00000FCFF03014B1860002070477C07002098
:102D00002DE9F04FB0F1006F89B006460F469046AE
:102D1000C0F0C080DFF89091644DD9F8E03505EA45
:102D2000832303F10063013B984200F2B380002942
:102D300000F0B38040EA02035B0740F0AE80FFF78B
:102D40007BFF044690BB05F0DFFC002840F0A88024
:102D5000D9F8E015009705EA812106F17842B2FB27
:102D6000F1F301FB132208F17843013B3344B3FB39
:102D7000F1F001FB1033DB0A01334FEAD22AA3EB57
:102D8000D222012A039388BFC6F30A050AF58037C9
:102D9000C6F108038CBFC5F500654546FF02B34682
:102DA0000693039B9A4505D305F0C0FC204609B065
:102DB000BDE8F08FA6F10803069A1A4495421CD884
:102DC000009B04950193CDF814B04FF00009059BCA
:102DD00009EB0301049B99453DD3009BAB442B4475
:102DE000A8EB0505B5F5006F009328BF4FF400650B
:102DF0000AF1010A07F50067D3E753F8081F5A687C
:102E0000B2F1FF3F08BFB1F1FF3FD5D0284B1868A2
:102E100010B96FF00504C7E727B14FF400623946D7
:102E200011F090FFDFF888900099D9F80030CBF3CB
:102E30000A001844AAB211F085FF4FF40061384629
:102E4000FFF710FF00BBD9F8003001934FF4006387
:102E500005970493B9E7019B07914B440293012026
:102E6000D3E9002305F09CFC88B90799019BD1E9BF
:102E7000000259F80310029B5B689A4208BF88421F
:102E800005D109F10809A2E76FF001048CE76FF0A2
:102E9000030489E74FF0FF3488E76FF0050485E706
:102EA0006FF0040482E700BF0070FF1F00FCFF0307
:102EB0007C070020B1F1006F70B510D30B4BD3F835
:102EC000E0650B4B03EA862303F10063013B994263
:102ED00005D838B192B211F035FF002070BD4FF027
:102EE000FF30FBE76FF00500F8E700BF0070FF1F41
:102EF00000FCFF03B0F1006F10B40DD3084BD3F802
:102F0000E045084B03EA842303F10063013B984248
:102F100002D810BCFFF7A6BE4FF0FF3010BC7047C0
:102F20000070FF1F00FCFF034FF0B04382B0DA6C6B
:102F30000243DA64DB6C03400193019B02B07047EB
:102F40002DE9F04186B01422002101A82BF054FC99
:102F50000220464EFFF7E8FF0420FFF7E5FF0120BF
:102F6000FFF7E2FF4FF43A413046002205F0D2FD70
:102F7000002210214FF09040002405F0CBFD0125E8
:102F800002274FF40A4301A93046CDE901354FF03D
:102F90001008CDE9034705F097FC01A93046CDE9BB
:102FA0000185CDE9037405F08FFC202301A930468B
:102FB000CDE90135CDE9037405F086FC01A94FF098
:102FC0009040CDE90185CDE9034405F07DFC082260
:102FD0004FF4881301A93046CDE901234FF00308CF
:102FE000CDE9034705F070FC4FF4441301A94FF0FD
:102FF0009040CDE90183CDE9035705F065FC4FF41E
:10300000405301A93046CDE90135CDE9034805F02B
:103010005BFC4FF404134021CDE9011314480395E0
:1030200001A905F051FC22462146062005F0F6F8DC
:10303000062005F025F922462146072005F0EEF886
:10304000072005F01DF922462146092005F0E6F883
:10305000092005F015F922462146092005F0DEF881
:10306000092005F00DF906B0BDE8F0810004004824
:103070000008004800B59BB04822002108A82BF0AA
:10308000BBFB1822002102A82BF0B6FB05F05CFD6B
:103090004FF0B0420120D2F8903023F01803C2F86C
:1030A0009030D2F8003423F4C06343F40073C2F8C4
:1030B0000034D2F8003403F4C0630193019B24234D
:1030C000089381230B930023CDE91003B02208A8B5
:1030D000CDE9122305F0B0FE08B172B6FEE74F232A
:1030E000CDE90230CDE90400CDE90600022102A8B5
:1030F00006F03CF908B172B6FEE71BB05DF804FBC0
:1031000008B504F007FCFFF7B5FFFFF719FFFFF75D
:103110004AFD01F001F900F0B1FF00F07FF802F084
:103120007DFD02F082FDFCE772B6FEE700B58DB0D2
:103130002C22002101A82BF05FFB1748174B0360DE
:103140001F2383604FF080420023C0E90433C0E9AD
:10315000072383614FF48073436206F0ADFB08B12F
:10316000FFF7E2FF0C4806F0D3FC08B1FFF7DCFFE5
:103170004FF0005300220793074808924FF48073E2
:1031800001A9029206920B9306F0F6FB08B1FFF735
:10319000CBFF0DB05DF804FB800700200028004045
:1031A00010B5044690B03822002102A82BF024FB71
:1031B0002268194B9A422CD14FF48033029302A813
:1031C0004FF480730F9306F0F5F908B1FFF7ACFFE9
:1031D0004FF0B0430220D3F8902042F40042C3F8ED
:1031E00090209A6D42F480629A659B6D002203F4F0
:1031F000806311460193019B05F010F8022005F051
:103200003FF800222A20114605F008F82A2005F090
:1032100037F810B010BD00BF002800401148124A16
:1032200008B54FF48273C0E9002300234FF4E06235
:10323000C0E902324FF400712822C0E906120722C9
:10324000C0E90433C0E90833C0E90B2383620823D3
:10325000436306F0CDFD18B1BDE80840FFF764BF39
:1032600008BD00BF7808002000300140F0B50546D9
:1032700089B01422002103A82BF0BEFA2A68374B2C
:103280009A4269D14FF0B04302261A6E42F480523E
:103290001A661A6E02F480520292029ADA6C42F0B6
:1032A0000102DA64DA6C02F001020192019ADA6C2E
:1032B00042F00202DA64DB6C03F00203009305249F
:1032C000009B0327D02303A94FF09040CDE903369C
:1032D000CDE9067405F0F8FA2023CDE903364FF066
:1032E0009040002603A90794CDE905671C4C05F022
:1032F000EBFA1C4826620723C4E90003802320461A
:10330000C4E90266C4E90436C4E9066605F018F8A3
:1033100008B1FFF709FF144AAC65A562134C0823F6
:10332000C4E900231021002380222046C4E90213AF
:10333000C4E90423C4E90633236205F001F808B1A7
:10334000FFF7F2FE002222206C651146A56204F010
:1033500065FF222004F094FF09B0F0BD0030014069
:10336000180800201C00024030000240B80700206E
:103370007047000008B504F0E3FA044B0120C3F8DD
:103380008800BDE8084005F037BC00BF00040058C5
:1033900008B504F0DCFA01F0CFF8FFF7D1FDFFF734
:1033A00002FC00F06BFEBDE80840FFF737BF08B530
:1033B00004F0CDFAFFF7C4FDFFF7F5FBBDE80840C8
:1033C000FFF72CBF08B504F0BBFABDE808400121A7
:1033D000002005F0C1BB70477047FEE7FEE7FEE73F
:1033E000FEE7FEE77047704770477047014806F0F8
:1033F000B5BB00BF8007002008B5012005F098FB91
:10340000014B01221A7008BDDC080020022005F0E3
:103410008FBB082005F08CBB014805F007B900BF41
:10342000F80C0020014805F001B900BF1808002081
:10343000014805F0FBB800BFB80700207047000046
:10344000014805F0F3B800BFAC0D00207047000044
:10345000014806F041BF00BF78080020014808F08D
:1034600079B800BF0C0E0020014806F0ABB900BFD0
:1034700080070020014807F0C0B900BFE40C00201D
:103480002DE9F04389B080460020109E07908946C0
:1034900015461F46FCF7CCFEF0B9104CCDE9009064
:1034A000CDE9020407AB0E480593142304933A4672
:1034B000434629460068FCF785FF2346324604F15F
:1034C000140153F8044B42F8044B8B42F9D1079B8B
:1034D000337509B0BDE8F0830120FAE7F308002056
:1034E000805F03087FB5124C00253C2302A863755A
:1034F000CDE90255257500F031FC042303AA0094A0
:1035000012210C48FFF7BCFF0B49142220462BF078
:1035100063F90646B0FA80F040096075074B0090E9
:103520002A462946022011F007FB304604B070BD40
:10353000DD0800202A600308901A00200C600308B0
:10354000094B0A4A1B78003B18BF01231370084B34
:10355000084A1B78003B18BF01231370064A00235A
:103560001370064A137070471609002018090020CE
:1035700015090020170900200E0900201A09002053
:103580000022024B1146012011F0D6BA3C6003081C
:103590000022024B1146012011F0CEBA54600308FC
:1035A0000022024B1146012011F0C6BA6C600308DC
:1035B0000022024B1146012011F0BEBA84600308BC
:1035C0000022024B1146012011F0B6BA9C6003089C
:1035D000034A044840F24B23002107F031BE00BFEC
:1035E0001C090020580D0020132BF0B52DD81825EC
:1035F000102415FB0343194D00244FF0800C4CFAA6
:1036000004F6A3F11007314205EB470714BF4FF052
:10361000240E4FF0140EA7F806E0A3F1080730427D
:1036200005EB470714BF4FF0240E4FF0140E013482
:10363000324205EB4306A7F806E00CBF1427242707
:10364000082CF78003F10103D9D1054B1B781BB976
:10365000BDE8F040FFF7BCBFF0BD00BF1C09002073
:103660001B09002010B500240022E3B211461046C9
:103670000134FFF7B9FF142CF6D110BDF8B504469C
:103680000D46FFF7EFFF104F002604EB44043C20EB
:1036900000F0C2FB142E04D1BDE8F8400A2000F06F
:1036A000BBBB3B19385D9A78597812FB05F211FBC8
:1036B00005F110FB05F0F3B2D2B2C9B2C0B2FFF708
:1036C00093FF0136E3E700BF050000202DE9F0413C
:1036D0000646012090460F4600F09EFB1C4A10252E
:1036E0004FF0800C2B4600244CFA04F1A3F110009B
:1036F0000F4202EB400014BF4FF0240E4FF0140EA7
:10370000A0F806E0A3F108000E4202EB400014BF4F
:103710004FF0240E4FF0140E013418EA010F02EBA3
:103720004301A0F806E00CBF14202420082CC88018
:1037300003F10103D8D11835B5F5F87FD2D1054B87
:103740001B781BB9BDE8F041FFF742BFBDE8F0812F
:103750001C0900201B090020002238B505460C4634
:1037600010461146FFF7B2FF082D38D8DFE805F004
:1037700005080F13171B1E2123000022114601E02C
:10378000002221461046BDE83840FFF79FBF0022C7
:1037900011462046F7E7224600210020F3E70022E9
:1037A00021462046EFE722460021EBE7224621464C
:1037B000F3E72246E2E7002211462046FFF786FFA4
:1037C0004FF4967000F028FB002122460846FFF7D0
:1037D0007DFFBDE838404FF4967000F01DBB38BD4A
:1037E000024B1878024B1978FFF7B6BF0300002090
:1037F0000000002008B5FFF7F3FFBDE8084001F026
:10380000C7BA000008B5FFF7EBFF01214FF0904069
:1038100005F07AF9064B012816BF022218701A70BB
:103820001878044B1978BDE80840FFF727BF00BFA0
:103830000300002000000020F0B585B002AC204657
:1038400011F0DCFB94E80300754C764D2378012BD6
:1038500085E8030006D0744A13781BB1734B1978BE
:10386000052920D1724B1A6852B92968196071492B
:103870000A601B680093704B1146022011F05CF93E
:103880006E4A6F4D1378DBB20A2B33D8DFE813F0A2
:103890001F0025005B0061006A0086009700A300FE
:1038A000B000B000B0002178012904D1127812B91B
:1038B0001B78052BE4D05F4B1A68002AE0D12968F9
:1038C00019605B490A601B6800935E4BD4E75E4B4E
:1038D0001B78DBB25D490B700CE05C4B002119706A
:1038E000514B1B78012B5A4B14BF0721062119702D
:1038F00001232B701378574C574F012B05D0574E8F
:10390000327802F0FF03002A77D0504A0023137068
:1039100023703B70FFF7A6FE514F524E3B78524C3E
:103920002BB933781BB923780BB92B784BB14F4B9C
:1039300001221A7002F006F800233B7033702370E6
:103940002B7005B0F0BD38490978012908BF012363
:10395000C0E7237813B93D4B01211DE02378012BEB
:10396000C8D129E0237833B92F4B1B78012BD9B26A
:1039700001D1364B10E023783D49012B05D02A4B6D
:103980001B7813B10B78002BB4D1304B0220187088
:1039900009780029AED008211970ABE7237823B944
:1039A000214B1B78012BD9B2E3D02378012B03D014
:1039B0001D4B1B78002B9DD1244B0221ECE7237873
:1039C0001BB92C4B1B78002BC5D02378012BF3D0CF
:1039D000284B1B78C3E723781BB9144B1B78042BA7
:1039E000B9D02378012BE7D0104B1B78052BB7E714
:1039F0000E4B19780429F8D1ADE7327812B9134B80
:103A00001B78DBB223701C4B20781978FFF7A4FEDB
:103A1000337803B123782378DBB23B707CE700BFB7
:103A20000D0900202C180020180900200B09002087
:103A30003C18002038180020B4600308040000205F
:103A400012090020D7600308020000201909002095
:103A50001309002003000020070900201B09002093
:103A6000110900200E09002014090020341800203C
:103A7000170900200C0900200000002038B5FFF7CE
:103A8000AFFE0F4B1A78012A05D01A78022A02D00D
:103A90001B78042B0DD10B4D0B4CFFF751FD2A78F1
:103AA00023789A42094B05D100221A702B78DBB299
:103AB000237038BD01221A70FFF7BEFEF6E700BF83
:103AC0000400002018090020010000200E09002039
:103AD0002DE9F041FFF784FE2A4B1A78022A4FD9CC
:103AE0001B78072B4CD8284E284D294FDFF8A4808F
:103AF000FFF780FEFFF724FD33782A782649DFF8A8
:103B00009CC09B1A18BF01233B703378244ADBB258
:103B10002B70137808781B1A224818BF01230370F2
:103B20001378214ADBB20B709CF8003014781B1B11
:103B30001E4C18BF012323709CF80030DBB21370B9
:103B4000007823781A4C18431A4B187012780978A9
:103B50000A432270227898F80010521A18BF0122E6
:103B60001A70154A127812B100223A701A70FFF7D3
:103B700063FE3378DBB22B702378DBB288F8003039
:103B8000BDE8F081040000200D0900200A09002092
:103B9000110900200100002009090020150900205A
:103BA0001609002010090020080900200F09002034
:103BB000180900200E0900201B0900200248036894
:103BC0000021596307F0B6BB580D0020002270B5E4
:103BD0000E4B1146022010F0AFFF01240A252946A2
:103BE00020461435FFF7B8FDEDB2322000F014F98D
:103BF0006E2DF4D10134E4B2092CEFD10022BDE8DE
:103C00007040034B1146022010F096BFF760030886
:103C10002A610308054808B50823036006F00AFC7A
:103C200018B1BDE80840FFF77FBA08BDE40C0020DA
:103C30004FF0B04307B55A6E42F001025A665B6E10
:103C4000002203F00103019311463220019B04F08E
:103C5000E5FA322003B05DF804EB04F011BB00007C
:103C60000CB407B5054A05AB1021019311F074FBA4
:103C700003B05DF804EB02B0704700BF6061030859
:103C800030B585B0044602A80D4611F091F9BDF992
:103C90000C30064A00931021029B2046FFF7E0FFFC
:103CA0002046FDF7E5FB288005B030BD60610308C4
:103CB0004FF0B04210B5936823F40043936011F0C5
:103CC000FFF9104B01241C7000F0ACF810F0CAFE94
:103CD0000D4810F0E1FE0D4B4FF400421A61032035
:103CE00010F0E0FEFEF7ECFE00F002F910F0D4FF59
:103CF0002146204610F0F0FF21462046BDE8104046
:103D000010F0D4BFF00C0020813C000800400058A7
:103D100010F0F8BF08B5FEF7DBFE40F6B833984266
:103D20000CD8B0F5E16F0BD3FE23A0F5E16058434A
:103D30004FF49663B0FBF3F0C0B208BDFE20FCE781
:103D40000020FAE77FB5684600F0B6F80198FEF764
:103D500065FB00B207B05DF804FB0000194A38B5F6
:103D6000D2F88035591C044619D103F0F7FD0546F9
:103D700003F000FE054403F0F7FD2B0EE3712B0C5E
:103D8000A3712B0A6371030EE370C0F30742C0F303
:103D900007232571C0B2A2706370207038BD190A64
:103DA000C3718171190C1B0E41710371D2F88435F6
:103DB000C370D2F88405C0F30722C0F30743000E96
:103DC000E9E700BF0070FF1F38B5094BD3F8803515
:103DD00003600133054609D103F0C0FD044603F03A
:103DE000C3FD444003F0C6FD44402C6038BD00BF15
:103DF0000070FF1F0121022010F058BF0021022097
:103E000010F054BF00207047024B187808B100F042
:103E1000BFB97047F00C002082B00190019802B049
:103E200000F052BAF0B5224A224CD2F8903043F456
:103E3000804389B0C2F8903003F0A2FD03F0A8FDE2
:103E400003F0AEFD012304930323069300254FF0F6
:103E5000B04305950795DA6C42F00202DA64DA6C39
:103E600002F002020292029ADA6C42F00202DA6472
:103E7000DB6C03F0020301934FF4805703A9204643
:103E8000019B03974FF4005604F01EFD03A9204642
:103E9000039604F019FD2A463946204604F03AFEFE
:103EA0002A463146204604F035FE09B0F0BD00BF79
:103EB000000800580004004810B50446FEF722FE32
:103EC000074BA36040F30F20FEF778F8054B064A36
:103ED0002360064B6060C4E90323002010BD00BFCF
:103EE0000000484200007A440D093E00AB03050083
:103EF000002070470120704708B52AF0DFFC162328
:103F000003604FF0FF3008BD08B52AF0D7FC162338
:103F10000360FEE770B50D4614460E46731B9C42C7
:103F200001DC204670BDAFF3008006F8010BF5E719
:103F300030B5104600234FF06042834200DB30BDB5
:103F4000D2F8804EE50707D5D2F8004EE40703D536
:103F5000CC5C156815B114700133EEE700BFF8E7CB
:103F60004FF0FF3070474FF400534B600020704714
:103F700001207047002070470B4A116810B50346B6
:103F800009B90A491160106809490A4C0344091B20
:103F90008B4206D92AF092FC0C2303604FF0FF30CD
:103FA00010BD1360FCE700BFF40C0020403A002075
:103FB000000001200008000037B5184B02689A4243
:103FC000054628D14FF0B043154C1A6E42F40062FA
:103FD0001A661B6E134A03F400630193019B1723B7
:103FE000C4E90023102100238020C4E902134FF408
:103FF0008073C4E904034FF4806C2023C4E906C332
:1040000020464FF40053236204F09AF908B1FFF7F9
:104010008BF86C62A56203B030BD00BF002C01407C
:10402000F80C00200800024010B5044686B01422A7
:10403000002101A82AF0E0FB22680F4B9A4218D118
:104040004FF0B04301A9DA6C42F00102DA64DB6C94
:1040500003F0010300930222009B4FF48073CDE92B
:1040600001324FF090400123CDE90332059304F073
:104070002BFC06B010BD00BF002C014010B58EB067
:104080001022002103A82AF0B7FB00241C2221469D
:104090000DEB0200CDE9004402942AF0ADFB1F486D
:1040A0001F4B8460C0E900343B23C0E90334C0E9FE
:1040B000054406F00BFE08B1FFF736F84FF48053C5
:1040C0001648039303A906F01FFF08B1FFF72CF869
:1040D000124806F02BFE08B1FFF726F800240F481F
:1040E00002946946CDE9004407F026F908B1FFF7CC
:1040F0001BF8602309480D94002207A9CDE9073475
:10410000CDE90944CDE90B4406F078FE08B1FFF78C
:104110000BF80248FFF788FF0EB010BD580D0020C5
:10412000002C0140014B1868704700BFA40D00200F
:104130000320704708B501464FF47A7200238002CD
:10414000890DFEF7B1F908BD4FF47A73A0FB0303A4
:10415000800A40EA83507047034B98689A689042FF
:10416000FBD1C043704700BF0028004008B5FFF7EF
:10417000F3FF014B186008BDA40D002008B5FFF740
:10418000EBFF024B1B68C01A08BD00BFA40D002046
:10419000024B187808B1FFF7DFBF7047A80D002069
:1041A00010B5074B074C0122DA654FF480712046A9
:1041B00005F0CEFA4FF0FF332363002010BD00BF9F
:1041C000002800408007002002460021014805F039
:1041D000D6BC00BF8007002002460121014805F03F
:1041E000CEBC00BF8007002010B58CB02C2200216F
:1041F000044601A82AF000FBFFF7D2FF0C4B0D4844
:104200001B681C440023089306934FF00053E443BB
:10421000079301224FF4807301A902940B9305F0D8
:10422000ABFB08B1FEF780FF00200CB010BD00BF53
:10423000A40D00208007002038B50546FFF78CFF4D
:1042400002210446074805F0A1FCC4F309024FF41B
:104250007A71A2FB0121920AA30A2A8043EA8050C4
:1042600038BD00BF800700200148002105F08EBC4A
:10427000800700200148012105F088BC800700204C
:10428000F8B50F4D2E78CEB90E4C4FF0FF3727639F
:10429000FEF74CFFFFF784FF4FF48071204605F0D6
:1042A00057FA2046276305F015FC324620460221C6
:1042B00005F065FCFFF75AFF01232B700020F8BDC5
:1042C000A80D002080070020014610B54FF47A7237
:1042D00000238002890DFEF7E7F80146FFF73CFF57
:1042E0000446FFF739FF031B8B4200D310BD00BF0C
:1042F000F7E710F0EDBF000010B5064C0221204694
:1043000005F044FC0221421C2046BDE8104005F0A7
:1043100036BC00BF800700201648174A08B54FF486
:10432000E133C0E9002300230C22C0E90233C0E9D5
:104330000523C0E90733C0E90933036107F0EFFE45
:1043400008B1FEF7F1FE0B48002108F060F808B153
:10435000FEF7EAFE0748002108F079F808B1FEF7F9
:10436000E3FE044808F033F818B1BDE80840FEF752
:10437000DBBE08BD0C0E00200044004070B596B0B6
:1043800006461422002103A82AF036FA382200211A
:1043900008A82AF031FA3268274B9A424AD1022300
:1043A000089308A84FF440230A9305F003F908B1D5
:1043B000FEF7BAFE4FF0B04300259A6D1F4C42F451
:1043C00000329A659A6D02F400320292029ADA6C17
:1043D00042F00102DA64DB6C03F001030193019BFC
:1043E0000C220223CDE9032303A907234FF09040B9
:1043F0000793CDE9055504F067FA114925621423A6
:10440000C4E900131023C4E9023520468023C4E91F
:104410000435C4E9065503F093FF08B1FEF784FEA6
:104420002520F46700220221A66203F0F7FE252072
:1044300003F026FF16B070BD00440040AC0D002014
:104440008000024002680C4B9A4210B5044612D11B
:104450004FF0B0420C21936D23F4003393654FF07D
:10446000904004F0DDFAE06F03F0DCFFBDE810409F
:10447000252003F013BF10BD0044004008B50A46D4
:104480000146024806F0CAFF002008BD0C0E0020BD
:1044900013B5114B114C18604FF40013009302AB8D
:1044A00013E90600204607F036FF2368DA69D103D6
:1044B000FCD4DA695202FCD59A68084842F48002BA
:1044C0009A6007F06EFF06490448012207F0DCFEFF
:1044D000002002B010BD00BFA00E00200C0E002076
:1044E000A80E002008B5074B1860FEF75CFBFFF72D
:1044F00013FF054AD2F8803043F00063C2F88030E1
:10450000002008BDA40E00200008005808B54FF098
:10451000B04308489A6B42F400329A639A6B22F4D3
:1045200000329A63FFF78EFF112003F0B7FE0020E0
:1045300008BD00BF0C0E002008B5074807F0EFFDCE
:1045400008B1FEF7F1FD054803F0FAFE18B1BDE829
:104550000840FEF7E9BD08BD0C0E0020AC0D0020A0
:104560000268044B9A4203D1034B00201B68184792
:10457000704700BF00440040A40E002002680B4BAF
:104580009A4210B504460FD1094B1B682BB1D0F8E5
:10459000902012B907480121984720460549BDE8F7
:1045A0001040012207F070BE10BD00BF0044004063
:1045B000A00E0020A80E00202DE9F04F9DB0FEF7C0
:1045C00081F913F02DFB024640B90146644B0220ED
:1045D00010F0B2FA01201DB0BDE8F08F012013F0F9
:1045E000C7FB12F0C3F80446039040B902460146E7
:1045F0005C4B022010F0A0FA13F086FBEAE75A4D5C
:10460000296812F003FD6968204612F019FD297A25
:10461000204612F049FD697A204612F079FD696959
:10462000204612F005FEE868FDF71EFF81B2204625
:1046300012F088FD2969204612F050FDA97A204623
:1046400012F018FD0221204612F0CAFD102120466A
:1046500012F008FE039812F011F90246049040B9D6
:104660000146424B022010F067FA03A812F0DEF870
:10467000C2E703A812F0DAF8049812F067FC0246C9
:1046800040B901463A4B022010F056FA04A812F045
:1046900013FAB1E7374EDFF8E0A0DFF8E0B000230F
:1046A00033604FF00208049805AB0A2208A912F003
:1046B0003FFA054628BB02460146314B022010F066
:1046C0003BFA30682C49FDF7CDFC4FF07C51FDF7EB
:1046D000C9FC3060049812F069FC044604A812F08A
:1046E000EBF913F011FB002C3FF474AF002D3FF4F5
:1046F00071AF0022234B1146032010F01DFA002059
:1047000069E731680998FDF7A5FBBDF8189030609E
:1047100000221D4BCDF800901146022010F00CFA3B
:1047200008AC0027BBB2994504F1080405D8B8F1DC
:10473000010FC6D04FF00108B5E754F8040C5146FC
:10474000FDF790FCFDF790FE019034F8083C0093D3
:1047500000225B461146022010F0EEF90137E1E736
:10476000BC610308D461030820000020096203082B
:10477000306203084418002000007A449362030862
:1047800059620308AA6203088262030830B504462E
:1047900085B0084614491546FDF764FCFDF73EFE5A
:1047A000CCB1114902902846FDF75CFCFDF736FEBE
:1047B0000E4901902846FDF74BFB0D49FDF706FD1C
:1047C000FDF752FE002200900A4B1146032010F024
:1047D000B3F905B030BD0090074B224621460320B7
:1047E00010F0AAF9F5E700BF00007A44CDCC4C3FA9
:1047F000CDCCCC3EC3620308F06203082DE9F04F34
:10480000ADF22C4D4FF4007200210AA829F0F4FFFC
:104810004FF4007200218AA8BB4E29F0EDFF00255D
:1048200037464FF000082C46B9682046FDF712FBCA
:10483000796804462846FDF70DFB08F10408B8F531
:10484000007F054607F11007EED14FF0705120466A
:10485000FDF708FC4FF0705104462846FDF702FCB6
:104860000025A94F05904FF00008A946B8682146D9
:10487000FDF7EEFA0146FDF7F5FB01464846FDF768
:10488000E9FA059981467868FDF7E2FA0146FDF7F5
:10489000E9FB01462846FDF7DDFA08F10408B8F502
:1048A000007F054607F11007E0D14FF070514846F0
:1048B000FDF7D8FB4FF0705104902846FDF7D2FB6E
:1048C00005460498FCF740FF904B00222BF008FFB0
:1048D000FDF76AFA06902846FCF736FF8B4B00225C
:1048E0002BF0FEFEFDF760FA0DF128080790474611
:1048F0004FF0000A4FF00009B168B069FDF7A8FA5F
:10490000FDF78CFD0028B8BF4042FDF757FB47F884
:10491000040B01464846FDF79DFA0AF1040ABAF570
:10492000FE7F814606F11006E6D17949FDF74EFC7F
:104930000AAE83464FF000090027594656F8040B8B
:10494000FDF786FA0146FDF78DFB01464846FDF767
:1049500081FA0137BFB27F2F8146EED16C49FDF756
:1049600035FC8246FCF7F0FE0022684B2BF0B8FEC7
:10497000FDF71AFA8AAE0990B14600220027404698
:10498000D8F8001040680892FDF762FAFDF746FD7E
:104990000028B8BF4042FDF711FB089A49F8040B04
:1049A00001461046FDF756FA7B1C9FB27E2F08F198
:1049B00004080246E3D15749FDF708FC4FF000090F
:1049C00080460023414656F8040B0893FDF740FA51
:1049D0000146FDF747FB089B01461846FDF73AFAEA
:1049E00009F101091FFA89F9B9F17E0F0346E9D1EE
:1049F0004849FDF7EBFB8146FCF7A6FE434B00223E
:104A00002BF06EFEFDF7D0F94FF086410646584672
:104A1000FDF728FB4FF0864108905046FDF722FB3A
:104A20004FF0864183460998FDF71CFB4FF0864105
:104A300007464046FDF716FB4FF086418046484644
:104A4000FDF710FB4FF0864181463046FDF70AFB2B
:104A5000314906462046FDF705FBFDF7DFFC2E49F0
:104A600082460698FDF7FEFAFDF7D8FC2A49029027
:104A70000498FDF7F7FAFDF7D1FC00221146274B09
:104A8000CDE900A0012010F057F823490798FDF761
:104A9000E9FAFDF7C3FC204902902846FDF7E2FA47
:104AA000FDF7BCFC1C4901900598FDF7DBFAFDF70A
:104AB000B5FC002211461A4B0090012010F03CF882
:104AC0003846FDF7ABFC054602905846FDF7A6FCBC
:104AD00001900898DFF84CB0FDF7A0FC00221146C9
:104AE000114B0090012010F027F83046FDF796FC9E
:104AF00002904846FDF792FC01904046FDF78EFC7F
:104B000000220A4B009013E0D00F00200000E03F8D
:104B10000000FE420000FC4200007A4406630308E5
:104B20004E630308AE0E002094630308DA630308A3
:104B30001146ADB201200FF0FFFFABF80050834DDE
:104B40002868FCF701FE002200232BF09FFE804620
:104B500089462046FCF7F8FD42464B46FCF794FC9C
:104B60007B4BDFF8F081DFF8F091002221F000416B
:104B7000FCF742FEFDF7F0F880B2A8F800002868C4
:104B80007649FDF76FFAFDF749FC0022CDE900A058
:104B9000DFF8CCA1734B114601200FF0CDFF9AF83E
:104BA0000020BBF800309BB2CDE900230022114663
:104BB0006D4B01200FF0C0FF99F80020B8F80030CD
:104BC0009BB2CDE900230022684B114601200FF073
:104BD000B3FF9AF80020BBF80030DFF894A19BB235
:104BE0009A426BD299F80020B8F800309BB29A42F2
:104BF0000CD260492046FDF7F1FB38B101238AF859
:104C000000309AF800305C4ADBB213705B4BDDF881
:104C100010C01A88013292B21A801A8892B20A2AF7
:104C200004BF00221A801888554A1C2180B24843CC
:104C30001450188880B201FB0020C0F804C0188806
:104C4000DDF818C080B201FB0020C0F808C0188849
:104C5000DDF81CC080B201FB0020C0F80CC0188831
:104C6000DDF820C080B201FB0020C0F810C0188819
:104C70001B8880B201FB00209BB201FB032247612D
:104C80009AF8000010763046FDF7EEFB3D4BC0B2BF
:104C900018809AF80030012BD8B204D100223A4B88
:104CA00011460FF049FF2C609AF80030002B49D0D4
:104CB0000DF22C4DBDE8F04F00F012BD2E4F3B78A9
:104CC000012B5FFA83F8EED1DFF8B0902C4EB9F8E3
:104CD0000030B9F800204FF01C0B9BB292B20BFBD6
:104CE00003F30BFB0262F0589168FDF7B3F821461D
:104CF000FDF774FB88B102238AF800309AF800307F
:104D0000022B05D10022214B114640460FF014FF23
:104D10009AF80030DBB23B70C5E7B9F800302F6875
:104D20009BB20BFB03662046B168FDF793F839464A
:104D3000FDF754FB18B103238AF80030B3E78AF873
:104D40000000B0E70DF22C4DBDE8F08FB00E002052
:104D500000005940AC0E0020D602002000007A442A
:104D6000D702002020640308466403087B6403081C
:104D7000B50E0020CDCC4C3FB40E0020D017002043
:104D8000B80E0020AA0E0020B5640308FA640308D8
:104D90002DE9F04F99B0FDF795FD12F041FF024665
:104DA00040B90146A64B03200FF0C6FE012019B002
:104DB000BDE8F08F012012F0DBFF10F0EFFB04469E
:104DC0000C9040B9024601469E4B03200FF0B4FE02
:104DD00012F09AFFEAE79C4F3B78012BDDB253D0EB
:104DE000022D70D0002D3AD1042110F09DFF012139
:104DF000204610F0C7FE9549204610F0F7FE4FF010
:104E00007F51204610F0D8FE9149204610F086FED2
:104E10009049204610F09CFE0221204610F0B8FF79
:104E20008D49204610F09AFF214606A810F0F8FEA2
:104E30008A4A13928A4A14924FF07C53002212A994
:104E40002046129315921692179310F015FF2946DB
:104E5000204610F035FF0321204610F04BFF0C9840
:104E600000243C7010F030FC02460D9000286DD1FB
:104E70007C4B014603200FF05FFE0CA810F0FCFBFA
:104E80000DA810F0AFFCA3E7774E294610F07AFE8C
:104E90006E49204610F0AAFEB168204610F03EFE92
:104EA000F168204610F054FE716A204610F084FE2E
:104EB000F16C204610F052FF6C4B0022114601208D
:104EC0000FF03AFECBE7684D012110F05BFEE96977
:104ED000204610F08BFE696A204610F06DFEA9682E
:104EE000204610F01BFEE968204610F031FEA86C49
:104EF000FDF7BAFA81B2204610F04AFFE96C20466D
:104F000010F02CFF214606A810F08AFE2B6B12939E
:104F10006B6B1393AB6B1493EB6B15932B6C16931A
:104F200012A96B6C1793204610F0A6FEA86AFDF735
:104F30009BFAC1B2204610F0C3FE286AFDF794FA2E
:104F4000C1B2204610F03EFF494BB6E710F0E0FC3E
:104F500038B90022474B114603200FF0EDFD002029
:104F600025E70026DFF810A1444DDFF814914FF03B
:104F7000210837460D980EA910F022FD02460028A0
:104F800040F0888001463F4B03200FF0D5FDDFF84D
:104F9000EC800D9810F0DCFCB8F8003000229BB2D9
:104FA000114600930120384B0FF0C6FD0C9D0121E6
:104FB000284610F0E7FD0421284610F0B5FE2349ED
:104FC000284610F013FE4FF07F51284610F0F4FDF4
:104FD0001F49284610F0A2FD1E49284610F0B8FDD2
:104FE0000221284610F0D4FE1B49284610F0B6FED8
:104FF000294606A810F014FE184A1392234A159267
:105000004FF07C534FF07E5212A92846169212930D
:105010001493179310F030FE0021284610F050FE34
:105020000321284610F066FE0C990DA810F004FC30
:105030000246002866D10146154B02201BE700BF3F
:10504000BC6103083F65030840180020000082424D
:10505000CDCC4C3F00002040CDCCCC3E00002041C8
:105060000AD7233CC1650308D41700205F650308F5
:105070008F650308DC650308D4020020D2170020E6
:10508000D00F0020FA65030823660308CDCC4C3E00
:1050900058660308109A0F999DF83800FFF776FBC1
:1050A0009DF838305BB110993846FCF7D3FE0F9964
:1050B00007463046FCF7CEFE0134E4B206469AF8C5
:1050C0000030012B16D12B88109A9BB209EB0313E9
:1050D0009A602B880F9A9BB209EB03135A602B88B6
:1050E0009BB25A1C92B2802B2A8003D1FFF786FB19
:1050F00000232B800F20FDF75DFCB8F101087FF441
:1051000039AF44E70D9810F003FC00283FF421AFBD
:105110000CA810F0B1FADFF84CB1DFF84CA14FF059
:1051200021090D980EA910F04BFC054600285CD112
:10513000024601464D4B03200FF0FEFCB8F800304C
:10514000DFF82C9100229BB2114600930120494BBD
:105150000FF0F2FC032C94BF0023012389F80030E8
:1051600045493846FCF77EFF07462046FCF726FFF8
:10517000804601463846FDF729F83F490746304644
:10518000FCF770FF4146FDF721F83C4B1F603C4B9C
:10519000002118608046FDF7F9F80646A8B94223B9
:1051A000404699F80090CDE90343FDF737F90290A6
:1051B0003846FDF733F95FFA89F9CDE90090314BB4
:1051C0003246314601200FF0B7FC0D9810F0C0FBBD
:1051D00004460DA810F006FB12F096FD002C3FF4DB
:1051E000E5AD85F00100C0B2E1E5109A0F999DF898
:1051F0003800FFF7CBFA9DF838305BB1109938468C
:10520000FCF728FE0F9907463046FCF723FE0134D1
:10521000E4B206469BF80030012B1BD1B8F80030F1
:10522000109A9BB20AEB03139A60B8F800300F9AF9
:105230009BB20AEB03135A60B8F800309BB25A1CB9
:1052400092B2802BA8F8002004D1FFF7D7FA0023F0
:10525000A8F800300F20FDF7ADFBB9F101097FF48C
:1052600060AF6BE7D4020020D00F0020FA6503087E
:105270000D0900207866030800007A4428180020F1
:1052800024180020B06603082DE9F043ADB01423C4
:105290000DF10E0204A9ADF80E3012F049FF0446DC
:1052A00048B902460146194B03200FF045FC204641
:1052B0002DB0BDE8F0830022154B164FDFF8588063
:1052C000DFF85890114603200FF036FC0025BDF89A
:1052D0000E30AAB29342EAD9AAB22CAB03EBC202B7
:1052E000032012F89C6C52F8A03C002E14BF3A46E2
:1052F0004246CDE9003200224B4611460FF01CFC1D
:10530000002E05F1010508BF3446E0E70A670308EF
:105310002D67030800670308056703085167030842
:1053200030B5102289B00025294604460DEB020055
:10533000039529F061FA14F0A5FA2A46A34B0090D0
:10534000294603200FF0F8FBFDF7BCFA12F068FCC9
:105350008DF80C0012F00EFD431B18BF0123012134
:105360008DF80D30029012F023FD029812F0C2FE6B
:10537000029812F037FD0298FFF786FF002840F0F0
:10538000008102A812F006FD12F0BEFC029812F095
:1053900045FD029812F05EFD0298FFF775FF0028A8
:1053A00040F0F38002A812F0F5FC12F0ADFC029878
:1053B00012F06CFD0022864B114603200FF0BCFB5F
:1053C000029812F07FFD0298FFF75EFF002840F080
:1053D000E08002A812F0DEFC12F096FC029812F0B7
:1053E0008DFD002211467B4B03200FF0A5FB002210
:1053F000794B114603200FF09FFB029812F00AFE32
:105400000298FFF741FF002840F0C78002A812F081
:10541000C1FC12F079FC029812F018FE002211462D
:105420006E4B03200FF088FB00226D4B11460320CA
:105430000FF082FB029812F025FE0298FFF724FF7E
:10544000002840F0AE8002A812F0A4FC12F05CFC30
:10545000029812F033FE00221146624B03200FF037
:105460006BFB0022604B114603200FF065FB029896
:1054700012F060FD0298FFF707FF002840F09580CA
:1054800002A812F087FC12F03FFC029812F06EFDA9
:1054900000221146554B03200FF04EFB0022544BC7
:1054A000114603200FF048FB029812F07BFD029892
:1054B000FFF7EAFE00287CD102A812F06BFC12F084
:1054C00023FC029812F08AFD00221146494B03206A
:1054D0000FF032FB0022404B114603200FF02CFB53
:1054E000029812F097FD0298FFF7CEFE002864D1D3
:1054F00002A812F04FFC12F007FC029812F0A6FD71
:1055000000221146354B03200FF016FB0022344BCE
:10551000114603200FF010FB029812F0B3FD029821
:10552000FFF7B2FE00284CD102A812F033FC12F0B3
:10553000EBFB029812F0C2FD00221146294B03201A
:105540000FF0FAFA002211462B4B03200FF0F4FA69
:1055500001238DF8173003AB03CB002220601868BD
:1055600061600C23A060114600930320234B0FF0D1
:10557000E3FA02A812F00EFC12F0C6FB002009B0FC
:1055800030BD01238DF80E3000E701238DF80F3078
:105590000DE701238DF8103020E701238DF811303D
:1055A00039E701238DF8123052E701238DF81330CB
:1055B0006BE701238DF8143083E701238DF8153054
:1055C0009BE701238DF81630B3E700BF6767030838
:1055D00090670308C3670308F46703082368030898
:1055E0005068030885680308B8680308EB68030877
:1055F0001C6903084C6903087A690308A769030852
:1056000002480122102103F085BA00BF00040048BF
:1056100013B5124C237803F0FF023BB9104B11462F
:10562000032002B0BDE810400FF086BAFDF75AFF24
:1056300000380C4B18BF0120400018701A78022A5D
:1056400004BF002222701B7800930022064B1146F3
:1056500003200FF071FA02B010BD00BF901A0020B5
:10566000C66903081B090020E269030838B5164D16
:105670002B7803F0FF0233BB144C2368012B0CD9A9
:105680002368042B09D81146114B03200FF054FA5C
:10569000104A0421012000F093FF2368042B12D943
:1056A00000220D4B114603200FF046FAFDF71AFFBA
:1056B00000380A4B18BF0120400018701B78022BDD
:1056C00004BF00232B7038BD901A00206C180020F6
:1056D000F96903081E6A0308236A03081B090020EE
:1056E00070B500268AB03E4C02961C22314603A8B3
:1056F00029F082F82578022D6AD0032D14D0012DCF
:105700002AD035460195237800930022354B114667
:1057100001200FF011FA02AA2946152000F050FFCF
:10572000002323700AB070BD2F4E304A042333701B
:1057300013702F4B01221A702E4B30781978FEF718
:105740000BF833788DF808302B4B1B788DF8093027
:1057500023788DF80A30D5E7234E244A032333708B
:105760001370234B1D70234B30781978FDF7F4FF2D
:1057700033788DF80830204B20491B788DF809309C
:1057800023788DF80A300B880A229BB2B3FBF2F320
:1057900030338DF80B300B889BB2B3FBF2F102FB78
:1057A0001133174930338DF80C300B889BB2B3FBA3
:1057B000F2F330338DF80D300B889BB2B3FBF2F16E
:1057C00002FB11333033DBB28DF80E30072599E739
:1057D000064B054E35701D70054B01221A70C2E74D
:1057E000B50E0020566A03080300002019090020A6
:1057F0000D0900200000002004000020AE0E002053
:10580000AA0E002038B5324D324C287BFCF7D2FB73
:105810003149FCF727FCA060687BFCF7CBFB2E49E5
:10582000FCF720FCE060A87BFCF7C4FB2A49FCF7EE
:1058300019FC6062E87BFCF7BDFB2849FCF712FC11
:10584000274BE0642361287CFCF7B4FB6060687C34
:10585000FCF7B0FBA061A87CFCF7ACFBE061E87C46
:10586000FCF7A8FB2062287DFCF7A4FBA062687D02
:10587000FCF7A4FB1849FCF7F5FB2063A87DFCF7B7
:1058800099FB6063E87DFCF799FB1449FCF7EAFBA0
:10589000A063287EFCF78EFBE063687EFCF78EFB3E
:1058A0000D49FCF7DFFB2064A87EFCF787FB0A4963
:1058B000FCF7D8FB6064E87EFCF77CFBA064287FE3
:1058C000FCF778FB074BE06202221A7038BD00BF7C
:1058D0008C020020D4170020CDCCCC3D0AD7233C2D
:1058E000CDCCCC3E4018002038B5114D114C287B52
:1058F000FCF764FB1049FCF7B5FBA060687BFCF784
:105900005DFB0D49FCF7AEFBE060A87BFCF756FBA6
:105910000949FCF7A7FB6062E87BFCF74FFB0749EE
:10592000FCF7A0FB064BE06401221A7038BD00BFF3
:105930008C020020D4170020CDCCCC3D0AD7233CCC
:1059400040180020F7B5374D374C2B78374ADBB27B
:105950002370374B1B78DBB26370364B1B78DBB29E
:10596000A3701378DBB2E370334B1B78DBB2237187
:10597000324B1B78DBB263711378012B49D1304B6A
:10598000304E1868FCF770FD80B2E0803068FCF79C
:105990006BFD2D4B80B220811888376880B2FCF7F0
:1059A0000DFB3946FCF71AFD18B13068FCF75CFDB9
:1059B000C0B2A072254B1B7823743BB1244B1B88CB
:1059C000DBB26374234B1B88DBB2A37468460FF011
:1059D00015FB214A137803B3204B1968E9B1196804
:1059E000009B12785B1AC2EB0212B3EB820F17D93D
:1059F0001B4A012111701278D2B2E2749BB2194A8B
:105A0000A382082313702B7003B0BDE8F040FDF7AC
:105A1000E7BE0023E3802381CCE7114B00221A70FC
:105A200003B0F0BD03000020481800200D0900203D
:105A30000400002018090020170900200C0900208C
:105A400028180020241800203C000020B50E00205B
:105A5000AE0E0020AA0E0020D50200203C18002027
:105A60008F1A002019090020024B01220021032077
:105A70000FF062B8926A0308024B01220021032052
:105A80000FF05AB8C86A030808B50122074B002175
:105A900003200FF051F8FFF7B3FDFFF7B3FE044A00
:105AA00000231370034A137008BD00BF0E6B030878
:105AB000401800208D1A002010B50F4B0122002144
:105AC00002200FF039F80D4B04225A706321012295
:105AD00000241A709975DA75DC611C62DC749C8292
:105AE000FFF78EFDFFF7C8FFFFF7BEFFFFF7CCFF04
:105AF000034B1C7010BD00BF446B03084818002006
:105B00008D1A00201FB5114B11491C6858681A7A6C
:105B10005B7ACDE90223FCF7A5FAFCF7A5FC0C495A
:105B200001902046FCF79EFAFCF79EFC0022094BF0
:105B30000090114603200EF0FFFFFEF73DFD6420AC
:105B400004B0BDE81040FEF767B900BF2000002098
:105B500000007A447B6B030870B586B00D4604469E
:105B6000FFF74EFD01F0D6FEFDF7EAF99620FEF7AD
:105B700053F90026AE420AD101AB03CB1B88238127
:105B8000094B2060002261601A7006B070BDFEF7FC
:105B90001DF801A8FFF7C4FB41F28830FEF73CF97D
:105BA0000136FFF7AFFFE5E78D1A002030B585B06D
:105BB0000446002503A8ADF80C50FCF787FE70B131
:105BC0009DF80C309DF80D20237062702946CDE9B8
:105BD00000320320034B2A460EF0AEFF012005B031
:105BE00030BD00BFB06B0308022801D8FFF708BD25
:105BF00070470000022804D802480022102102F059
:105C000089BF704700040048022803D802481021C9
:105C100002F085BF704700BF0004004808B5FEF7DA
:105C200047F8BDE8084000F0CBBE4FF0FF300FF062
:105C3000CDB87047014BD870704700BF4C000020B2
:105C4000014B1874704700BF4C00002007B5064B8D
:105C500000221B5C00931146044B02200EF06CFFE7
:105C600003B05DF804FB00BFEF6B0308D56B0308BE
:105C700008B5002102200FF071F80A4B1B7803F0E1
:105C8000FF014BB9084B1A68042A05D81A6810207E
:105C900001321A600FF062F8BDE8084003480FF0C7
:105CA000C5BA00BF901A00206C180020F41900201B
:105CB000002101200FF052B813B5104A104C42F2E7
:105CC0001073002818BF03460E48236013600FF0BE
:105CD0005FFA21680B480FF0E3FA0A480FF0A6FAC2
:105CE00023684FF47A72B3FBF2F30022009311465B
:105CF000054B01200EF020FF02B010BDCC020020A9
:105D000048000020F4190020F36B030813B50F4C72
:105D10002060236813B942F2107323600C480FF01F
:105D200037FA21680A480FF0BBFA09480FF07EFAEB
:105D300023684FF47A72B3FBF2F30022009311460A
:105D4000044B01200EF0F8FE02B010BDD00200207E
:105D5000881800201F6C030873B50446002855D02E
:105D600090F90650002D58D12F48304E0FF010FA00
:105D70002A462F484FF4006102F0CCFE2A462946FD
:105D80002C4B02200EF0D8FEE379012B0CBF2A4BDE
:105D90002A4B2A46294602200EF0CEFE284DE379F2
:105DA00033702B682B602B680BB9264B2B60264871
:105DB0000FF0EEF9296824480FF072FA22480FF02C
:105DC00035FA00222B6800931146204B03200EF079
:105DD000B3FE1F4B1868FFF76FFF31781D4A1E4B4B
:105DE000012908BF13460022009311461B4B0120D6
:105DF0000EF0A2FE94F90530019394F9043000935B
:105E00000022174B114603200EF096FE00210220BF
:105E100002B0BDE870400EF0A1BF0022114B114648
:105E200002200EF089FEE5E7A01800208E1A00205F
:105E300000040048616C0308766C0308936C030847
:105E4000CC020020A086010070180020B06C03086E
:105E500048000020586C03085C6C0308EC6C0308D5
:105E6000246D03080B6D030808B50E4B1B78022B3D
:105E700003D1002108200EF071FF0B4800224FF4DF
:105E8000004102F047FE084800224FF4007102F082
:105E900041FEBDE80840044800224FF4006102F0D2
:105EA00039BE00BFB00000200004004802480022B4
:105EB0004FF4004102F02EBE0004004802480022C8
:105EC0004FF4007102F026BE000400480A46014962
:105ED000FCF7F0BF00F0030870B51F4801224FF433
:105EE000004102F017FE1C4801224FF4007102F03D
:105EF00011FE01224FF40061174802F00BFE174813
:105F00000FF046F906F004FF044650B10022144B8E
:105F1000114602200EF010FEBDE8704011480FF04F
:105F200085B9114D114B0246014602200EF004FEC8
:105F300001260F4B2E702246214602200EF0FCFD5A
:105F40000C4806F079FD2878314606F0CDFA034872
:105F50000FF06CF9E0E700BF00040048F4190020DE
:105F60004D6D0308DC190020B00000206B6D0308A4
:105F70007F6D03084C00002070B58AB0FDF7CAFEA3
:105F80000446FCF7A5FD0546FFF7DCFC23B203EB56
:105F900043039E4CFE2203EB4313B3FBF2F3DBB24D
:105FA000A3759B4B1A78042A00F22E81DFE812F0C9
:105FB0002D0005005F008D00CB0096494868002247
:105FC00002704868102646704868A678867048684F
:105FD000A47DC47048681B782C0A04714868457118
:105FE00049680395C87802908978019103EB83038F
:105FF000894903EB83030B4400931146874B01202F
:106000000EF09AFD06200AB070BD824B21785A68C6
:1060100011705A68617851705A68A17891705A6805
:10602000E178D1705A68217911715A68617951719A
:106030005A6879495379059313790493D378039374
:1060400093780293537803EB830303EB83030B44AE
:1060500001931378724A03EB830302EB430300229C
:10606000009311466F4B01200EF066FDCAE7694BA5
:1060700021785A6811705A68617851705A68A1780D
:1060800091705A68A17DD1705A68290A11715A68B5
:10609000614955715A680495D378039393780293B4
:1060A000537803EB830303EB83030B4401931378CF
:1060B0005B4A03EB830302EB430300220093114688
:1060C000594B01200EF038FD9CE7524B21785A685D
:1060D00011705A68617851705A68E1789170E2885D
:1060E0005968C2F30722CA705A68E188117122897F
:1060F0005968C2F307224A715A68218991714B4944
:106100005A680978D1715A68E38821899BB289B2AB
:10611000CDE903319378029353783F4903EB83032E
:1061200003EB83030B44019313783D4A03EB830392
:1061300002EB43030022009311463D4B01200EF079
:10614000FBFC08205FE7334D22786B6832491A70F8
:106150006B6862785A706B68A2789A706B68E278A4
:10616000DA706B6822791A716B6862795A71E38808
:106170006A68C3F3072393716B68E288DA71228936
:106180006B68C2F307221A7222895A72A27A9A7233
:10619000227CDA72E27C1A73A28AC2F307225A7353
:1061A000A28A9A735A7802EB820202EB82020A44B4
:1061B00001921B781A4A03EB830302EB430300228C
:1061C0001146009301201B4B0EF0B6FC6B68E28871
:1061D0002189A57AE089247C89B280B2CDE90704BF
:1061E000CDE9051592B204925A7903921A79029276
:1061F000DA7801929B78009300220F4B1146012020
:106200000EF09AFC0F20FEE60020FCE64818002065
:106210000400002040000020B10000209E6D030813
:1062200028020020F36D03086D6E03088F1A00200A
:10623000D86E0308646F0308A16F030800B5034616
:106240008DB000282CD0407802280AD003282AD00C
:10625000164B0022114602200DB05DF804EB0EF043
:106260006BBC1A7F0B92DA7E0A929A7E09925A7E52
:1062700008921A7E0792DA7D06929A7D05925A68F4
:106280000492DA68039293F914200292B3F912206F
:1062900001921B7C00930022054B11460EF04CFC32
:1062A0000DB05DF804FB034BD3E700BFB2700308E9
:1062B000C97003083B71030801284FF000020CBFAE
:1062C000024B034B114602200EF036BC5A710308F4
:1062D0006C71030808B5002140200EF03FFD054B0E
:1062E0001B782BB1BDE80840002102200EF036BD1E
:1062F00008BD00BF8E1A002008B506F012FD80B957
:1063000006F0D8F901280CD1BFF34F8F0549064B91
:10631000CA6802F4E0621343CB60BFF34F8F00BF43
:10632000FDE708BD00ED00E00400FA051FB50446D6
:10633000002837D00378002B34D001224FF40071AD
:106340001E4802F0E7FB1E480EF070FF00221146C7
:106350001C4B02200EF0F0FB94F91830039394F9D3
:106360000A300293237C0193E368009300221146D4
:10637000154B03200EF0E0FB0022144B11460320C6
:106380000EF0DAFB237A012B0ED1617A104A114B01
:10639000002918BF13460022009311460E4B03201C
:1063A0000EF0CAFB04B010BD00220C4B11460320B6
:1063B00004B0BDE810400EF0BFBB00BF00040048B1
:1063C000D018002085710308B6710308E77103082F
:1063D0008171030880710308F471030805720308D2
:1063E00038B504460D4607484FF40061FCF782FDBE
:1063F00030B92A4621460348BDE83840FCF780BC46
:1064000038BD00BF00F0030810B506F01FFD10F105
:10641000080F07D1064B0022BDE8104011460220AC
:106420000EF08ABB013001D1024BF4E710BD00BF72
:10643000137203082972030813B506F04FF90028F8
:106440005CD12F4C132323702E4B1A7802F0FF01DE
:10645000002A3BD0142222701870FFF78DFD00280F
:106460004CD0294B1B78012B88BF00206070274C33
:10647000637A63B106F01EF9012808D120460EF0B8
:1064800087FE234800224FF4006102F043FB214BBA
:106490001B48D978002206F037F90146D8B9012205
:1064A0001D4B10460EF048FB00241C480EF070FEF9
:1064B0001B4B1A481968A14238BF21460EF0F0FE66
:1064C000164802B0BDE810400EF0B0BE154B1A7869
:1064D000A2B11970C1E70631E6D106F0E5F804462D
:1064E0000028E1D001224FF47A730021B0FBF3F3CE
:1064F000104600930C4B0EF01FFBD6E702B010BD08
:10650000400000208C1A00201B090020A018002049
:10651000000400484C00002041720308F4190020D8
:1065200048000020341800205072030808B50848BD
:106530004FF4006102F0F3FA064B1B78012B05D0F3
:10654000BDE80840002180200EF008BC08BD00BF57
:106550000004004804000020054B01221A70054B7E
:106560001B781BB1002102200EF0F8BB704700BF62
:106570008C1A00208E1A0020022810B510D0402856
:1065800015D0012816D101464FF0904002F0BCFA18
:10659000094B187000210220BDE810400EF0DEBB50
:1065A00001464FF0904002F0AFFA044BF1E70021B2
:1065B0000420F1E710BD00BF1609002015090020D6
:1065C00073B505460C46164606F088F803460028C3
:1065D00046D000242D480EF0DBFD2D4B2B481968CA
:1065E000A14238BF21460EF05BFE284802B0BDE84C
:1065F00070400EF01BBE4A68F05CD0540133DAB232
:106600009442F8D8234B0D701A781B78012A88BF62
:1066100000244C700022CDE900341F4C1F4B114662
:1066200001200EF089FA637A63B106F043F801287D
:1066300008D120460EF0ACFD194800224FF400614D
:1066400002F068FA174B1848D978002206F05CF877
:10665000014638B9154B012203200EF06DFAB8E758
:106660001149CCE70631B4D106F01EF804460028E3
:10667000B0D04FF47A730122B0FBF3F30021009302
:1066800003200B4B0EF058FAA4E700BFF4190020CA
:10669000480000201B090020A01800206E7203088B
:1066A000000400484C000020400000204172030814
:1066B00050720308044B1B7823B9044A05210120BA
:1066C000FFF77EBF704700BF1B0900209F720308C1
:1066D00010B5002490B03C22214601A8009428F077
:1066E0008BF82C4B2022DA7219788DF8001059782B
:1066F0008DF8011099788DF80210D9788DF8031073
:1067000019798DF8041059798DF8051099798DF85B
:106710000610D9798DF80710197A8DF80810597A72
:106720008DF80910997A8DF80A108DF80B20214602
:106730000DF10B0258180131007B02F8010F1C29E2
:10674000F8D193F828208DF8282093F829208DF887
:10675000292093F82A208DF82A2093F82B208DF8F1
:106760002B200DF12B0100229818013290F82C00FB
:1067700001F8010F142AF7D107484FF40061FCF724
:10678000B9FB20B9044840226946FCF7B9FA10B0B9
:1067900010BD00BF8C02002000F8030810B50022D5
:1067A00004461146054B02200EF0C6F92046044966
:1067B000BDE8104040220EF0C5BA00BFA572030824
:1067C00000F8030810B5354C207963794D2BC0B221
:1067D00053D1C0EB001080000A2838BF0A204FF4C4
:1067E0007A7358432E4B1860FFF766FAA079E37965
:1067F0004D2BC0B249D1C0EB0010800001284FF4EE
:106800007A7338BF01205843FFF780FA237A254A6C
:106810002549DBB21370254B01221A70637A244A92
:10682000DBB2137094F82830224A03EB83035B0039
:10683000DBB2137094F829301F4A03EB83035B002B
:10684000DBB2137094F82B301C4A03EB83035B001C
:10685000DBB213700023E21892F82C20D2B2CA5493
:106860000133142BF7D1A378012B16D1E37A202B17
:1068700013D1BDE81040FFF71FB96379482B0ABF59
:106880004FF4616363795843A6E7E379482B0ABF65
:106890004FF46163E3795843B0E710BD8C020020E8
:1068A0004800002004000020901A0020030000206F
:1068B0001B090020D7020020D6020020D5020020AC
:1068C00010B590B000213C2201A8009127F094FF60
:1068D0004022374968460EF035FA9DF800203AB953
:1068E0009DF80100102803D19DF80210012914D051
:1068F000002211462F4B02200EF01EF9FFF7E8FE92
:106900002D48142200210EF027FA4FF47A70FDF77B
:1069100083FAFFF757FF10B010BD284B1A7058705C
:1069200099709DF80310D9709DF8041019719DF8A5
:10693000051059719DF8061099719DF80710D971CD
:106940009DF8081019729DF8091059729DF80A10E7
:1069500099729DF80B1001F03F01D972D87AD1B22B
:1069600088421BD89DF8282083F828209DF82920EC
:1069700083F829209DF82A2083F82A209DF82B20CF
:1069800083F82B200DF12B0100229818013211F809
:10699000014F80F82C40142AF7D1BAE701F14000EA
:1069A0006844194410F8340C08730132D6E700BF6C
:1069B00000F80308B9720308901A00208C02002026
:1069C000F0B58BB000240125052610231822CDE94F
:1069D0000332CDE90566784B02942246214603270F
:1069E000CDE90055022009940EF0A6F8734B0294ED
:1069F00022462146CDE9005702200EF09DF8CDE950
:106A0000016402266E4B00962246214630460EF067
:106A100093F86C4B009522462146CDE9017430462F
:106A20000EF08AF809A9204606F060F9099BC3F325
:106A300007220292C3F307421B0E019200932246E3
:106A4000614B214630460EF077F809A9284606F03A
:106A50004DF9099BDAB20392C3F307220292C3F302
:106A600007421B0E019200932246584B21463046A6
:106A70000EF062F8564B5748009422464FF4FA71D4
:106A80000EF028FB544B5548009422464FF4FA71FF
:106A90000EF020FB524B534800942A464FF4FA71F3
:106AA0000EF018FB2046FCF725F908B1FCF73CFB7B
:106AB0004D4B009400224FF4FA614C480EF00AFB53
:106AC0004B4A002101200EF005FA4A4A002102201B
:106AD0000EF000FA484A002104200EF0FBF9474A64
:106AE000002108200EF0F6F900F06EFE44494548FA
:106AF00006F0B2F8444805F09FFF3A480EF096FBC6
:106B0000424B0021187805F0EFFC41490094414BBD
:106B10000968414800220EF0DDFA3F480EF086FB7E
:106B2000FFF7CEFE3D4A002110200EF0D3F93C4A7B
:106B3000002120200EF0CEF93A4A002140200EF02C
:106B4000C9F9394A002180200EF0C4F9374A0021E2
:106B50004FF480700EF0BEF9354A00214FF40070FA
:106B60000EF0B8F9334A00214FF480600EF0B2F90C
:106B7000314A00214FF400600EF0ACF92F4A002199
:106B80004FF480500EF0A6F92D4B2E4819682E4B6D
:106B9000009401220EF09EFA2A480EF047FB2B4B80
:106BA0002B4819682B4B009401220EF093FA2848C9
:106BB0000EF03CFB0BB0F0BDF9720308397303080B
:106BC0005A7303087B7303089C730308BD7303089F
:106BD000BD5E0008D0180020AD5E0008B818002087
:106BE0002D650008A0180020695E0008DC1900204F
:106BF0003DC800083964000809640008D95E00082F
:106C000000000301640000204C000020B0000020C0
:106C100048000020715C0008F41900206D5600083F
:106C20007D3A0008D13A000805380008813500088F
:106C300091350008A1350008B1350008C1350008BC
:106C4000D002002088180020D5620008CC02002065
:106C5000701800205965000873B50D4D00262E6090
:106C6000FEF750FFC820FDF7D7F828683146FBF73C
:106C70008DFB04460028F3D12868FBF7CFFB054BBA
:106C800000902246214603200DF056FF02B070BD51
:106C900044180020E173030830B50024A5B07C221D
:106CA000214605A8049427F0A7FD53238DF8103042
:106CB00001254FF48873ADF81230ADF800408DF81F
:106CC0001450FDF727F8FE23B0FBF3F000EB400073
:106CD00000EB4010394B8DF8150022462146032069
:106CE0000DF02AFF6846FEF761FF9DF800309DF821
:106CF000012013430FD158238DF81630072430227A
:106D000080212F4827F078FD224604A92C4827F03F
:106D100009FE25B030BD0E238DF81630294B1868BA
:106D200059681B8901AC03C4294601A82380FEF7DA
:106D300013FF01AB03CB2388234CCDF81B10ADF818
:106D40001F30CDF81700FEF7DDFE2068FBF78CFB47
:106D50000A254FF47A7380B2B0FBF3F0B0FBF5F381
:106D600005FB130030308DF821002068FBF77CFB19
:106D7000642380B2B0FBF3F0B0FBF5F305FB130026
:106D800030308DF822002068FBF76EFB80B2B0FB3C
:106D9000F5F0B0FBF5F305FB130030308DF8230060
:106DA0002068FBF761FB80B2B0FBF5F305FB130035
:106DB00030308DF824001524A1E700BF14740308B7
:106DC0000C1A0020661E0308441800202DE9F04725
:106DD0000378592B94B0044640F06482052963D8A7
:106DE0004378443B162B5FD8DFE813F0A4015E0024
:106DF00080015E0088015E005E005E005E00C400EF
:106E00005E006B015E005E005E00FF015E005E00E2
:106E1000EE005E005E005E0017008678482E17D1F7
:106E2000BA4A14210120FFF7CBFB41F28830FCF76E
:106E3000F3FF0022B64B114603200DF07DFE40F615
:106E4000B830FCF7E9FF14B0BDE8F047FFF754BADB
:106E5000532E12D130228021AE4827F0CDFCFFF70F
:106E60001BFF41F28830FCF7D7FFAA4A1521012009
:106E700014B0BDE8F047FFF7A3BB432E17D10024A1
:106E800004A88DF8104005F04FFDA24A4C23137062
:106E9000102393709DF81030547001204133D0704E
:106EA00013710521FFF78CFB14B0BDE8F087442E69
:106EB000FAD1984C984DA670592323705A236370C9
:106EC000FFF7CAFE2868FBF7A9FA0022934B00904F
:106ED000114603200DF030FE2B228021601D27F08B
:106EE0008BFC00232670637001261023A370E670CC
:106EF0002671FCF70FFFFE23B0FBF3F000EB400020
:106F0000042300EB40106071A3712868FBF7ACFA12
:106F10000A274FF47A7380B2B0FBF3F0B0FBF7F3BB
:106F200007FB13003030E0712868FBF79DFA6423FB
:106F300080B2B0FBF3F0B0FBF7F307FB1300303087
:106F400020722868FBF790FA80B2B0FBF7F0B0FB34
:106F5000F7F307FB1300303060722868FBF784FA00
:106F600080B2B0FBF7F307FB13003030A07222466B
:106F70000B217CE78378303BDBB2092B94D8684C3B
:106F8000684A23702378DBB25372624A5923137024
:106F90004D23537023780321303301209370FFF782
:106FA0000FFB2378009300225F4B114601200DF068
:106FB000C3FDFFF78DFB23780BB1FCF753FB14B037
:106FC000BDE8F047FCF738BC8578482D1AD1514C04
:106FD000562323701023A37018230120002563710A
:106FE000224605230821A371E3716570E0702071CA
:106FF000FFF7E6FA4D4B00942A46114602200DF0A9
:107000009BFD51E7432D7FF44FAF00213C2205A8A3
:10701000049127F0F1FB04A8FFF7C0FB444B2122A9
:107020008021184627F0E8FB9DF8102000F80E2C70
:107030009DF8112000F80D2C9DF8122000F80C2C62
:107040009DF8132000F80B2C9DF8142000F80F5C1D
:1070500003460A21A0F10F04B2FBF1F001FB10225C
:1070600003F8092C9DF8152003F8082C9DF816202C
:1070700003F80A0CB2FBF1F001FB102203F8062C16
:107080009DF8172003F8052C9DF818209DF81B503B
:1070900003F8042C9DF8192003F8032C9DF81A20FE
:1070A00003F8070C03F8022C07A92A46184603F830
:1070B000015C27F037FC05F10F012246C9B201201F
:1070C000F0E6807839280CD83038C0B2FEF78CFD55
:1070D000104A2378137063785370A3789370032158
:1070E000C5E614B0BDE8F047FFF7E4BA8078392868
:1070F000F7D83038C0B2FEF77DFDE9E7807839284F
:10710000EFD83038C0B2FEF77FFDE1E72D740308F9
:10711000427403080C1A0020441800206474030809
:107120001B0900208C02002087740308B074030838
:107130001B1A00208378303BDAB2092AD1D8C578EF
:10714000303DEAB2092ACCD80179A1F14802D2B285
:107150000B2AC6D8AE4840FA02F2D007C1D40A22A0
:107160004D2902FB03553BD13C235D43A94B4FF412
:107170007A7068431860A84B1860FEF79DFDA74A17
:107180002378137063785370A3789370E378D37087
:107190000521237913710120FFF712FAA04B102269
:1071A00000261E705A7001229A70DA70A178303968
:1071B00001EB8100E178303901EB4001C9B219716E
:1071C00022795A71974A1278D2B21A72964A127874
:1071D000D2B25A72FFF77CFA944B009532460CE714
:1071E0004829C3D14FF46163BFE78378303BDAB2FB
:1071F000092A3FF676AFC578303DEAB2092A3FF654
:1072000070AF0179A1F14802D2B20B2A3FF669AF03
:107210007F4840FA02F2D2073FF563AF0A224D29B8
:1072200002FB035539D13C235D43814A4FF47A7305
:107230006B4313601068FEF769FD784A237813707A
:1072400063785370A3789370E378D3700521237922
:1072500013710120FFF7B4F9714B102200261E7044
:107260005A7001229A70DA70A178303901EB8100EE
:10727000E178303901EB4001C9B299712279DA71B4
:10728000684A1278D2B21A72674A1278D2B25A7227
:10729000FFF71EFA674B0095A0E74829C5D14FF4C8
:1072A0006163C1E7502B40F0B48102297FF6FCAD49
:1072B0004078A0F13003012B3FF6F6ADA378312BD7
:1072C0007FF4F2AD052936D1E378302B40F0D08041
:1072D000544D594E00232B702B7803F0FF0253B905
:1072E0002379303BDBB23370337800931146534B34
:1072F00002200DF021FC4C49514A00230B703378D9
:10730000DBB213702B78464ADBB213720B78DBB218
:107310005372FFF7DDF9414B22781A7062785A7088
:10732000A2789A70E278DA7022791A71FCF784FAFE
:1073300005213A4A9BE5082940F08E80E378462BE8
:1073400040F010812579A5F13000C0B2092800F283
:107350005E816179A1F13003092B00F25881A27995
:10736000A2F13003092B00F25281E379A3F1300638
:10737000092E00F24C8105EB85067600314D203652
:1073800001EB8101F6B249002E7020312E4E263AD3
:10739000C9B2D2B2317002EB82022C4903EB8303F3
:1073A00052005B000A802033294ADBB213701C4A6A
:1073B00082F828006379303BDBB282F82930A37968
:1073C000263BDBB282F82A30E379303BDBB282F82D
:1073D0002B302B782BB9337803F0FF020BB91D4B00
:1073E0001A70FFF775F90D4B22781A7062785A708F
:1073F000A2789A70E278DA7022791A7162795A71F9
:10740000A2799A71E279DA71FCF716FA082190E70D
:10741000DEF7FFFF48000020CC0200200C1A0020FD
:107420008C020020040000201B090020DA740308ED
:10743000D002002011750308020000204E750308D9
:1074400003000020D7020020D60200203C000020CC
:10745000D5020020D402002004292FD1E278A2F125
:107460003003DBB2092B11D9A2F14103192B0AD940
:10747000FFF720F90022854B1146012014B0BDE82A
:10748000F0470DF059BBA2F13703DBB280490B7016
:10749000804B21781970312199705870DA707C4BCB
:1074A0007D4A1B78DBB213727C4B1B78DBB25372C4
:1074B000FFF70EF9FCF7C0F904213AE71D294FD96F
:1074C000A61C0025DFF8D091DFF8D4A13746A846E6
:1074D00017F8012F303AD2B2092A3ED809EB05033A
:1074E00003201A731B7BCDE902533B780022CDE9C0
:1074F0000053114653460DF01FFB01351E2DE7D1F9
:10750000B8F1000FB4D1FEF77DF9624B50221A702A
:1075100000225A7010229A700122DA7003F8042FA8
:10752000203416F8012F03F8012FB442F9D15A4B39
:1075300000221A7010225A7001229A70DA70544A8E
:107540001278D2B21A72554A1278D2B25A721E22E8
:10755000DA72FFF7BDF82321EBE64FF00108CCE724
:10756000072985D900254C4FDFF8348102342E4697
:1075700014F8012F303AD2B2092A46D879190320DB
:107580000A730B7BCDE9025323780022CDE9005327
:10759000114643460DF0D0FA0135082DE8D1002EF2
:1075A0007FF466AFFEF7A0F93A4B3B4C50221A70BD
:1075B00010229A70002501225D70DA7003F8042F02
:1075C00062190135127B082D02F1300203F8012FF8
:1075D000F6D100225023114600930120314B0DF0CB
:1075E000ABFA00232370102363700123A370E370B0
:1075F000274B1B78DBB22372284B1B78DBB26372FC
:10760000E572FFF765F80D2193E60126C4E7002136
:107610008FE6412B7FF448AC4378432B7FF444AC96
:1076200016297FF441AC204D421C002312F8011FA3
:10763000E9540133142BF9D1FDF7EAFF1B4B5B7DB5
:10764000012B1ED114490023EA5CC8180133D2B2C1
:10765000142B80F82C20F7D1104B00221A701B78C5
:10766000DBB24B72FFF734F80A4A631E153413F885
:10767000011F02F8011B9C42F9D1064A1621FFF7AF
:10768000F6BB064B02221A70EEE700BFAD75030889
:10769000040000200C1A00208C0200201B0900208E
:1076A0006A75030892750308901A0020DD0800200F
:1076B000F0B5054689B00C46002957D03B48012259
:1076C0004FF4004101F026FA39480DF0AFFD26785D
:1076D0009EB3002D68D068682E7870B3032E0BD04F
:1076E000132E45D0022E28D16978012925D00B060A
:1076F00023D4FFF76BFB20E06B78012B07D10078D8
:10770000012802D0022800D008B905F0C7F80025EA
:107710000DF11F008DF81F5005F006F9254A4C2386
:107720001370102393709DF81F3055700120413362
:107730000521D0701371FEF743FF237C052B15D86C
:1077400094F90A20059294F9092004921A4A52F8F1
:107750002330039394F90830CDE901630022E368F4
:1077600000931146154B03200DF0E6F909B0F0BD6A
:107770006F78012FE1D1057815F001050CD12A466B
:107780000F4B294603200DF0D7F92A4607484FF43E
:10779000006101F0BFF9D0E700221146094B032038
:1077A0000DF0CAF93A46F1E72E46C6E70004004854
:1077B000B81800200C1A002038760308E575030875
:1077C000D2750308DC750308034B0022C3E90222CB
:1077D0000122C3E900227047A41A00200048704724
:1077E000A41A00204FF0B04382B0DA6C0243DA648E
:1077F000DB6C03400193019B02B070472DE9F0411F
:1078000086B000240220154D0594FFF7EBFF0420FD
:10781000FFF7E8FF124F03944FF4807601230DEB3E
:107820000001CDE901632846032304934FF4005877
:1078300001F04AF801A93846CDF8048001F044F877
:1078400022464146384601F065F92846224631462F
:1078500001F060F9204606B0BDE8F0810004004860
:1078600000080048032810B50ED8012810D868B9C0
:1078700002460B484FF4807101F04CF90022094890
:107880004FF4005101F046F9002010BD0122F0E74D
:10789000002203484FF4807101F03CF90122EEE729
:1078A000000400480008004802207047002070478C
:1078B00001207047002814BF16200F2070470000D9
:1078C0000D48854600F025F80C480D490D4A002367
:1078D00002E0D458C4500433C4188C42F9D30A4A85
:1078E0000A4C002301E013600432A242FBD326F0CD
:1078F000EBFFFBF705FCFEE7000001200000002085
:10790000F806002018DC0308F8060020403A0020A2
:10791000FEE7704710B5032000F06EFC01F07CFA22
:10792000064B18600F20FCF76DFA044618B9FBF7F8
:1079300053FD204610BD0124FBE700BFD802002004
:107940004FF0E022136923F00203136170474FF0F8
:10795000E022136943F0020313617047014BD3F82F
:10796000900570470070FF1F014BD3F894057047D6
:107970000070FF1F014BD3F8980570470070FF1F80
:10798000024A536843F0010353607047002004E04B
:10799000024A536843F0020353607047002004E03A
:1079A000024A536843F0040353607047002004E028
:1079B0008068C0F380007047F7B500230193044648
:1079C000002800F0E980856D25B9FBF723F8E5650F
:1079D00084F8545023689A68D00040F1A1809A68D6
:1079E000D10000F1B480A26D42F01002A265E26DF8
:1079F00042F00102E26501251846FFF7D9FFA26DAA
:107A000002F01002024340F0C980A26D206922F406
:107A1000817242F00202A2659A68D2075DD4226B9D
:107A2000A67E94F82CC0003A18BF01221703D4E9AF
:107A300002120A43217E42EA8132617E42EAC13269
:107A400042EA4632002842EA4C02B4BF20F000412C
:107A50004FF400113A430A4394F82010012903D14E
:107A6000002E76D142F48032616A21B1A66A01F417
:107A7000E07131430A43D968E66C21F4FE3121F408
:107A8000FF711143D96094F83C206168012A01F02C
:107A9000404C4CEA060609D1D4E910273A43324358
:107AA000A66C324342EA0C0242F001061F693E4ACC
:107AB0003A4032431A6121F00042B2F1804F0CD0BB
:107AC000B1F1004F09D0394ED6F8082701F47011F2
:107AD00022F470120A43C6F808275A69666BA16B34
:107AE00022F0070232435A615A6922F0700242EAD8
:107AF00001125A61002835D19A6A62F00F029A6227
:107B00005B6903F007039E423CD10023E365A36D4C
:107B100023F0030343F00103A365284603B0F0BD3F
:107B20009A68234922F0104222F0170242F0805254
:107B30009A60204A1268B2FBF1F2013252000192BF
:107B4000019A002A3FF44BAF019A013AF7E700256A
:107B500052E7A16D41F02001A165E16D41F0010105
:107B6000E16581E7B0F5001FCAD19A6AE269013A7E
:107B700092006FF00F0102F01C0201FA02F2216E76
:107B80000A43BCE7A36D23F0120343F01003A3657F
:107B9000E36D43F00103E3650125BEE7A36D43F008
:107BA0001003A365F8E700BF02FCFF1F002001409F
:107BB000400D0300D8020020F8B54569082D0446A1
:107BC0000E460AD00368DB68D80705D5A36D43F0DD
:107BD0002003A3650120F8BD0425FCF715F907462D
:107BE00023681A682A4220D0A26D42F40072A2656E
:107BF000DA6812F4406F14D1A27E92B91A681207A3
:107C00000FD51846FFF7D4FE20BB5A6822F00C02AD
:107C10005A60A26D22F4807222F0010242F0010249
:107C2000A265227EFAB10020D5E7711CD9D0FCF7FD
:107C3000EBF8C01BB04201D8002ED1D123681B68DD
:107C40002B40CDD1A26D84F8543042F00402A265DD
:107C50000320C0E7A26D42F02002A265E26D42F06F
:107C60000102E265DDE70C221A60DCE70368186CAC
:107C700070470000F7B50023019390F85430012BB2
:107C8000044600F0C08005680269012380F8543082
:107C90002846FFF78DFE002840F0AF80D1E9003084
:107CA000022822F004027ED0B2F1004FC3F3110E7D
:107CB00035D1AA6A42EA0E02AA628A68686902EAB3
:107CC000032222F07C4222F0FF0220EA03210A4331
:107CD000002B6A611DDA4D4A4D4DD2F80817AB42B0
:107CE00001F0E07043D10D0213D4D2F8083723F02D
:107CF000E073034343F40003C2F80837454B1A68A6
:107D0000454BB2FBF3F20C2302FB03330193019BBF
:107D100053BB0020002384F8543003B0F0BD226E22
:107D200000F01F074FF00F0C0CFA07FC6FEA0C066F
:107D300022EA0C0CBEF1000F11D1C3F38462BA40E9
:107D400042EA0C0222668008E26901309042B4D80F
:107D5000A86AC3F38362BA4006403243ACE793FAA1
:107D6000A3F2B2FA82F2EAE7019B013BCEE72B4D88
:107D7000AB420BD1C901CCD4D2F8083723F0E07361
:107D8000034343F08073C2F80837C2E7244DAB4287
:107D9000BFD14B02BDD4D2F8083723F0E0730343C0
:107DA00043F48003EFE7B2F1004F01BFAA6AC3F3C7
:107DB00011018A43AA62002BABDA154813498342AA
:107DC000D1F8082709D1D1F8083702F0A07223F0C2
:107DD000E0731A43C1F808279BE71048834204D197
:107DE000D1F8083702F44002F1E70D48834290D100
:107DF000D1F8083702F0C072E9E7A26D42F0200224
:107E0000A265184686E7022087E700BF00200140F0
:107E1000001000B0D8020020400D0300004000B860
:107E2000002000B4026838B504461046FFF7C0FDD4
:107E300008B9002038BD9368990707D4936823F0E8
:107E4000004323F0170343F010039360FBF7DCFFBC
:107E5000054623689B685B07EBD5FBF7D5FF401B06
:107E60000228F6D923689B685A07F2D5A36D43F020
:107E70001003A365E36D43F00103E3650120D9E737
:107E800073B50023026801939368DD07044602D5A9
:107E9000002002B070BD9168214B194209D0A36D3A
:107EA00043F01003A365E36D43F00103E365012094
:107EB000EFE7936823F0004323F0170343F0010337
:107EC0009360184BD3F8083718021CD4637E012B3B
:107ED000DED0FBF799FF144E054622681368DB07D6
:107EE000D6D49368D9075FBF9368334043F001034A
:107EF0009360FBF789FF401B0228EED923681B68BB
:107F0000DA07EAD4CBE7094B094A1B68B3FBF2F363
:107F100001330193019B002BD8D0019B013BF8E773
:107F20001700008000200140E8FFFF7FD8020020FA
:107F3000400D030038B504460068FFF739FD0546DB
:107F400020BB94F85430012B20D0012384F8543006
:107F50002046FFF795FFB0B9A36D226823F4706344
:107F600023F0010343F48073A3651C23E0651360D1
:107F700084F85400936823F0004323F0170343F080
:107F80000403936038BD84F85450FBE70220F9E7FE
:107F9000026838B5936891680446C80701D4002088
:107FA00038BD9907FBD4936803F00503012B19D161
:107FB000936823F0004323F0170343F00203936018
:107FC00003231360FBF720FF054623689B68DB074C
:107FD000E5D5FBF719FF401B0228F6D923689B68FB
:107FE000DA07F2D5A36D43F01003A365E36D43F008
:107FF0000103E3650120D3E770B5044600284BD0A8
:10800000836D43F002038365FFF70CFF054668B9F3
:108010002046FFF7BDFF054608B90123A365226886
:10802000936823F0104323F01703936023685A6882
:1080300022F4677222F003025A6040F29F321A6003
:10804000D968164A0A40DA601A6922F040421A6179
:108050005A6922F007025A611A6A02F0F0221A6283
:108060005A6A02F0F0225A62DA6A02F0F022DA6208
:108070009A6A0B4A00269E62D2F8083723F0FE73F4
:10808000C2F808372046FAF7D9FCE6652666A665E9
:1080900084F85460284670BD0125FBE700023E834A
:1080A0000020014010B590F85430012B044615D043
:1080B000012380F85430FFF7B5FE58B92046FFF78A
:1080C00067FF38B9A36D23F4807323F0010343F0F5
:1080D0000103A365002384F8543010BD0220FCE79F
:1080E000F7B50023019390F85430012B04467FD05C
:1080F000012380F85430FFF74BFF23689A6812F091
:108100000102054607D0A36D43F01003A3650023C9
:1081100084F854302DE0A16D364F21F4817141F087
:108120000201A165DE68D96826F4FF4626F07C06C8
:1081300021F40041360421F00301360CD9600820F7
:108140009968394041F0004199609968002913DA33
:108150000199013101910199B1F52E3FF5D3A36D3C
:1081600023F0120343F01003A365002384F8543076
:108170000125284603B0F0BDD3F8B410013801F052
:108180007F010A44DCD199681A48014041F001019D
:108190009960D3F8B41021F07F0141EAD202C3F80C
:1081A000B4209A68024042F002029A60FBF72CFE6B
:1081B000074623689A68D20708D4DA683243DA603F
:1081C000A36D23F0030343F001039FE7FBF71CFEBD
:1081D000C01B0228EDD923689B68D907E9D5A36D98
:1081E00043F01003A365E36D43F00103E365BFE7CC
:1081F0000225BEE7E8FFFF7F0749CA6822F4E06274
:108200000302120403F4E063120C134343F0BF6350
:1082100043F40033CB60704700ED00E0164B30B5FF
:10822000DC68C4F30224C4F10703251D042B28BF16
:108230000423062D4FF0FF358CBF033C002405FAC4
:1082400003F321EA0303A54022EA0502A340002824
:1082500043EA0203ACBF00F16040084A4FEA03134F
:10826000B8BF00F00F00DBB2AABF00F561401354A5
:1082700080F8003330BD00BF00ED00E014ED00E0F9
:10828000002807DB044A4109012300F01F00834056
:1082900042F82130704700BF00E100E000280CDB0D
:1082A0004309064900F01F0020330122824041F8B3
:1082B0002320BFF34F8FBFF36F8F704700E100E0C3
:1082C00070B5D0E913456560446D14B1D0E9164529
:1082D0006560D0E9105404F01C060124B4406C60C1
:1082E000046863608368102B0BBFA260A160E1602B
:1082F000E26070BD0268416CD3B210B5083B142433
:10830000B3FBF4F30B4CA24288BF0B4A21F00301EC
:1083100099BF01F1804202F502325218073382649C
:10832000064AC26403F01F03012202FA03F3036545
:1083300010BD00BF070402401C0802408008024034
:1083400038B500285CD002682E4B9A424FF01401D9
:108350004AD82D4B1344B3FBF1F32C499B00C0E9E1
:108360001013022380F825301368056923F4FF43B6
:1083700023F070031360D0E9024323432B43456984
:1083800011682B4385692B43C5692B43056A2B4331
:108390000B431360FFF7AEFFB4F5804F04BF00231B
:1083A00043604368816C03F07F020A60D0E91314D4
:1083B000013B032B4C601ED8154B164981651344B5
:1083C0009B000121013A01FA02F200214365C265D6
:1083D0001960114B5A6400230122C36380F82430D2
:1083E00080F82520184638BD0C4B1344B3FBF1F33D
:1083F0000B499B00B3E70023C0E91533C365EAE7E7
:108400000120F0E707040240F8FFFDBF0000024032
:108410003F8200104009024000090240F8FBFDBF06
:108420000004024038B5002841D00268136823F0E8
:10843000010313601F4B9A424FF0140130D81E4BBA
:108440001344B3FBF1F31D499B00C0E91013012451
:1084500003F01C0304FA03F3002515604B60FFF7DB
:1084600049FF836C41681D60D0E913325A604A1E8F
:10847000032A06D8124B0B449B0094401D60114BFD
:108480005C640023C363C0E91533C0E90B33C0E962
:108490000D33C36580F8253080F82430184638BD88
:1084A000094B1344B3FBF1F308499B00CDE70120CE
:1084B000F5E700BF07040240F8FFFDBF00000240DF
:1084C0003F82001000090240F8FBFDBF000402409B
:1084D00070B590F82450012D04463BD090F82560EB
:1084E0000125AE4280F824504FF000062CD1022521
:1084F00080F825500568C6632E6826F001062E60B8
:10850000FFF7DEFE036BBBB12B6843F00E032B605D
:10851000A36C1A68D20342BF1A6842F480721A60D0
:10852000636D1BB11A6842F480721A602B6843F0C5
:1085300001032B60002070BD2B6823F004032B6027
:108540002B6843F00A03E2E78023C36380F82460CA
:108550002846F0E70220EEE7034640B190F82520D8
:10856000022A06D00422C263002280F824200120BF
:1085700070470268806C116821F00E01116001687B
:1085800021F480710160116821F001011160D3E9CB
:10859000100202F01C0101228A404260D3E913213B
:1085A00051605A6D32B1116821F480711160D3E9C4
:1085B000162151600122002083F8252083F8240031
:1085C000704708B590F82530022B03D00423C3630D
:1085D000012008BD03681A6822F00E021A601A68AA
:1085E00022F001021A60826C136823F48073136016
:1085F000D0E9101303F01C02012393404B60D0E933
:1086000013325A60436D33B11A6822F480721A60D3
:10861000D0E916325A60012380F82530002380F813
:108620002430836B03B198470020D2E770B4426CCA
:10863000046C036826681D6802F01C020421914046
:1086400031420FD015F0040F0CD01A6892065EBFAD
:108650001A6822F004021A60036B6160002B33D0A9
:1086600070BC184702219140314217D015F0020F1B
:1086700014D01A68940606D41A6822F00A021A6006
:10868000012280F82520114A93428CBF104B114BD8
:108690005960002380F82430C36ADFE70821914045
:1086A000314211D029070FD5196821F00E01196048
:1086B000012303FA02F26260C36380F825300023CD
:1086C00080F82430436BC9E770BC704780000240DB
:1086D00000040240000002400A4A536943F4802328
:1086E00030B55361EFF3108472B60023CD58C550F6
:1086F0000433B3F5807FF9D11369DB03FCD484F331
:10870000108830BD00400058064B5A69002ABFBF90
:10871000054A9A6002F188329A60BABF5869C00F60
:10872000002070470040005823016745044B5A69F8
:1087300042F000425A615869C043C00F704700BF01
:108740000040005870B50546FBF75EFB124E04462C
:108750003369D90313D43369DA0744BF0122326184
:108760004CF2FA32134011D10B4E306910F48020D4
:108770000BD0FBF749FB001BA842F6D304E0FBF744
:1087800043FB001BA842E3D3032070BD024A1361E0
:10879000024A01205360F8E700400058B41A002054
:1087A0002DE9F041184D98462B78012B06460C46D2
:1087B000174626D001232B704FF47A7000236B608C
:1087C000FFF7C0FFA0B9012E16D1104A536943F03C
:1087D000010353612760BFF36F8FC4F804804FF427
:1087E0007A70FFF7AFFF094A536923EA0603536122
:1087F00000232B70BDE8F08139462046FFF76CFF5F
:10880000EDE70220F6E700BFB41A00200040005850
:10881000054A536923F47E7343EAC00040F4803074
:1088200040F0020050617047004000582DE9F041CF
:10883000234F3B78012B054688463FD001233B70F0
:108840004FF47A7000237B60FFF77CFF044688B901
:108850002B68042B13D11B4A536943F4803343F034
:10886000040353614FF47A70FFF76CFF0446154B15
:108870001A681B6800233B702046BDE8F0814FF06A
:10888000FF33C8F800306E68D5E901321344B342B3
:108890000AD93046FFF7BCFF4FF47A70FFF752FF5A
:1088A00050B1C8F800600446064A536923F47E7349
:1088B00023F002035361DAE70136E5E70224DBE740
:1088C000B41A0020004000582DE9F04F524C00230C
:1088D0004FF00F090A6832FA03F501D1BDE8F08FB5
:1088E000012505FA03F818EA020200F08E804E68AE
:1088F000032706F003054FEA430E07FA0EFC6F1E2E
:10890000012F6FEA0C0C32D8876807EA0C0ACF688F
:1089100007FA0EF747EA0A078760476827EA080858
:10892000C6F300179F4047EA08074760C76807EA91
:108930000C088F6807FA0EF747EA0807022DC76090
:1089400017D14FEAD30800EB880803F0070AD8F8DC
:1089500020704FEA8A0A09FA0AFB27EA0B0B0F6913
:1089600007FA0AF747EA0B07C8F8207001E0032D61
:10897000DCD1076805FA0EF507EA0C073D4316F44B
:10898000403F056041D023F0030707F1804707F51A
:10899000803703F0030CBD684FEA8C0C4FF0070ED4
:1089A0000EFA0CFEB0F1904F25EA0E0E2FD01B4DA3
:1089B000A8422ED005F58065A84214BF07250225E0
:1089C00005FA0CF545EA0E05BD602568D74316F497
:1089D000801F0CBF3D4015432560656816F4001FDD
:1089E0000CBF3D4015436560D4F8805016F4803FBD
:1089F0000CBF3D401543C4F88050D4F88450B603F2
:108A000054BF3D401543C4F88450013362E700254C
:108A1000D6E70125D4E700BF00080058000400484D
:108A2000374A2DE9F04F00234FF0010A4FF0070BB2
:108A30004FF00F0931FA03F401D1BDE8F08F0AFAC3
:108A400003FC1CEA010654D023F0030404F1804423
:108A500004F5803403F00307A568BF000BFA07F89C
:108A6000B0F1904F08EA050E45D0264DA84244D0FB
:108A700005F58065A8420CBF02250725BD40754558
:108A800017D1D2F8805025EA0605C2F88050D2F8F6
:108A9000845025EA0605C2F88450156825EA0605C3
:108AA0001560556825EA06055560A56825EA08059C
:108AB000A560056803265C0006FA04F423FA06F6AE
:108AC000254300EB8606056003F00705376AAD0015
:108AD00009FA05F527EA05073762856825EA0405DE
:108AE0008560456825EA0C054560C56825EA0404EB
:108AF000C46001339EE70025C0E70125BEE700BF43
:108B000000080058000400480369194214BF0120FE
:108B1000002070470AB181617047816270474369E4
:108B200001EA030221EA030141EA0241816170473F
:108B3000044AD168014208B502D0D060FDF71CFD9F
:108B400008BD00BF00080058024A136843F4807350
:108B500013607047000400580D4B10B55B690C465C
:108B600028B99A0507D500F027F820B110BD9B055C
:108B700001D400F019F8074A1369012C23F004030B
:108B8000136101D130BFF1E740BF20BF20BFEDE747
:108B90000004005800ED00E0024B186800F4C060CB
:108BA000704700BF00040058024A136843F4804332
:108BB00013607047000400580C4A136823F4804384
:108BC00013600B4B1B6832214B430A49B3FBF1F393
:108BD0005169890500D533B9536913F4007F14BF77
:108BE000032000207047013BF2E700BF000400585B
:108BF000D802002040420F000B4A136823F00703FD
:108C000043F002031360094B1A69012842F0040281
:108C10001A6105D130BF1A6922F004021A61704747
:108C200040BF20BF20BFF6E70004005800ED00E081
:108C30004FF0B0431868C0F3404070474FF0B04366
:108C40001868C0F3400070474FF0B042536823F4F7
:108C50007F4343EA0023536070474FF0B0431868E6
:108C6000C0F34060704700007FB54FF0B0432C4A1E
:108C7000D3F80831C0F3031003F00F0352F820407B
:108C8000284A52F82330B4FBF3F4FFF785FF264B54
:108C9000054693E80700B5F5007F04AB03E907003C
:108CA00010D0224B9C4218D303F5B70303F67F5331
:108CB0009C4229D903F5741303F510639C4225D80F
:108CC00002230BE01A4B9C4207D91A4B9C421BD93A
:108CD00003F5370303F5D853F0E7002304AA02EBAA
:108CE000830353F80C4C144D2B6823F007032343E4
:108CF0002B60FBF789F806462B6803F007039C42BC
:108D000006D1002004B070BD0123E7E70024EAE7A4
:108D1000FBF77AF8801B0228EED90320F2E700BFA8
:108D200050760308B0760308701E0308C0CF6A00AF
:108D3000BFEA21013F933402004000584FF0B04396
:108D400010B59A68D96812F00C0205D00C2A4AD1E5
:108D500001F00303012B51D14FF0B0412B480B68B8
:108D600013F0080306D00B6813F0080337D1D1F8CD
:108D7000941007E00C68240756BFD1F894300968B6
:108D8000C3F3032350F82330002A0CBF18460020F9
:108D90004FF0B0418A6802F00C020C2A1ED1CA685A
:108DA00002F00302022A2ED0032A06D10B68184AC9
:108DB00013F4801F174B18BF13464FF0B042D06812
:108DC000D168D268C0F306205843C1F302130133BF
:108DD000B0FBF3F0530F0133B0FBF3F010BD0B68A1
:108DE000C3F30313CEE7042A05D0082A06D11B6873
:108DF00013F4801305D006480023C9E70023184662
:108E0000C6E70448C4E7024BD7E700BF5076030823
:108E10000024F4000048E80108B5FFF78FFF4FF089
:108E2000B043044A9B68C3F3031352F82330B0FBEA
:108E3000F3F008BDB07603082DE9F04104460028A0
:108E400053D04FF0B0439D68DE6803689B0605F081
:108E50000C0506F0030668D5026A1DB10C2D46D13B
:108E6000012E44D1002A40D04FF0B043A16A1A68C5
:108E7000170756BFD3F894301B681B0903F0F003A3
:108E800099421FD90846FFF7EFFE00282DD14FF079
:108E9000B042136843F0080313601368A16A23F01B
:108EA000F0030B431360606AFFF7CEFEFFF7B4FFD9
:108EB000AB4B1860AB4B1868FAF7A4FF002834D00E
:108EC000BDE8F0814FF0B042136843F0080313602F
:108ED000136823F0F0030B431360606AFFF7B4FEDE
:108EE0000846FFF7C1FE0028E0D00120E8E74FF078
:108EF000B043002A54D01A6842F001021A60FAF70F
:108F000083FF0746FFF79AFE002842D04FF0B04299
:108F1000136843F0080313601368A16A23F0F00399
:108F20000B431360606AFFF78FFE2368D80748D4AD
:108F30002368990700F18C8023681E0740F1FA80AE
:108F4000A3694FF0B046002B00F0E180D6F89430D2
:108F5000E16903F01002914200F0C48003F00302C3
:108F6000022AC2D0D80740F1B380D6F8943023F05B
:108F70000103C6F89430FAF747FF0746D6F8943055
:108F8000990740F1A580FAF73FFFC31B112BF5D9D4
:108F900004E0FAF739FFC01B0228B3D903208FE79A
:108FA0001A6822F001021A60FAF72EFF0746FFF74F
:108FB00045FE0028B9D0FAF727FFC01B0228F6D9D2
:108FC000ECE7082D03D00C2D05D1032E03D16368E7
:108FD000002BADD189E74FF0B043A1681A6822F4A5
:108FE00080120A431A606268B2F5803F10D11A6895
:108FF00042F480321A60FAF707FF0746FFF718FEBF
:10900000002895D1FAF700FFC01B6428F6D9C5E700
:10901000B2F5041F04D11A6842F400121A60E6E7A0
:10902000196821F480311960196821F40011196060
:10903000002AE0D1FAF7E8FE0746FFF7F9FD00281D
:109040003FF476AFFAF7E0FEC01B6428F5D9A5E738
:10905000042D236903D00C2D0ED1022E0CD1002B30
:109060003FF443AF4FF0B0426169536823F0FE43D1
:1090700043EA016353605FE74FF0B046BBB133682A
:1090800043F480733360FAF7BFFE074633685A052E
:1090900005D4FAF7B9FEC31B022BF7D97EE7736834
:1090A000626923F0FE4343EA0263736044E7336876
:1090B00023F480733360FAF7A7FE074633685B0535
:1090C0007FF53AAFFAF7A0FEC31B022BF6D965E78E
:1090D0004FF0B042E169D2F8943023F010030B4313
:1090E000C2F894304FF0B047D7F8943043F0010302
:1090F000C7F89430FAF788FE0646D7F894309A07F6
:1091000018D4FAF781FE831B112BF6D946E7D6F85F
:10911000943023F00103C6F89430FAF775FE074641
:10912000D6F894309B0705D5FAF76EFEC31B112BBA
:10913000F6D933E72368580754D50B4F3B68D90558
:1091400014D4FFF701FDFAF75FFE06463B68DA0527
:109150000CD4FAF759FE831B022BF7D91EE700BF88
:10916000D8020020DC02002000040058E3684FF021
:10917000B046002B58D023F08003052B02BFD6F851
:10918000903043F00403C6F890304FF0B046FAF741
:109190003BFED6F8903043F001030746C6F8903006
:1091A00041F28838D6F890309B0705D4FAF72CFEA8
:1091B000C31B4345F6D9F1E6E36823F00403812B92
:1091C0001BD1FAF721FED6F8903043F08003C6F8A1
:1091D000903007464FF0B04641F28838D6F89030CC
:1091E000180504D5E36A002B4AD1002068E6FAF797
:1091F0000BFEC01B4045F1D9D0E6FAF705FED6F8C4
:10920000903023F08003C6F8903007464FF0B04608
:1092100041F28838D6F890301905E3D5FAF7F4FD15
:10922000C01B4045F6D9B9E6FAF7EEFDD6F8903006
:1092300023F080030746C6F8903041F28838D6F80C
:1092400090301A0516D4FAF7DFFDD6F8903023F0E7
:109250000103C6F8903007464FF0B04841F2883617
:10926000D8F890309B07BDD5FAF7CEFDC31BB342AB
:10927000F6D993E6FAF7C8FDC01B4045DFD98DE665
:109280000C2D4ED0022B4FF0B0431A6822F08072A2
:109290001A6033D1FAF7B8FD0546FFF7DEFC38BB9C
:1092A000D4E90C314FF0B0420B43D0682D49014056
:1092B0000B43E16B0B43216C0B43616C0B43A16BC4
:1092C00043EA0123D360136843F080731360D368CB
:1092D00043F08053D360FAF797FD0446FFF7BDFCD7
:1092E000002882D1FAF790FD001B0A28F6D955E62E
:1092F000FAF78AFD401B0A28CFD94FE6FAF784FD1A
:109300000446FFF7AAFC30B94FF0B042164BD168C3
:109310000B40D36069E7FAF777FD001B0A28F0D904
:109320003CE6012B3FF4E1AD4FF0B043D868236B2E
:1093300000F003029A427FF4D8AD626B00F0700334
:1093400093427FF4D2ADA26B00F4FE43B3EB022F45
:109350007FF4CBAD636C00F06040C01A18BF0120F1
:10936000AEE500BF8C80C111FCFFFEEE2DE9F0419F
:109370000D46044610B90120BDE8F081684E3368FF
:1093800003F007038B4216D323689A0727D54FF0C3
:10939000B047A268BB6823F0F0031343BB60FAF741
:1093A00033FD0646BB68DB0319D4FAF72DFD831B9A
:1093B000022BF7D911E0336823F007030B43336026
:1093C000FAF722FD0746336803F00703AB42DBD010
:1093D000FAF71AFDC01B0228F5D90320CCE7236851
:1093E000580617D54FF0B0476269D7F8083123F017
:1093F0000F0343EA1213C7F80831FAF705FD0646D2
:10940000D7F80831D90305D4FAF7FEFC831B022BE9
:10941000F6D9E2E723685A0713D54FF0B047E26860
:10942000BB6823F4E0631343BB60FAF7EDFC064628
:10943000BB689B0305D4FAF7E7FC831B022BF7D923
:10944000CBE72368180714D54FF0B0472269BB68F3
:1094500023F4605343EAC203BB60FAF7D5FC064627
:10946000BB68590305D4FAF7CFFC831B022BF7D94D
:10947000B3E72368DA070FD4294C236803F0070306
:10948000AB4239D8FFF7C8FC264B1860264BBDE825
:10949000F0411868FAF7B6BC6268022A1DD1FFF7DE
:1094A000C7FB00283FF467AF4FF0B04641F2883861
:1094B000B36823F003031343B360FAF7A5FC074630
:1094C000B368626803F00C03B3EB820FD4D0FAF7F1
:1094D0009BFCC01B4045F3D97FE7032A02D1FFF76D
:1094E000BCFBDEE712B9FFF7A9FBDAE74FF0B043A8
:1094F0001B685B05D8D43EE7236823F007032B43A2
:109500002360FAF781FC0646236803F00703AB42A9
:10951000B8D0FAF779FC801B0228F5D95DE700BFC7
:1095200000400058D8020020DC02002008B5FFF7F8
:1095300073FC4FF0B043044A9B68C3F3022352F814
:109540002330D84008BD00BF9076030808B5FFF768
:1095500063FC4FF0B043044A9B68C3F3C22352F844
:109560002330D84008BD00BF907603084FF0B043C9
:10957000D3F89000C0F3400070474FF0B0410209AB
:10958000D1F8883002F47F22000123EA020300F4BC
:109590007F200343C1F8883070474FF0B041020C80
:1095A000D1F88830120423EA020343EA0040C1F8EC
:1095B000880070470368DA0370B5044639D5FFF7B1
:1095C000C3FAFAF721FC614E05463368DB0532D554
:1095D0004FF0B043616BD3F8902002F44072914297
:1095E0001DD0D3F89010D3F8902042F48032C3F805
:1095F0009020D3F8902021F4407022F480328D071F
:10960000C3F89020C3F8900009D5FAF7FDFB41F2AA
:1096100088360546FFF7AAFF012840F090804FF0FA
:10962000B042616BD2F8903023F440730B43C2F820
:109630009030002605E0FAF7E7FB401B0228C4D96A
:1096400003262568E8070AD54FF0B0416268D1F8D3
:10965000883023EA124392B21343C1F88830A90735
:109660000AD54FF0B041A268D1F8883023EA1243FE
:1096700092B21343C1F88830AA0609D54FF0B04220
:109680002169D2F8883023F440630B43C2F8883054
:10969000AB0502D5206AFFF780FF680502D5606A36
:1096A000FFF77BFF290502D5A06AFFF776FF6A0660
:1096B00002D56069FFF761FF2B0602D5A069FFF7AD
:1096C0005CFFE80502D5E069FFF757FFE90610D512
:1096D0004FF0B042E168D2F8883023F440730B4376
:1096E000C2F88830B1F5807F02BFD36843F0807341
:1096F000D3602A040ED54FF0B042216BD2F88830E7
:1097000023F040430B43C2F8883019B9D36843F0C3
:109710008073D3606B0410D54FF0B042E16AD2F889
:10972000883023F040530B43B1F1005FC2F888301A
:1097300003D1D36843F48033D360304670BDFAF769
:1097400063FB401BB0427FF665AF79E70004005829
:1097500030B590F82C30012B02464FF0020022D099
:10976000174B82F82D00CA24012582F82C505C6228
:1097700053245C62B1F5807F146B996914D121F494
:1097800088519961596C24F0010421F00041596419
:109790001463DD650A4BFF2159620020012382F822
:1097A0002D3082F82C0030BD21F408519961D96C1C
:1097B00024F0020421F00041D9641463D865E9E77C
:1097C0000028004070B50B4E036B756D1D40EA0715
:1097D000044603D50123F365FAF78BFDAB0704D5E7
:1097E0000223F365204600F0C9F9012384F82D30E7
:1097F00070BD00BF0028004038B50A4CE36823F074
:109800002003E360FAF700FB0546E3689B0601D5F9
:10981000002038BDFAF7F8FA401BB0F57A7FF4D98A
:109820000320F6E700280040F8B5114DEC6814F06D
:10983000400406461AD1EB6843F08003EB60FAF768
:10984000E3FA23460746EC6814F0400401D1032BE9
:1098500001D11846F8BDFAF7D7FAC01BB0F57A7FE8
:10986000234684BF032386F82D30ECE70023F0E77E
:109870000028004038B50F4CE36823F08003E36014
:10988000A3699B06054606D4FFF7B6FF10B1032077
:1098900085F82D0038BDA36923F02003A361FFF7ED
:1098A000ABFF10B1032085F82D00A36943F020031E
:1098B000A361EFE70028004038B5044600284BD0EC
:1098C00090F82D3003F0FF021BB980F82C20F9F737
:1098D00067FC0223214D84F82D30EB68DB0636D47B
:1098E000CA236B6253236B622046FFF79DFF10B1C2
:1098F000FF236B6238BDAB6923F08E6323F0400316
:10990000AB6121696368AA690B431343A2691343DE
:10991000AB61D4E9022343EA02432B61D4E9093164
:10992000EA680B4322F4F8521343EB602046FFF73A
:10993000A1FF0028DCD1D4E90713AA690B4322F068
:109940006042134362691343AB61FF236B620123DF
:1099500084F82D300020CDE70120CBE7002800401F
:109960000023092803D840EA0310C0B270470A3820
:109970000133C0B2F5E700002DE9F04790F82C3034
:10998000012B05464FF0020069D0012385F82C30E9
:109990004E4B85F82D00DE6806F44076B6F5807FE4
:1099A00078D04C69087891F8019091F802A091F86C
:1099B0002470002A55D19B6913F0400308BFCB7077
:1099C000FFF7CEFF80464846FFF7CAFF02465046E3
:1099D000FFF7C6FF81463846FFF7C2FF0B6ACF7814
:1099E000234343EA875343EA090343EA084343EA2C
:1099F000022343EA0063354ACA2050625320506272
:109A00008C6A8869B4F5807F946945D124F48854C0
:109A100094610124D465B6F5807F09BFCB691364D6
:109A20000343536418BF5064284B4A681A672A6B73
:109A300042F001022A639A6942F488529A61244AE8
:109A4000D2F8803043F40033C2F880301F4BFF223D
:109A50005A620020012385F82D3085F82C00BDE8DE
:109A6000F087B4F1803F07D0B4F5000F04D09B69B4
:109A700013F0400308BFCB700B6ACA781C4344EA5A
:109A80000A0444EA004343EA092343EA825343EACF
:109A90000763B0E70023AEE724F40854946102247E
:109AA000D465B6F5807F09BFCB6993640343D36463
:109AB00018BFD064054B4A685A672A6B42F002020D
:109AC0002A639A6942F40852B8E700BF00280040B0
:109AD0000008005890F82C20012A03464FF002009D
:109AE00012D00A4A83F82D00CA21516253215162D3
:109AF000916941F020019161FF2151620020012212
:109B000083F82D2083F82C00704700BF0028004008
:109B100090F82C20012A03464FF0020019D00D4A7C
:109B200083F82D00CA2151625321516291690A487C
:109B300041F080019161D0F8801041F48021C0F89B
:109B40008010FF2151620020012283F82D2083F82C
:109B50002C0070470028004000080058064B5A6D42
:109B6000520610B5044603D54022DA65FAF7C4FB65
:109B7000012384F82D3010BD002800407047890073
:109B800001F1804101F531410A607047890001F11E
:109B9000804101F531410868704700002DE9F34725
:109BA0001F46894690460446FAF72EF90A9D3D4421
:109BB0002D1AFAF729F9264B1E68C6F3CB366E43E9
:109BC000824601962268936839EA03030CBF012399
:109BD0000023434501D100202EE07B1CF3D0FAF78F
:109BE00013F9A0EB0A00A84229D323685A6822F08F
:109BF000E0025A606268B2F5827F0AD1A268B2F5CB
:109C0000004F02D0B2F5806F03D11A6822F04002F3
:109C10001A60A26AB2F5005F07D11A6822F40052F6
:109C20001A601A6842F400521A60012384F85D3009
:109C3000002384F85C30032002B0BDE8F087019A6D
:109C4000019B002A03F1FF33019308BF1546B9E7D2
:109C5000D80200202DE9F74F994600238DF80330F4
:109C6000044688461746FAF7CFF80C9D4D442D1A46
:109C7000FAF7CAF82C4BD4F800B01E6823235E43D1
:109C8000360D6E43824601962268936803EA080304
:109C9000BB4201D100203AE0B8F5C06F07D137B917
:109CA0009BF80C30DBB28DF803309DF80330B9F12E
:109CB000FF3FEAD0FAF7A8F8A0EB0A00A84229D3A0
:109CC00023685A6822F0E0025A606268B2F5827F27
:109CD0000AD1A268B2F5004F02D0B2F5806F03D16D
:109CE0001A6822F040021A60A26AB2F5005F07D13A
:109CF0001A6822F400521A601A6842F400521A607C
:109D0000012384F85D30002384F85C30032003B025
:109D1000BDE8F08F019A019B002A03F1FF33019304
:109D200008BF1546B0E700BFD802002073B50B4648
:109D300000920D4616464FF4C05100220446FFF72C
:109D400089FF024630B1236E43F0200323660320CF
:109D500002B070BD00962B4680212046FFF71EFF03
:109D600002460028EFD100962B464FF4C0612046F2
:109D7000FFF770FF0028EBD0E5E74368B3F5827F7B
:109D8000F7B504460E4617460BD18368B3F5004F6E
:109D900002D0B3F5806F04D12268136823F040032A
:109DA000136000973346002280212046FFF7F6FE1D
:109DB000054628B1236E43F020032366032514E0F3
:109DC0006368B3F5827F10D1A368B3F5004F02D06A
:109DD000B3F5806F09D10097334600224FF4C0617C
:109DE0002046FFF737FF0028E4D1284603B0F0BD36
:109DF000F8B5044600287ED0436A002B50D1426853
:109E0000B2F5827F00D0C36194F85D3003F0FF02A9
:109E100023B984F85C202046F9F728FA2268E06824
:109E2000022384F85D301368B0F5E06F23F040033F
:109E300013604FF0000337D91D46B0F5706F18BF9F
:109E4000A362A7686368A169A66A07F4044703F4DC
:109E500082733B43276907F002073B43676907F0BA
:109E600001073B4301F400773B43E76907F03807FC
:109E70003B43276A07F080073B4306F400573B4308
:109E8000B6F5005F136014D1236B8BBBB0F5E06FA8
:109E90000DD902232363136843F40063136008E0C1
:109EA0000023C0E90433AFE74FF48055C7E701232F
:109EB0002363636A676B03F0100307F0080700F47D
:109EC00070603B43090C034301F004010B432B4337
:109ED000B6F5005F536004BFA38D1361D36923F40B
:109EE0000063D36100200123206684F85D30F8BD53
:109EF000022BDED1CFE70120F9E7000070B5044660
:109F000090F85C00012800F0CF80012084F85C000C
:109F100094F85D0066680128C5B20AD0B6F5827F64
:109F200040F0C080A068002840F0BC80042D40F0C4
:109F3000B980002951D0002A4FD0002B4DD094F881
:109F40005D00A16304281CBF052084F85D0000208B
:109F50002066C4E91300A06AE387B0F5005F2168BA
:109F6000A3872264A4F84430A4F8463007D10868D7
:109F700020F400500860086840F400500860486809
:109F800020F4C0404860E068B0F5E06FA06D29D9CA
:109F90004B6823F480534B6094F85D30434E444D3E
:109FA000042B444B18BF1D46434B18BF3346C0E932
:109FB0000B35424B436300238363B4F846300C31C6
:109FC0009BB2FEF785FA0346002848D0236E43F083
:109FD00010032366012384F85D300120002384F8F8
:109FE0005C3070BD4D6845F480554D60656DAD6960
:109FF000B5F5806F0AD113F0010F4B681ED123F421
:10A0000080434B60E38FC3F34E03E3878369B3F56B
:10A01000806FC1D14B6823F480534B60B4F8463055
:10A0200013F0010F4B6811D123F400534B60B4F8C7
:10A030004630C3F34E03A4F84630ADE743F4804303
:10A040004B60E38FC3F34E030133DEE743F4005369
:10A050004B60B4F84630C3F34E030133EBE722689C
:10A06000606D516841F001015160C0E90B33C0E9F6
:10A070000D33E38FA16B9BB20C32FEF729FA002857
:10A08000A4D123681A6852065EBF1A6842F04002E3
:10A090001A605A6842F020025A605A6842F002027E
:10A0A0005A609BE7022099E702209AE7F5A1000891
:10A0B000C5A00008D1A00008FFA00008DDA000088E
:10A0C0007047704708B5806AFFF7FBFF08BD70470F
:10A0D00008B5806AFFF7FBFF08BD7047806A026819
:10A0E00008B5536823F003035360036E43F0100375
:10A0F0000366012380F85D30FFF7EFFF08BD7FB5F1
:10A10000064600230393846A8DF80B30F9F77CFE32
:10A1100033681B689A06054668D42268536823F0A2
:10A1200020035360A36AB3F5005F13D101220090AE
:10A13000642311462046FFF731FD18B1236E43F02A
:10A1400002032366E3682668B3F5E06F2ED9F3684F
:10A150000393039BA2682368002A43D16268B2F587
:10A16000827F3FD15A6822F003025A6064212A4656
:10A170002046FFF702FE08B1202323660023A4F83F
:10A1800046302268012384F85D309368DB0606D5EB
:10A19000236E43F0020323664FF6EF739360236E42
:10A1A00023B32046FFF799FF04B070BD337BDBB2C9
:10A1B0008DF80B309DF80B30236B022BCAD1012296
:10A1C0000095642311462046FFF7E8FC18B1236E82
:10A1D00043F002032366337BDBB28DF80B309DF82E
:10A1E0000B30B7E75A6822F00102BEE72046FFF7BE
:10A1F00067FFD9E77FB5064600230393846A8DF88D
:10A200000B30F9F701FE33681B68990605465ED4EA
:10A210002268536823F020035360A36AB3F5005FFC
:10A220001BD1E368B3F5E06F3ED1236B012B3BD12B
:10A23000009064234FF400724FF4C0612046FFF792
:10A2400009FD18B1236E43F00203236623681B7BCC
:10A25000DBB28DF80B309DF80B302A466421204686
:10A26000FFF764FD18B1236E43F0200323662368D3
:10A270005A6822F003025A600022E287A4F84620BE
:10A28000012284F85D209A68D20606D5226E42F03B
:10A29000020222664FF6EF729A60236EBBB120462F
:10A2A000FFF71BFF04B070BD009564234FF480627C
:10A2B0004FF4C0612046FFF7CDFC18B1236E43F088
:10A2C000020323662368DB680393039BC5E72046EC
:10A2D000F8F7F2FAE6E70000036830B559689A68C3
:10A2E00002F04105012D85B0044606D14D0604D586
:10A2F000C36C05B0BDE830401847950704D5080683
:10A3000002D5236D2046F4E712F4B07F59D08D06B4
:10A3100057D550060FD594F85D0003284FF000057F
:10A3200049D0206E40F0040020660095D868009067
:10A3300098680090009895060CD5206E40F00100BA
:10A3400020660020029098680290186820F0400073
:10A3500018600298D00508D5226E42F008022266E5
:10A36000002203929A680392039A226E4AB35A68B3
:10A3700022F0E0025A60012284F85D208A0722D090
:10A380005A68A06D22F003025A6040B1104B8363FB
:10A39000FEF717F918B1236E43F040032366606D92
:10A3A00078B10B4B8363FEF70CF950B1236E43F089
:10A3B0004003236605E00195DA6801929B680193EA
:10A3C000019B05B030BD2046FFF787FEF9E700BFCF
:10A3D000D5A3000808B5806A0023A0F84630C387DB
:10A3E000FFF77BFE08BD0000034AD2F8903043F42B
:10A3F0000043C2F89030704700040058034AD2F876
:10A40000903023F40043C2F89030704700040058A5
:10A41000074B1A6822F040021A6040F441704FF472
:10A42000B85218605A601A6842F040021A607047C9
:10A430000000015837B5054600284ED0837903F057
:10A44000FF046BB1032C0BD0254B4FF400629A61D3
:10A450002868FFF7DDFF002401232B71AC602FE09B
:10A4600000236B712846F9F7E3FB1E4AD2F89030BF
:10A4700043F48053C2F89030002CE5D102234FF012
:10A48000B042AB71D2F8943023F40043C2F8943058
:10A49000154B1B681C214B43DB0C64214B43019380
:10A4A000019B93B90124AC60FFF79EFF0C4B9A68A7
:10A4B00042F400629A604FF400629A61002CC7D0A7
:10A4C0000123AB71204603B030BD019B013B0193DA
:10A4D000D2F894305B04E3D4E6E70124F2E700BF4E
:10A4E0000004005800080058D802002037B5174D66
:10A4F0002B6802461C204343DB0C64204343144872
:10A500000193019B93B901209060114C21732B683A
:10A510001C214B43DB0C64214B430193019B6BB922
:10A52000012090600A4BDB6803B030BD019B013B0A
:10A53000019383689C07E4D50020E6E7019B013B7B
:10A540000193A368DB07E9D5ECE700BFD802002040
:10A550000000015837B5184D2B6802461C204343B4
:10A56000DB0C6420434315480193019BA3B90120F0
:10A570009060124CFF2323732B681C256B43DB0C6C
:10A5800064256B430193019B73B9012090600B4BD1
:10A59000DB680B7003B030BD019B013B0193836806
:10A5A0009C07E2D50020E4E7019B013B0193A368EF
:10A5B000DB07E8D5EBE700BFD80200200000015818
:10A5C0000E4B0F491B681822534382B01B0D6422A7
:10A5D000534301934B69019AC3F3800322B90223C9
:10A5E0008360012002B07047019A013A01924A69E2
:10A5F000920701D5002BEDD10020F3E7D80200200F
:10A600000004005807B50379012B0FD10A4B1B68D2
:10A61000182253431B0C0193FFF7F0FE019B013BF3
:10A620000193019B002BF9D1FFF7DEFE03B05DF82B
:10A6300004EBFFF7C5BF00BFD8020020F8B51E46E7
:10A640008379012B154604460F46DAB22DD14379A2
:10A65000012B2AD0022342718371FFF7D3FF0D2112
:10A660002046FFF7CBFEFFF741FF390A2046FFF7F0
:10A670003DFFF9B22046FFF739FF2E44B5420ED117
:10A680002046FFF7B1FEFFF79BFFA06801230038CB
:10A69000A3714FF0000318BF01206371F8BD15F8D6
:10A6A000011B2046FFF722FFE8E70220F6E7F8B596
:10A6B0001E468379012B154604460F46DAB22FD188
:10A6C0004379012B2CD04271FFF79CFF1D212046BE
:10A6D000FFF794FEFFF70AFF390A2046FFF706FF4F
:10A6E000F9B22046FFF702FF00212046FFF7FEFEE9
:10A6F0002E44B5420ED12046FFF776FEFFF760FFED
:10A70000A06801230038A3714FF0000318BF012097
:10A710006371F8BD29462046FFF71CFF0135E8E7C5
:10A720000220F6E7F8B51F468379012B154604464B
:10A730000E46DAB22CD14379012B29D04271FFF7B2
:10A7400061FF06F0EF03A3F18402534253412371EA
:10A7500031462046FFF752FEFFF7C8FE2F44AF42B6
:10A7600010D1FFF741FE842E02D02046FFF728FFCC
:10A77000A06801230038A3714FF0000318BF012027
:10A780006371F8BD15F8011B2046FFF7AFFEE6E741
:10A790000220F6E7F8B51E468379012B15460446DC
:10A7A0000F46DAB227D14379012B24D04271FFF74B
:10A7B00029FF39462046FFF721FEFFF797FE0021CB
:10A7C0002046FFF793FE2E44B5420ED12046FFF7F8
:10A7D0000BFEFFF7F5FEA06801230038A3714FF0D0
:10A7E000000318BF01206371F8BD29462046FFF71A
:10A7F000B1FE0135E8E70220F6E737B50023ADF8F2
:10A80000043001AA022312210546FFF7C3FFBDF859
:10A810000440022364BA01AAA4B219462846FFF7ED
:10A8200081FFE20702D528460AF01EF8A30702D5E9
:10A8300028460AF01FF8600702D528460AF044F8B7
:10A84000210702D528460AF045F8E20602D5284637
:10A850000AF046F8A30602D528460AF02FF860064B
:10A8600002D528460AF00CF8210606D514F48071AA
:10A8700018BF012128460AF009F8A20502D528468A
:10A880000AF014F8630402D528460AF02FF803B042
:10A8900030BDF8B51E468379012B154604460F4698
:10A8A000DAB227D14379012B24D04271FFF7AAFEF7
:10A8B0000E212046FFF7A2FDFFF718FE394620467D
:10A8C000FFF714FE2E44B5420ED12046FFF78CFD53
:10A8D000FFF776FEA06801230038A3714FF0000354
:10A8E00018BF01206371F8BD15F8011B2046FFF762
:10A8F000FDFDE8E70220F6E7F8B51E468379012B57
:10A90000154604460F46DAB22BD14379012B28D0E5
:10A910004271FFF777FE1E212046FFF76FFDFFF71C
:10A92000E5FD39462046FFF7E1FD00212046FFF70F
:10A93000DDFD2E44B5420ED12046FFF755FDFFF751
:10A940003FFEA06801230038A3714FF0000318BF39
:10A9500001206371F8BD29462046FFF7FBFD013554
:10A96000E8E70220F6E70000036A23F00103036230
:10A97000036A70B5446882690D6822F4803222F05F
:10A9800073022A438D6823F002032B43124DA84221
:10A9900006D0124EB04203D0A6F58066B04214D164
:10A9A000CE6823F008033343A84223F0040306D003
:10A9B0000B4DA84203D005F58065A84205D124F4CB
:10A9C0004075D1E9054634432C43446082614A68AE
:10A9D0004263036270BD00BF002C0140004801408B
:10A9E00000440140036A23F480730362036A4268EF
:10A9F00070B5C4690D6824F4803424F073042C43CA
:10AA00008D6823F4007343EA05230F4DA8420ED14D
:10AA1000CD6823F4006343EA052323F48063D1E97E
:10AA2000055622F44052354342EA051206E0074D2E
:10AA3000A842F4D005F58065A842F0D042604A688B
:10AA4000C461C263036270BD002C01400044014038
:10AA5000036A23F480530362026A30B54468C36911
:10AA60000D6823F0807323F4E64343EA05238D68E1
:10AA700022F4005242EA05320A4DA84207D005F5F9
:10AA8000C055A84203D005F58065A84204D14D69A0
:10AA900024F4804444EA85144460C3614B68036431
:10AAA000026230BD002C0140036A23F4803303624C
:10AAB000026A30B54468436D0D6823F4803323F097
:10AAC00070032B438D6822F4003242EA05420B4D9D
:10AAD000A84207D005F5C055A84203D005F580650A
:10AAE000A84204D14D6924F4803444EA052444602A
:10AAF00043654B688365026230BD00BF002C014096
:10AB0000036A23F480130362026A30B54468436D1C
:10AB10000D6823F0807323F4E04343EA05238D6836
:10AB200022F4001242EA05520A4DA84207D005F568
:10AB3000C055A84203D005F58065A84204D14D69EF
:10AB400024F4802444EA8524446043654B68C3654B
:10AB5000026230BD002C0140704710B5846A626A01
:10AB600082420BD101232377D2690AB984F83E309F
:10AB70002046F9F723F80023237710BDA36A834208
:10AB800008D102222277DB69002BF1D1012384F85E
:10AB90003F30EDE7E36A834208D104222277DB6984
:10ABA000002BE5D1012384F84030E1E7236B834299
:10ABB000DED108222277DB69002BD9D1012384F86A
:10ABC0004130D5E7704710B5846A636A834207D184
:10ABD000012323772046FFF7F5FF0023237710BDDD
:10ABE000A36A834201D10223F3E7E36A834201D1DE
:10ABF0000423EEE7236B8342ECD10823E9E7704797
:10AC000010B5846A636A834209D10123237784F8EB
:10AC10003E302046FFF7F3FF0023237710BDA36AE1
:10AC2000834205D102232377012384F83F30F0E7E4
:10AC3000E36A83424FF0010304D10422227784F8AF
:10AC40004030E6E7226B824203BF0822227784F875
:10AC5000413084F83D30DCE71A4A0368904210B571
:10AC600002D0B0F1804F09D14C6823F070039042BC
:10AC700043EA040309D0B0F1804F06D0124A904253
:10AC800003D002F58062904203D1CA6823F4407376
:10AC900013434A6923F08003134303608B68C36244
:10ACA0000B688362074B984207D003F5C053984264
:10ACB00003D003F58063984201D10B69036301233C
:10ACC000436110BD002C01400044014010B5044612
:10ACD00050B390F83D3003F0FF021BB980F83C20E0
:10ACE000F9F76AF90223206884F83D30211DFFF747
:10ACF000B3FF012384F84830002084F83E3084F804
:10AD00003F3084F8403084F8413084F8423084F891
:10AD1000433084F8443084F8453084F8463084F871
:10AD2000473084F83D3010BD0120FCE710B50446E3
:10AD300050B390F83D3003F0FF021BB980F83C207F
:10AD4000FFF70AFF0223206884F83D30211DFFF73A
:10AD500083FF012384F84830002084F83E3084F8D3
:10AD60003F3084F8403084F8413084F8423084F831
:10AD7000433084F8443084F8453084F8463084F811
:10AD8000473084F83D3010BD0120FCE7036A23F012
:10AD900010030362036A426870B584690D6824F089
:10ADA000807424F4E64444EA05248D6823F02003EB
:10ADB00043EA05130F4DA8420ED1CD6823F080035E
:10ADC00043EA051323F04003D1E9055622F440621B
:10ADD000354342EA850206E0074DA842F4D005F566
:10ADE0008065A842F0D042604A6884618263036251
:10ADF00070BD00BF002C01400044014038B590F800
:10AE00003C30012B044673D001200C2A84F83C000E
:10AE10004ED008D8042A2BD0082A39D0BAB1002342
:10AE200084F83C3038BD102A52D0142AF7D120685B
:10AE3000FFF766FE436D0A6943F400634365436DA3
:10AE400023F480634365436D43EA02234EE02068A8
:10AE5000FFF78AFD83690A6943F008038361836908
:10AE600023F0040383618369134383610020D6E7E1
:10AE70002068FFF78BFF83690A6943F400638361ED
:10AE8000836923F480638361836943EA0223ECE7E7
:10AE90002068FFF7A7FDC3690A6943F00803C3618F
:10AEA000C36923F00403C361C3691343C361DDE7CE
:10AEB0002068FFF7CDFDC3690A6943F40063C361ED
:10AEC000C36923F48063C361C36943EA0223EDE7E6
:10AED0002068FFF7E9FD436D0A6943F00803436505
:10AEE000436D23F004034365436D13434365BDE79E
:10AEF000022097E710B584680A4324F47F4442EAAD
:10AF000003222243826010BD38B590F83C30012BFB
:10AF100004464FF0020000F0958084F83D000122C5
:10AF2000206884F83C208568474B2B4083600B6881
:10AF3000602B54D037D8402B6BD019D8202B0DD094
:10AF40000AD833F0100109D0012384F83D300023E2
:10AF500084F83C30104638BD302BF5D1826822F49D
:10AF6000401222F070021A4342F0070282602BE086
:10AF7000502BE9D14A68CD68016A036A23F00103C6
:10AF80000362836921F00A0123F0F00343EA051309
:10AF90000A4383610262836823F4401323F0700341
:10AFA00043F057030FE0B3F5805F0DD0B3F5005FBA
:10AFB0000CD0702BC8D1CB68D1E90121FFF79AFFE3
:10AFC000836843F0770383600022BDE7CB68D1E953
:10AFD0000121FFF78FFF836843F48043F3E7036A9F
:10AFE0004D68C96823F0100303628269036A22F482
:10AFF000704223F0A00343EA051342EA0132826162
:10B000000362836823F4401323F0700343F0670363
:10B01000D9E74A68CD68016A036A23F00103036235
:10B02000836921F00A0123F0F00343EA05130A4380
:10B0300083610262836823F4401323F0700343F0BA
:10B040004703C0E7024685E78800CEFF036A01F0A8
:10B050001F0110B501248C4023EA04030362036A34
:10B060008A401A43026210BD38B50D46082D0446C9
:10B0700011461BD005D85DB1042D14D094F84300BF
:10B0800008E00C2D15D0102DF8D190F8420001E009
:10B0900090F83E00A0F1020CDCF1000040EB0C0047
:10B0A00050B1022076E090F83F00F3E790F84000BE
:10B0B000F0E790F84100EDE7082D1AD007D86DB100
:10B0C000042D13D094F84320012A19D00CE00C2D44
:10B0D00027D0102DF6D194F842000CE094F83E20D1
:10B0E000501E424242415AB9012053E094F83F2099
:10B0F000F6E794F84000421E504250410028F3D039
:10B100000029F1D0002BEFD0082D4FF0020256D0CD
:10B110000AD885B1042D3ED0042D84F84320E3D114
:10B120003BE094F84100E6E70C2D5CD0102DF3D104
:10B1300084F84220D8E7606A84F83E203A4AC26226
:10B140003A4A02633A4A426322683432FDF7C0F950
:10B150000028C9D12268D36843F400732068D36003
:10B1600029460122FFF772FF324A904250D0324BFB
:10B1700098424DD003F58063984249D0B0F1804F9A
:10B180004DD182682D4B1340062B02D0B3F5803F82
:10B1900045D1002038BD84F83F20A06A224AC2620F
:10B1A000224A0263224A426322683832FDF790F94C
:10B1B000002899D12268D36843F48063CEE7E06A1F
:10B1C00084F84020184AC262184A0263184A42634F
:10B1D00022683C32FDF77CF9002885D12268D368CB
:10B1E00043F40063BAE7206B84F841200E4AC26240
:10B1F0000E4A02630E4A426322684032FDF768F944
:10B2000000287FF471AF2268D36843F48053A5E728
:10B21000436C904243F400434364B2D0AEE703680A
:10B2200043F001030360B4E75BAB0008C7AB000861
:10B2300001AC0008002C014000440140070001005F
:10B24000FFF712BF082938B504460D464FD004D881
:10B2500061B1042944D0012038BD0C29FBD102681A
:10B26000006BD36823F48053D36005E00268406A22
:10B27000D36823F40073D360FDF7A3F9206800229C
:10B280002946FFF7E3FE2A4B984207D003F5C05347
:10B29000984203D003F5806398420DD1026A41F2CF
:10B2A00011131A4208D1026A40F244431A4202BF03
:10B2B000436C23F400434364026A41F211131A42BF
:10B2C00008D1026A40F244431A4202BF036823F0E5
:10B2D0000103036001238DB984F83E300020BBE7F1
:10B2E0000268806AD36823F48063D360C4E702688D
:10B2F000C06AD36823F40063D360BDE70C2D13D07C
:10B3000007D8042D0AD0082D0BD0012384F8433030
:10B31000E4E7102DF9D184F84230DFE784F83F30BC
:10B32000DCE784F84030D9E784F84130D6E700BF45
:10B33000002C0140FFF786BF70B590F83C30012B20
:10B3400002464FF0020020D082F83D000F4D1068F9
:10B3500043688468A84202BF4E6823F470033343F5
:10B360000E6823F070033343A842436002D0B0F16B
:10B37000804F04D1896824F080030B43836001234C
:10B38000002082F83D3082F83C0070BD002C014066
:10B39000026852E8003F23F0C00342E8003102682F
:10B3A0000029F5D102F1080353E8003F23F400031C
:10B3B00002F1080C4CE800310029F3D12023C0F839
:10B3C0008830704710B5026852E8003F23F490734C
:10B3D00042E8003102680029F5D10F4C02F1080360
:10B3E00053E8003F234002F1080C4CE800310029EB
:10B3F000F4D1C36E012B07D152E8003F23F01003B4
:10B4000042E800310029F7D12023C0F88C30002316
:10B41000C366436710BD00BFFEFFFFEFF8B50446EB
:10B420001346D4F88850202D32D1F1B1EAB1E06F43
:10B43000A4F85620A4F8542000262122C4F89060D5
:10B440002165C4F88820226888B1124FC762124F64
:10B450000763124F2832C0E90D76FDF739F830B195
:10B460001023C4F89030C4F888500120F8BD236838
:10B4700040221A62226802F1080353E8003F43F0B9
:10B48000800302F1080141E800300028F3D1EDE724
:10B490000220EBE7A1B40008E9B40008F5B4000805
:10B4A00008B50346806A1B681B6813F0200317D198
:10B4B000A0F85630026802F1080353E8003F23F079
:10B4C0008003083242E8003102680029F2D152E8D4
:10B4D000003F43F0400342E800310029F7D108BDA6
:10B4E000F9F73EF8FBE7704708B5806AFFF7FBFF06
:10B4F00008BD7047806A38B50468D0F88830D0F845
:10B500008C50A268120606D5212B04D10023A0F886
:10B510005630FFF73DFFA3685B0606D5222D04D108
:10B520000023A0F85E30FFF74DFFD0F8903043F0D5
:10B530001003C0F89030FFF7DCFF38BD08B5806A13
:10B540000023A0F85E30A0F85630FFF7D2FF08BD08
:10B55000704700000368D9691A682DE9F04140F688
:10B560000F0631429D68044610D18E0640F1978047
:10B5700002F0200605F080573E4300F09080436FB4
:10B58000002B00F08580BDE8F0411847AB4EAC4879
:10B590002E401040304300F08280CF0709D5D005FF
:10B5A00007D501201862D4F8900040F00100C4F8DB
:10B5B00090008F0709D5E80707D502201862D4F854
:10B5C000900040F00400C4F890004F0709D5E80748
:10B5D00007D504201862D4F8900040F00200C4F8A7
:10B5E00090000F070BD502F02000304307D0082051
:10B5F0001862D4F8900040F00800C4F890000E05DE
:10B600000AD5500108D54FF400601862D4F8903084
:10B6100043F02003C4F89030D4F89030002B37D09A
:10B620008B0609D502F0200205F080552A4303D08D
:10B63000636F0BB1204698472668D4F89020B36812
:10B6400002F0280203F0400353EA0205204621D00D
:10B65000FFF7B8FEB3685F0617D5226802F108034A
:10B6600053E8003F23F04003083242E8003100294C
:10B67000F3D1D4F8800040B1724B8363FCF7A1FF93
:10B6800030B1D4F88000836B7DE72046FFF731FFAF
:10B69000BDE8F081FFF72DFFC4F89050F8E7E06EA9
:10B6A000012840F08980CE0640F18680D00640F126
:10B6B000838010221A629A6851064BD5D4F88020F4
:10B6C00011684A6892B2002AE2D0B4F85C00904255
:10B6D000DED9A4F85E200A6892062FD453E8002F22
:10B6E00022F4807243E800210029F7D103F1080217
:10B6F00052E8002F22F0010203F1080040E8002187
:10B700000029F3D103F1080252E8002F22F0400291
:10B7100003F1080040E800210029F3D12022C4F8F9
:10B720008C20E16653E8002F22F0100243E800214C
:10B730000029F7D1D4F88000FCF70EFF022323671D
:10B74000B4F85E30B4F85C10C91A89B22046FFF72D
:10B75000FFFE9DE7B4F85E20B4F85E00B4F85C101C
:10B7600080B292B2002893D0891A89B200298FD072
:10B7700053E8002F22F4907243E800200028F7D10C
:10B78000314D03F1080252E8002F2A4003F1080668
:10B7900046E800200028F4D12022C4F88C206067FD
:10B7A000E06653E8002F22F0100243E80020002852
:10B7B000F7D102232367C9E7CF0209D56E0207D567
:10B7C0004FF4801220461A62BDE8F04100F0A0BD9F
:10B7D00008060BD502F0800005F40005284305D0CB
:10B7E000A36F002B3FF454AF2046CCE64F0611D593
:10B7F00056060FD553E8002F22F0400243E80021FF
:10B800000029F7D12023C4F88830A1672046F8F733
:10B81000A7FE3DE70D0206D5500004D52046BDE841
:10B82000F04100F077BDCB017FF532AF002ABFF6C3
:10B830002FAF2046BDE8F04100F06BBD01000010C5
:10B84000200100043DB50008FEFFFFEFD0F88C207A
:10B85000B0F86010222A08B5036855D15B6A826D82
:10B860000B401370836D01338365B0F85E30013B8C
:10B870009BB2A0F85E30B0F85E309BB2002B42D194
:10B88000026852E8003F23F4907342E800310368F5
:10B890000029F5D103F1080252E8002F22F001023D
:10B8A00003F1080C4CE800210029F3D12022C0F854
:10B8B0008C20184A41679342016705D1C26E012A64
:10B8C0000ED0F8F75BFE1EE05A681102F6D553E879
:10B8D000002F22F0806243E800210029F7D1EDE734
:10B8E0000022C26653E8002F22F0100243E8002134
:10B8F0000029F7D1DA69B0F85C10D20644BF1022F3
:10B900001A62FFF725FE08BD9A6942F008029A61A3
:10B91000F9E700BF00800040D0F88C20B0F860103C
:10B92000222A08B5036852D15A6A1140826D22F862
:10B93000021B8265B0F85E20013A92B2A0F85E2048
:10B94000B0F85E2092B2002A40D153E8002F22F4D2
:10B95000907243E800210029F7D103F1080252E870
:10B96000002F22F0010203F1080C4CE8002100290D
:10B97000F3D12022C0F88C20174A41679342016717
:10B9800005D1C26E012A0ED0F8F7F8FD1EE05A6804
:10B990001102F6D553E8002F22F0806243E800211F
:10B9A0000029F7D1EDE70022C26653E8002F22F00C
:10B9B000100243E800210029F7D1DA69B0F85C10E1
:10B9C000D20644BF10221A62FFF7C2FD08BD9A6971
:10B9D00042F008029A61F9E7008000402DE9F84F33
:10B9E0000368B0F86060D3F81CB01F689D68D0F899
:10B9F0008C20222A044640F0B980B0F8683043B168
:10BA0000DFF87491DFF874A14FF000081BF0200FED
:10BA100020D1B4F85E309BB2D3B1B4F868209A421A
:10BA200016D9226802F1080353E8003F23F080533F
:10BA3000083242E8003122680029F2D1504B636796
:10BA400052E8003F43F0200342E800310029F7D1DB
:10BA5000BDE8F88F2368A26D5B6A33401370A36D55
:10BA60000133A365B4F85E30013B9BB2A4F85E30AD
:10BA70002368D3F81CB01BF0070F2ED01BF0010F6A
:10BA800009D0F90507D501221A62D4F8902042F0B6
:10BA90000102C4F890201BF0020F09D0EA0707D575
:10BAA00002221A62D4F8902042F00402C4F89020D6
:10BAB0001BF0040F09D0E80707D504221A62D4F856
:10BAC000903043F00203C4F89030D4F8903023B1A2
:10BAD0002046FFF70EFDC4F89080B4F85E309BB2AC
:10BAE000002B93D1226852E8003F23F4807342E890
:10BAF000003123680029F5D103F1080252E8002F34
:10BB000002EA090203F1080040E800210029F3D10C
:10BB100020225345C4F88C20616721670AD05A68F7
:10BB2000110207D553E8002F22F0806243E800217C
:10BB30000029F7D1E26E012A14D10022E26653E80F
:10BB4000002F22F0100243E800210029F7D1DA6922
:10BB5000B4F85C10D20644BF10221A622046FFF7E8
:10BB6000F7FC53E72046F8F709FD4FE79A6942F0E2
:10BB700008029A616CE700BFFEFFFFEF0080004003
:10BB80004DB800082DE9F84F0368B0F86060D3F8AD
:10BB90001CB01F689D68D0F88C20222A044640F013
:10BBA000B780B0F8683043B1DFF87091DFF870A16A
:10BBB0004FF000081BF0200F20D1B4F85E309BB28C
:10BBC000D3B1B4F868209A4216D9226802F108036A
:10BBD00053E8003F23F08053083242E800312268E6
:10BBE0000029F2D14F4B636752E8003F43F0200336
:10BBF00042E800310029F7D1BDE8F88F2368A26D33
:10BC0000596A314022F8021BA265B4F85E20013A5D
:10BC100092B2A4F85E20D3F81CB01BF0070F2ED010
:10BC20001BF0010F09D0F90507D501221A62D4F8DB
:10BC3000902042F00102C4F890201BF0020F09D0BE
:10BC4000EA0707D502221A62D4F8902042F00402D3
:10BC5000C4F890201BF0040F09D0E80707D5042290
:10BC60001A62D4F8903043F00203C4F89030D4F84C
:10BC7000903023B12046FFF73CFCC4F89080B4F824
:10BC80005E309BB2002B95D1226852E8003F23F42E
:10BC9000807342E8003123680029F5D103F10802DE
:10BCA00052E8002F02EA090203F1080040E80021EF
:10BCB0000029F3D120225345C4F88C206167216705
:10BCC0000AD05A68110207D553E8002F22F080628B
:10BCD00043E800210029F7D1E26E012A14D10022A5
:10BCE000E26653E8002F22F0100243E80021002909
:10BCF000F7D1DA69B4F85C10D20644BF10221A6298
:10BD00002046FFF725FC55E72046F8F737FC51E7BA
:10BD10009A6942F008029A616EE700BFFEFFFFEFEA
:10BD20000080004019B9000838B50446036821694D
:10BD3000A2681D68C0690A4361690A4377490243E2
:10BD400029400A431A605A68E16822F440520A43C3
:10BD50005A60734AA16993421CBF226A11439A68D0
:10BD600022F06E4222F430620A439A60DA6A616A13
:10BD700022F00F020A43DA626A4A934219D14FF065
:10BD8000B043694AD3F8883003F0030343F44033E7
:10BD9000934200F0B480B3F1031F24D0013A9342E0
:10BDA00040F0B580B0F5004F40F08F80FCF7C6FF43
:10BDB0006EE05E4A93421CD14FF0B0435C49D3F829
:10BDC000883003F00C0343F440228A4200F097804D
:10BDD00006D8002B7CD0574B9A42E3D0012026E0B6
:10BDE000B2F10C1FFAD1B0F5004F53D04FF4004020
:10BDF00075E04B4A9342F1D14FF0B043D3F888300D
:10BE000003F44063B3F5006F18D006D85BB1B3F507
:10BE1000806FE3D1FCF792FF07E0B3F5406FDDD10F
:10BE20004FF400400BE0FDF781FB40B900204FF0DC
:10BE30000113A3660023C4E91D3338BD3E4865687D
:10BE40003E4B626A05EB450133F81220B0FBF2F37A
:10BE50009942C3D8B3EB053FC0D800231946F6F783
:10BE600023FB090241EA10616B080002C0182A4650
:10BE70004FF0000341F10001F6F716FB304BA0F53F
:10BE800040729A42AAD82368D860CFE7FDF74EFBEC
:10BE90000028CBD06168294B626A33F81220B0FBCE
:10BEA000F2F24B0803EB42034FF6EF72B3FBF1F3F0
:10BEB000A3F11001914291D823F00F02216892B2B0
:10BEC000C3F342031343CB60B0E7FCF737FF04E052
:10BED000B0F5004FDAD0FDF729FB0028A6D0636843
:10BEE000616A164A32F81120B0FBF2F000EB530001
:10BEF000B0FBF3F04FF6EF73A0F11002C1E7B0F51D
:10BF0000004F0D48EBD1C5E7FDF720FBC0E7B0F5CA
:10BF1000004FF9D0FDF71AFBDFE700BFF369FFCF51
:10BF2000008000400038014002000300004400404F
:10BF300008000C0004000C000024F400F076030854
:10BF4000FFFC0F00836ADA0710B506D50168C46AE2
:10BF50004A6822F4003222434A609C0706D50168F1
:10BF6000046B4A6822F4803222434A60590706D59E
:10BF70000168446B4A6822F4802222434A601A070F
:10BF800006D50168846B4A6822F4004222434A6065
:10BF9000DC0606D50168C46B8A6822F4805222430D
:10BFA0008A60990606D50168046C8A6822F40052FA
:10BFB00022438A605A060FD50168446C4A6822F40D
:10BFC00080122243B4F5801F4A6005D14A68846C10
:10BFD00022F4C00222434A601B0606D50268C16CE7
:10BFE000536823F400230B43536010BD2DE9F8433D
:10BFF000DDF8209005460F46164698462A68D36914
:10C0000037EA03030CBF01230023B34201D0002011
:10C0100029E0B9F1FF3FF2D0F7F7F6FEA0EB0800F8
:10C0200048452C6802D8B9F1000F1ED154E8003FF2
:10C0300023F4D07344E80032002AF7D104F1080356
:10C0400053E8003F23F0010304F1080141E8003206
:10C05000002AF3D12023C5F88830C5F88C3000239E
:10C0600085F884300320BDE8F88323685A07C5D5D6
:10C07000E3691B05C2D54FF40063236254E8003F17
:10C0800023F4D07344E80032002AF7D104F1080306
:10C0900053E8003F23F0010304F1080141E80032B6
:10C0A000002AF3D12023C5F88830C5F88C30C5F8B4
:10C0B0009030D4E773B504460026C0F89060F7F7D7
:10C0C000A3FE23681B681A07054619D423681B685A
:10C0D0005B070AD56FF07E43009300222B464FF496
:10C0E00080012046FFF782FFB0B900202023C4F86A
:10C0F000883084F88400C4F88C30E06620670CE057
:10C100006FF07E430093324603464FF40011204601
:10C11000FFF76CFF0028D9D0032002B070BD10B526
:10C12000044650B3D0F888301BB980F88430F8F753
:10C1300025F922682423C4F88830136823F001030A
:10C1400013602046FFF7F0FD012816D0A36A13B153
:10C150002046FFF7F7FE23685A6822F490425A609F
:10C160009A6822F02A029A601A6842F00102204678
:10C170001A60BDE81040FFF79DBF012010BD000010
:10C1800030B581658168A0F85C200023B1F5805F3F
:10C19000A0F85E20436735D10369002B40F2FF13FE
:10C1A00018BFFF23A0F860300023C0F8903022238E
:10C1B000C0F88C30016801F1080353E8003F43F0F8
:10C1C0000103083141E800340368002CF2D1456EC8
:10C1D00084680169B5F1005F32D1B0F868509542CA
:10C1E0002ED8B4F5805F244A03D1244C002908BF1F
:10C1F00022464267B1B153E8002F42F4807243E80F
:10C200000021F7E729B90369002B14BF7F23FF231F
:10C21000C8E7B1F1805FC5D10369002B14BF3F238C
:10C220007F23BFE703F1080252E8002F42F080525B
:10C2300003F1080040E800210029F3D1002030BDBF
:10C24000B4F5805F0E4A03D10E4C002908BF224688
:10C25000426741B153E8002F42F4907243E8002155
:10C260000029F7D1EAE753E8002F42F0200243E823
:10C2700000210029F7D1E1E7DDB9000885BB0008FE
:10C280004DB8000819B90008D0F88C30202B30B414
:10C2900015D1B9B1B2B100230468C3660A4B9C4200
:10C2A0000AD063681B0207D554E8003F43F080635F
:10C2B00044E80035002DF7D130BCFFF761BF022004
:10C2C00030BC70470120FBE700800040436E30B572
:10C2D0002BB90123A0F86A30A0F8683030BD03689C
:10C2E000094D9A689968094C490FC2F342626B5C28
:10C2F000615CDB00B3FBF1F3A0F86A30AB5CA25CDD
:10C30000DB00B3FBF2F3E7E71077030808770308D5
:10C310007047704770471FB504AB03E9060090F8FB
:10C320008430012B04463AD0012380F88430242342
:10C33000C0F8883003681A6822F001021A609A680F
:10C3400022F440120A439A6071B95A68BDF80C0091
:10C350009DF80E1022F0100202435A605A6822F033
:10C360007F4242EA01625A601A6842F001021A6092
:10C37000F7F74AFD6FF07E42034600924FF48001CA
:10C3800000222046FFF732FE38B92023C4F8883057
:10C39000002384F8843004B010BD0320F8E70220A5
:10C3A000F9E790F88430012B0FD0012380F8843016
:10C3B000016851E8002F42F0020241E80023002BFF
:10C3C000F6D180F88430184670470220704710B5C7
:10C3D00090F88430012B044617D02423C0F888300D
:10C3E00003681A68196821F00101196042F00052CF
:10C3F0004FF0005141661A60FFF768FF2023C0F834
:10C400008830002084F8840010BD0220FCE770B55D
:10C4100090F88430012B044617D005682423C0F817
:10C4200088302E682B6823F001032B60AB6823F063
:10C4300060431943A960FFF749FF20232E60C0F82D
:10C440008830002084F8840070BD0220FCE770B5BD
:10C4500090F88430012B044617D005682423C0F8D7
:10C4600088302E682B6823F001032B60AB6823F023
:10C4700060631943A960FFF729FF20232E60C0F8ED
:10C480008830002084F8840070BD0220FCE70000A2
:10C4900038B5084D052455F8043B2BB9013C14F080
:10C4A000FF04F8D1204638BDDB6898470028F5D056
:10C4B000F9E700BF081C0020034BD870034B1B6832
:10C4C0001B6C03B118477047F01B0020EC1B0020C9
:10C4D000034B1874034B1B685B6C03B11847704720
:10C4E000F01B0020EC1B0020F0B5314D314B95F9CD
:10C4F0000420314E91B00C46012795F905108DF8B6
:10C50000047002288DF809208DF80A1010D18DF8DA
:10C510000800D8711C7202F063FD337803B114B1C6
:10C5200001A803F0C1F9254B059A1A6011B0F0BDBE
:10C5300059714FF480711A71D9801C7233788DF85B
:10C54000087053BB1F2306A88DF81C208DF81830E7
:10C5500002F024FF20238DF8183006A82B798DF8DF
:10C560001C3002F01BFF22238DF8183006A86B79CF
:10C570008DF81C3002F012FF21238DF8183006A828
:10C580006B798DF81C3002F009FF29238DF81830E3
:10C5900006A80B4B079302F001FF02F021FD0123D7
:10C5A00006A88DF818308DF81C3002F0F7FEB4E7BD
:10C5B000F01B002010030020CC1A0020C01B00201C
:10C5C000000400017FB5092301A88DF8043003F0B1
:10C5D0006BF90038044B059A1A6018BF01204042DD
:10C5E00007B05DF804FB00BFC01B002070B5044617
:10C5F0000B46144962784A700020A2780A720870CB
:10C600001A884A729A788A72DB780B746368CB60F6
:10C610000D4B1B68DA6A2AB1237803F0FB030A2B5F
:10C6200000D09047094E002556F8043B1BB15B6AC9
:10C630000BB1204698470135EBB2052B6DB2F3D113
:10C6400070BD00BFE0020020EC1B0020081C002091
:10C6500070B5044611480123037063784370A378D2
:10C660008372E368C360E3780376236943762379B2
:10C6700043720B4B1B689B6A03B19847094E002518
:10C6800056F8043B1BB19B690BB120469847013516
:10C69000EBB2052B6DB2F3D170BD00BFF4020020E8
:10C6A000EC1B0020081C0020014B1868704700BFDD
:10C6B000C01B002000B58BB0012368468DF8003008
:10C6C00002F046FD38B99DF80400003818BF01207B
:10C6D0000BB05DF804FB0020FAE7000008B501F09C
:10C6E00037FE40B9FFF7E6FF012806D0054B197A5F
:10C6F000D879FFF7F9FE012008BDBDE80840FFF733
:10C70000C7BE00BF100300202DE9F04186B00546EA
:10C710000E46174601F01CFE002873D101F030FED2
:10C72000044640B9FFF7C6FF01280AD03D4B197AED
:10C73000D879FFF7D9FE6FF00204204606B0BDE8B5
:10C74000F081DFF8E48088F80860003E18BF012619
:10C750008DF80460354E687833798DF8123069466B
:10C7600002F094FC00283FD08DF804400394ADF80B
:10C7700010406FF0060495E803002D4B83E803009A
:10C78000337988F80A30394601A803F091F9294B2A
:10C79000059A1A6011283FD801A353F820F000BF72
:10C7A0000BC8000805C8000819C8000819C8000807
:10C7B00019C8000819C8000819C8000837C70008B8
:10C7C00019C8000819C8000819C80008FFC70008E0
:10C7D00019C8000819C8000805C8000805C80008DD
:10C7E00005C800081FC800082B788DF808306B7842
:10C7F000ADF810306B6803934FF0FF34BBE76FF078
:10C8000005049AE76FF0010497E70B4B00221A70BA
:10C81000E31D18BF144690E74FF0FF348DE76FF02B
:10C8200004048AE710030020F4020020F01B00201B
:10C8300004030020C01B0020BF1B002037B501F0FF
:10C84000A9FD134D052455F8043B4BB11A693AB1C3
:10C850009B682BB1984718B155F8043C1B69984761
:10C86000013C14F0FF04EED1FFF712FE68B9094D48
:10C870002B7853B1084BADF80040D978019422468B
:10C880006846FFF741FF00B92C7003B030BD00BF10
:10C89000081C0020BF1B0020F01B002030B58BB00F
:10C8A000044601F055FD0546002835D1FFF702FF8B
:10C8B000012834D168468DF8005002F049FC40BB95
:10C8C0009DF80430A34204D0012C22D0022C12D0B7
:10C8D00014B100200BB030BD002BFAD068468DF8A3
:10C8E000044002F05BFDA0B90E4B1B681B6B002BD4
:10C8F000EFD09847EDE763B968468DF8044002F041
:10C900004DFD30B9074B1B681B6B002BE1D0204657
:10C91000EFE74FF0FF30DDE76FF00100DAE76FF08F
:10C920000200D7E7EC1B002010B504468AB018B906
:10C930004FF0FF300AB010BD002368468DF800307C
:10C9400002F006FC0028F3D19DF804302370F1E7D3
:10C950007FB500220B4620498DF8072001220A707E
:10C9600042784A700446002A33D102790A721A8842
:10C970004A729A788A72DB780B740369CB60C37849
:10C98000164D8DF80830037B8DF8093083680393CA
:10C990002B68DB6A0BB102A898472B689B6B13B11D
:10C9A000227E02B198470E4E052556F8043B1BB176
:10C9B000DB690BB120469847013D15F0FF05F4D126
:10C9C0000DF10700FFF7B0FF637913B1054B0122AA
:10C9D0001A7004B070BD00BFE0020020EC1B002004
:10C9E000081C0020BF1B002010B504468AB018B9EF
:10C9F0004FF0FF300AB010BD202368468DF800309C
:10CA000002F0A6FB0028F3D1024A9DF904302370FE
:10CA10001371EFE7F01B002000B58BB023230190CA
:10CA200068468DF8003002F0B9FC003818BF0120CC
:10CA300040420BB05DF804FB70B5654C01468EB00A
:10CA40001822204606F08CF8624B00221A70FAF782
:10CA5000C5FE23784068012202FA03F1014004D1A7
:10CA60005D4B084608F068F8FEE75C495C481A46EA
:10CA700002F0F8F818B14FF0FF300EB070BD272368
:10CA800004A88DF8103002F089FC564E564D00284F
:10CA900070D1012333702B68DB690BB100209847FC
:10CAA000272304A88DF8103002F052FB059B93F861
:10CAB0004820227093F8182193F81A316270A370FD
:10CAC000464BD3E9020105F03BFF05460028D2D1D1
:10CAD000464E062304A88DF8103002F039FB059B62
:10CAE000736104A802F05AFC022304A88DF81030E8
:10CAF000059602F02DFB0836032304A88DF81030AC
:10CB0000059602F025FB0F2605F0E0FF012304A89F
:10CB10008DF814308DF8106002F040FC10230DEBFE
:10CB200003008DF810308DF8145002F037FC042308
:10CB30008DF8103004A8A3788DF8143002F02EFC84
:10CB40003A238DF8103004A86369059302F026FC9F
:10CB500002A920788DF8086004F09CF8003818BF0E
:10CB60000120E0711420FFF757FFE07903F062F92C
:10CB7000284682E728238DF810302B681B6943B1C3
:10CB800004A802F0E5FA2B6805981B6940F2C4512D
:10CB90009847272304A88DF8103002F0FFFB50B906
:10CBA000012304A88DF8103002F0D2FA9DF8143059
:10CBB000002B7FF46EAF3378002B7FF46CAF05222F
:10CBC00004A88DF81020059302F0E8FB78E700BF79
:10CBD000F01B0020BF1B002018770308C41B002097
:10CBE000DC1B0020CC1A0020EC1B00202C1C002099
:10CBF00037B500230D4601930446D0B900F0A8FBD9
:10CC00000190019BD3B10F4A42F824300E4A9A6238
:10CC10000E4A1268916B1963916C596392690C49C1
:10CC2000D9625A6128465B680A49F2229847002077
:10CC300006E001A900F092FB0028E2D04FF0FF309F
:10CC400003B030BD081C0020E9C40008EC1B002024
:10CC5000C5C50008CD1A0020194B07B51860194B3F
:10CC6000194A1A60194A5A60194A9A60194ADA60D0
:10CC7000194B02681A6042685A6082689A60C268FA
:10CC8000DA60164A1A6182695A61154BC26B5A60A2
:10CC9000144A019119609A601946134ADA6000201B
:10CCA000FFF7A6FF48B901A800F056FB003818BFEF
:10CCB0000120404203B05DF804FB4FF0FF30F9E77C
:10CCC000EC1B0020DC1B002051C6000851C90008E5
:10CCD00065CD0008EDC50008C41B0020450C010807
:10CCE0001C1C0020B9C40008D1C4000849B118B107
:10CCF000012804D000207047034B0B60FAE7034B78
:10CD0000FBE74FF0FF307047000400010100010213
:10CD100008B503F0ABF8002814BF6FF00100002045
:10CD200008BD08B502F084F9002814BF6FF00100B7
:10CD3000002008BD10B504468AB018B94FF0FF3086
:10CD40000AB010BD212368468DF8003002F000FAC9
:10CD50000028F3D1024A9DF9043023705371EFE7A4
:10CD6000F01B00202DE9F0412F4D304F00232B7098
:10CD700043786B703B689B6A8AB004460BB12846C7
:10CD80009847DFF8AC80002658F8043B1BB11B6ABB
:10CD90000BB1204698470136F3B2052B76B2F3D19A
:10CDA0002378052B2FD00B2B35D0012B25D1214CEF
:10CDB000062368468DF8003002F0CAF90199E0793F
:10CDC00005F004FE10B91C4B019A5A611B48FFF78D
:10CDD0000BFE1B48FFF7AEFF6B788BB9A371194BA5
:10CDE0005878FFF75BFD3B685B6A0BB111489847C9
:10CDF0006B7813B9E07905F07BFE0AB0BDE8F081ED
:10CE0000FF23A371EFE7104B01225A74227A9A7420
:10CE1000627ADA74F1E76378002BEED00AB0BDE8ED
:10CE2000F041FFF7CFBB00BFF4020020EC1B002055
:10CE3000081C0020100300202C1C002014030020DC
:10CE400015030020F01B0020E002002030B58BB05D
:10CE5000FFF767FF0446F0B903F0FCFE831C1DD00A
:10CE6000F8B9134D2B685B69DBB1272368468DF851
:10CE7000003002F06DF92B6801985B694FF4B961DD
:10CE8000984703F0F9FE78B92CB9094B1B68DB69A8
:10CE90000BB10120984720460BB030BD6FF007045E
:10CEA000EFE74FF0FF34ECE74FF0FF34F3E700BF5C
:10CEB000EC1B0020014B1878704700BF601C00205D
:10CEC000014B5878704700BF601C0020704700007D
:10CED000044B9A7A0AB101225A70034B5B6903B181
:10CEE00018477047601C00201C03002073B5224CBB
:10CEF0006378002B33D008F007F966680546FFF722
:10CF0000D3FB0644AE4214D2A37A93B1E0228DF84B
:10CF100000208DF80130217AE368019301226846F0
:10CF2000FFF7F2FB08B1073010D100236370A37242
:10CF3000656094F83430EBB1002384F834300F4B43
:10CF40005B6BBBB102B0BDE87040184740F2DC51EA
:10CF50000B4808F0A5F90A4808F068F9E8E794F8E2
:10CF60003520002AE5D094F8360084F83530FFF7F4
:10CF700095FCDEE702B070BD601C00201C030020A1
:10CF8000441C002037B5104D104CC8B1C1B16272BD
:10CF9000012300222860E16023700D480D4B0092B0
:10CFA0004FF0FF3108F096F800250B48258220222B
:10CFB000294605F0E9FD6570A574A58603B030BD6E
:10CFC00000232B602370EFE75C1C0020601C002016
:10CFD000441C0020D1CE0008741C00202DE9F0472D
:10CFE0008E4C23788CB0002B56D0C2780AB9837B44
:10CFF00013B1238A01332382437B002B4CD0E02AD8
:10D000004AD10023A372876897F80080B8F1220FF5
:10D0100027D8B8F1220F30D8DFE818F04100FB0024
:10D0200052005A0061006E0075008E009D00B40031
:10D03000C7002F002F002F002F002F002F002F00E0
:10D040002F002F002F002F002F002F002F002F0068
:10D050002F002F002F002F002F002F00C900D0001D
:10D06000D400B8F17E0F00F0CC80B8F17F0F00F053
:10D07000DF80B8F17D0F00F0AB80A57A002D00F0C5
:10D080005B81674C637A3BB94FF47A71204608F0B4
:10D0900007F9204608F0CAF80CB0BDE8F087E3684D
:10D0A00001220021A2721970A37AE1689818A07277
:10D0B0000620C854A37AE1689818A072CA54DCE725
:10D0C000584B9B6A002BD8D0012102209847D4E707
:10D0D0007B7884F83630012384F83530CDE704239B
:10D0E0008DF804307B78003B18BF012301A88DF830
:10D0F000083002F053F9C0E77878003818BF0120F3
:10D1000002F098FEB9E7484E0FCE01AD0FC50FCE25
:10D110000FC596E8070085E807007B780A2BACD896
:10D12000424A12685268002AA7D00CA901EB830377
:10D1300053F82C0C9047A0E77878431E012B9CD81D
:10D140003A4B01381B6818BF012020729B68002BE6
:10D1500093D0984791E7E26801230821A3721170E8
:10D16000627A057BA17AAA4228BF2A46934284D2DA
:10D1700085685A1CEB5CE56801334E1CA6726B5443
:10D18000D3B2EDE7E3680122A27209221A70A37AF2
:10D19000E268218A581CA072D154A27A238AE168DD
:10D1A0001B0A501CA0728B5467E7238265E7052396
:10D1B0008DF8043001A802F077FB5EE7194BDB6ABB
:10D1C00098475AE7194B78781B686075DB68BEE7AB
:10D1D000037B072B7FF451AF06238DF80430B7F89B
:10D1E0000130ADF808307B793A791B0443EA022319
:10D1F000FA781343642253430393BB798DF81030BC
:10D20000D8E73B2201A88DF804208DF8083002F001
:10D21000C5F8012384F834302FE700BF601C0020DC
:10D22000441C00201C0300207C1E03085C1C002002
:10D230002A2301A88DF8043001F08AFF94F80A909F
:10D24000E6689DF808009DF809509DF80A709DF861
:10D250000BC09DF80D309DF80E209DF80F109DF825
:10D260000CE009F1010A84F80AA006F80980354E9D
:10D2700094F80A903668D4F80C8009F1010A84F811
:10D280000AA096F803A008F809A094F80A90D4F828
:10D290000C8009F1010A84F80AA096F802A008F8A7
:10D2A00009A094F80A90D4F80C8009F1010A84F8D6
:10D2B0000AA096F801A008F809A094F80A9009F1CC
:10D2C000010A84F80AA096F80080E66806F809804A
:10D2D00094F80A80E66808F1010984F80A9006F8D3
:10D2E00008C094F80AC0E6680CF1010884F80A80C6
:10D2F00006F80C70A77AE66807F1010C84F80AC0FA
:10D30000F555A57AE6686F1CA7727055A07AE56896
:10D31000461CA6722954A17AE0684D1CA57242549D
:10D32000A27AE168501CA0728B54A37AE268591C5F
:10D33000A17202F803E0A0E6034807F029FF657038
:10D34000AAE600BF5C1C0020441C002070470000BF
:10D35000004870471C030020002070474FF0FF304A
:10D3600070470000044B054A93F81831022B18BF90
:10D37000062382F89034704704230020C828002038
:10D38000034BD3F8483313B15B6903B118477047B7
:10D39000C8280020034A137843F004031370FFF7F2
:10D3A000EFBF00BFAC1C00201FB50A4B8DF8090071
:10D3B00093F87C208DF80A2093F88C2093F848008D
:10D3C0000D3202A98DF8082003F064FCC0B205B04C
:10D3D0005DF804FB0423002008B5074807F0D8FED9
:10D3E000064B93F81A2412B1012283F81924BDE8E0
:10D3F0000840FFF7C5BF00BFC82C0020C828002088
:10D4000010B50C4CD4F8403343F08003C4F84033DB
:10D4100094F81A3413B10020FFF7DEFF94F891342A
:10D4200023F0120343F0120384F89134BDE8104056
:10D43000FFF798BFC82800202DE9F041DFF8AC8045
:10D4400098F81831022B06460D4602D0284BDB6AAD
:10D45000984702F0A6FD044628B1022002F097FD8D
:10D46000002002F099FD98F81831012B17D102F035
:10D470009AFD074630B1002002F08AFD002002F03C
:10D480008CFD3C4602F091FD48B1002002F081FD88
:10D49000002002F083FDBDE8F041FFF763BF002CE0
:10D4A000F9D1144C94F8902494F81A34BAB90BB109
:10D4B00084F84164304602F017FFD8F82C0007F0DA
:10D4C0002DFED4F8B4339842E5D30B4807F060FE44
:10D4D00094F8913443F0100384F89134DBE70BB1F6
:10D4E00084F84154284602F0FFFEF1E704230020AF
:10D4F000907E0308C8280020602C0020074A10B541
:10D50000137843F002031370FFF73AFFBDE81040B1
:10D51000034B01220021022007F00EBBAC1C0020AF
:10D5200061770308074A10B5137843F008031370B6
:10D53000FFF726FFBDE81040034B01220021022027
:10D5400007F0FABAAC1C0020717703082DE9F0410E
:10D550000F4616461D46804607F0D6FD0B4A0C4C7A
:10D560001378278123F0110343F01103C4E9000865
:10D57000137066812573FFF703FFBDE8F041054B8B
:10D5800001220021022007F0D7BA00BFAC1C002006
:10D59000981C00208177030813B507F0B5FD0D4BEB
:10D5A0006C461860204607F003FD94E803000A4A21
:10D5B0000A4B83E80300137843F020031370FFF74E
:10D5C000DFFE074B01220021022002B0BDE810401F
:10D5D00007F0B2BAA81C0020AC1C0020002C0020D0
:10D5E0008E7703082DE9F04192B0064602F0D9FC8F
:10D5F000002840F05881AD4D95F81831012B09D025
:10D600002B6BAB4C93B194F80431BBB1042B6FD0AE
:10D61000032003E002F0C7FC18B10F2012B0BDE8F0
:10D62000F08102F0C2FC0028EAD0F6E7B5F820311C
:10D63000D4F81C24013B53432B63E4E79D4803F0DB
:10D6400060FA002840F0128194F80C3123802B6B93
:10D650000C930DF1180895F839308DF838304046A4
:10D6600095F81C318DF83A3007F0C8FCD5F8283110
:10D67000009302AF98E80600D5F82431384607F049
:10D6800054FC97E803000FAB83E80300EB6A0D93AB
:10D6900000238DF844302388ADF8463095F83031BA
:10D6A00001228DF839201BB98DF844208DF83930CE
:10D6B000814B0093814B95F84800A3F179020CA9A6
:10D6C00003F05DFBC0B10B28A8D1D4F8941499B134
:10D6D000002EA3D0D4F84033794843F02003C4F897
:10D6E000403307F0DDFD764807F0A0FD002095E708
:10D6F000704803F03AFAA4E795F8487095F9693054
:10D7000095F9392095F87D106E4E384603F044FBAC
:10D71000009641B2EB6C95F850203846183603F06D
:10D72000DFFA0096EB6C95F8502095F9701095F89B
:10D73000480003F0D5FAD4F8C413AB6DD4F8DC2359
:10D740000B44C4F8B033EB6D1344C4F8B43394F80D
:10D750000431042B07D02B6E0B44C4F8B0336B6E2E
:10D760001344C4F8B4330023089395F83031002BE8
:10D7700040D100238DF8133095F839308DF82130E1
:10D7800095F838308DF82230D5F880300993D5F8E7
:10D7900084300A932388ADF82C3095F8303194F812
:10D7A0001B648DF82E3095F84800474B8DF82060AB
:10D7B0000DF1130208A903F0A7FA012384F84134FC
:10D7C00095F8393084F842349DF8133084F84334A6
:10D7D000D4F81C34C4F85064C4F84834C4F858343D
:10D7E00002F0E5FBC8B1D4F81C0402F0F2FBA0B1D2
:10D7F000102013E708A802F0A7FC60B995F93900DA
:10D8000094F837629DF82070FFF7CEFD3E44B04299
:10D81000AFD2082002E7132000E795F81831012B5A
:10D8200001D102F0D8FB02F0C5FB0023059394F868
:10D83000043195F9395094F81B649BB1042B7FF4A3
:10D84000E7AE05A802F0B4FE58BB94F8183413B143
:10D85000059B013B0593174B05983246E9B202F050
:10D860000DFF02E0134802F0DDFE08B11120D5E6FD
:10D87000D4F8403394F80C11218043F00203C4F82B
:10D88000403394F8183411480133DBB284F818346B
:10D8900084F845340E4B00259B6AC4F89854984789
:10D8A00024E71220BAE60E20B8E600BF04230020C9
:10D8B000C8280020D0290020342300205C2D00201F
:10D8C000302C0020802C0020E42C0020CA280020CE
:10D8D000907E030873B5134D134E0096EB6C95F8CC
:10D8E000502095F9781095F8480003F0F9F995F86B
:10D8F0003031337595F8480040F2012306F13C02BF
:10D900003146738203F0F8F950B196F83C3086F84E
:10D910008230064B00205B6B9847F37C86F8A8307A
:10D9200002B070BD04230020B02C0020907E0308BC
:10D93000F8B5324C94F81831012B05460ED0022B65
:10D940004ED0002B57D138B9D4E91B0104F1740330
:10D9500083E803000020F8BD012806D102F02CFB6B
:10D960000028F8D184F81851F5E7022843D1244E55
:10D9700084F8180106F5747CBCE80F0006F57A7788
:10D980000FC79CE8030094F8E92094F8003187E879
:10D99000030086F8FB53D2B1022B18D1D4F804311E
:10D9A0006367C6F8EC3394F87D3094F8082186F864
:10D9B000F83394F88C3084F8782086F8F93396F8A8
:10D9C0001B2486F8E82340F20133A6F8FA3300233B
:10D9D00086F81A340B4BDB6A9847FFF77BFFB9E7F1
:10D9E00048B9074B84F81801062283F89024054BA8
:10D9F000DB6A9847AEE70320ADE700BF04230020B1
:10DA0000C8280020907E0308F0B5504C504EB4F862
:10DA1000DC202287D4E92D0194F8B12084F8692014
:10DA200004F16C0282E80300D4E92F0104F17402CE
:10DA300082E80300B4F8C420A4F87C2091B0D4F8A4
:10DA4000CC20D4F8C810C4F884200025D4F8D02005
:10DA5000C4F888200123A4F82031C4F8801084F889
:10DA60003051A56284F81B5184F83A5084F81D5156
:10DA700084F81E51C4F83451C6F89854A6F81854C6
:10DA800086F81A54A4F838518DF8183004F5097343
:10DA9000039304F50A7394F84800049303A92D4BEB
:10DAA00084F84551C4E94F55A4F84651059303F055
:10DAB000FFF8E36EC6F8D43394F87D3086F8E0338F
:10DAC00094F88C3086F8E1334FF48073A6F8E23393
:10DAD00086F8D05394F8303186F8E43306F574773D
:10DAE0000FCF06F57A740FC497E8030040F20123C4
:10DAF00084E80300A6F8FA33D6F8483386F81B54B6
:10DB0000CDE901551BB15A685B6901920293124B32
:10DB10000793A3F148020892A3F1140209920F4A55
:10DB20000B9229330A93A2F19C030C93A2F1980360
:10DB30000D93131D0E9301A902F14C0307A802F5E2
:10DB400099620F9302F022FA11B0F0BD0423002075
:10DB5000C8280020B01C0020302D0020E823002021
:10DB6000F8B50D4F0D4E0C4607F012FB3B6B984776
:10DB70000B4A96F84800214603F0BEF850B1094D13
:10DB8000706D95F8243485F86A347B6B9847E37C94
:10DB900085F89034F8BD00BF907E03080423002070
:10DBA000EC2C0020C82800200F4890F81B3480F887
:10DBB000B8330E4B93F8692080F8BB2393F87D208F
:10DBC00080F8C82393F88C2080F8C92393F830316B
:10DBD00080F8CC330022A0F8CA2300F56E7100F55E
:10DBE0006070FFF7BDBF00BFC828002004230020DD
:10DBF000114890F89034EBB190F81B3480F8D03392
:10DC00000E4BDA6EC0F8D42393F87D2080F8E02321
:10DC100093F88C2080F8E12393F8303180F8E433D6
:10DC20004FF48072A0F8E22300F5747100F566707D
:10DC3000FFF796BF704700BFC828002004230020CC
:10DC400070B5344C2421204604F0A0FF636A98424A
:10DC500018BF60624FF01C012F4814BF012500253A
:10DC600004F094FF636C984218BF60644FF48071B5
:10DC70002A4818BF45F0020504F088FFD4F848315F
:10DC8000984218BFC4F848014FF0D401244818BF87
:10DC900045F0040504F07AFFD4F82032984218BF0A
:10DCA000C4F820024FF000011E4818BF45F00805D7
:10DCB00004F06CFFD4F82432984218BFC4F8240250
:10DCC0004FF46071184818BF45F0100504F05EFF6E
:10DCD000D4F8A835984218BFC4F8A8054FF014012D
:10DCE000124818BF45F0200504F050FFD4F8C035A5
:10DCF00098420F4B18BFC4F8C005D3F8483318BF7B
:10DD000045F040052BB11B691BB12846BDE87040AA
:10DD1000184770BD042300202C2300204C23002032
:10DD200050240020282500202C250020B028002089
:10DD3000C82800202DE9F04F8FB04FF00009012BCB
:10DD400006460F4690468DF80D90ADF8109002D81B
:10DD50004C46BC4202D30FB0BDE8F08F305D02F0FC
:10DD600033FA2044B842F6DC335D651C023BEDB269
:10DD7000112BF0D801A252F823F000BFC5DD000836
:10DD8000EFDD0008EDDE000815DF000893DF000876
:10DD9000B9DF00081FE0000847E00008CDE00008F8
:10DDA00057DD000857DD000821E1000857DD0008B5
:10DDB00057DD0008C9E10008F1E1000829E2000888
:10DDC0005DE20008052002F0A7FA70B105210020ED
:10DDD00002F068FA725DBA4BE51C0234E4B283F8D3
:10DDE0005C24325D83F85D24EDB22C46B1E700235C
:10DDF0008DF80E308DF80F308DF814308DF8183006
:10DE0000B9F1000F6DD1AF4C4FF0050994F87C20AB
:10DE10008DF831206B1E94F839208DF8332033446F
:10DE200094F838200B938DF8342094F81A3194F834
:10DE300068208DF83520D4F82C218DF832300A92E4
:10DE400073B37B1C5B1BDBB28DF8303006AB0193E8
:10DE500005AB009394F848000DF10F030DF10E028D
:10DE60000AA902F05DFF8DF80D0000F007000728F9
:10DE700013D194F939209DF90E3084F839309A4243
:10DE80009DF80F3084F83830B8BF01229DF8143067
:10DE9000B8BF84F81D2184F868304FF0000A09E00B
:10DEA0000523D1E701220DF10D01032002F0A4F8B2
:10DEB0000AF1010A5FFA8AF29DF81830B3FBF9F112
:10DEC0009142EFD82B44DDB26B1EDBB29F420BD9DF
:10DED000F25C032A9AD0AF4288BF1D464FF0010979
:10DEE00083E70534E5B2F9E71D46F7E7735D754949
:10DEF00003F00F03012281F81B31023402FA03F30D
:10DF0000A1F82031E4B2002204A9042002F074F840
:10DF100025466AE707238DF80D30735DC3F30212BF
:10DF200003F00F038DF82830E31CDBB28DF82920B5
:10DF3000F25C231DDBB2651DF35C0234E4B21B040A
:10DF400043EA0223325D5F4C13436422534394F847
:10DF500048000B930AA902F0F2FE00F00703072B1A
:10DF6000EDB28DF80D000CD19DF8283084F870309A
:10DF700084F878300B9BE36663679DF8293084F85A
:10DF800069308DF81000012204A9052002F034F850
:10DF90002BE74B4BD3F8483363B11B6853B1984719
:10DFA00008F03F038DF810008DF81130022204A90B
:10DFB0000620EBE7FF20F3E703238DF80D30735DB8
:10DFC0008DF81C300AAB0693E31CDBB2A51DF25C96
:10DFD000231DDBB206A9F35C1B0443EA0223A21C47
:10DFE000D2B20534B25C134364225343E4B20A93C1
:10DFF00000230B93335D8DF83030324B93F848009B
:10E0000002F0A3FEC3B20028EDB28DF80D30FFF68A
:10E01000ECAE8DF81030012204A90720B6E7735D3D
:10E0200003F00F03012B4FF47A7238BF01235343DF
:10E03000244A0234936503F57A73D365E4B200226F
:10E0400004A9082062E7735D1E4DC3F340128DF8EA
:10E05000152095F84800C3F3001205A903F00F033B
:10E060008DF814208DF8163002F075FE0234013060
:10E07000E4B23FF44DAFBDF81430134AA5F87C303C
:10E080009DF816309DF814A0D05CF3F793FF02239F
:10E09000C5F880000AA995F848008DF828308DF859
:10E0A0002AA002F0F7FD95F93930069040B2984267
:10E0B000B8BF184685F83900002204A9092025E7D1
:10E0C000C8280020042300209B77030803238DF831
:10E0D0000D30735D8DF82830E31CDBB2651DF25CFA
:10E0E000231DDBB20234F35CE4B21B0443EA0223D7
:10E0F000325D1343642253430B93644B0AA993F894
:10E10000480002F02EFEC3B20028EDB28DF80D30AB
:10E11000FFF66BAE8DF81030012204A90A2035E716
:10E12000092002F0F9F8DFF868B1002849D0092188
:10E13000002002F0B7F80023ADF81E30A31CDBB2BC
:10E14000F25CE31CDBB216F803A0735D4FEA0A4AE7
:10E150004AEA022A4AEA030A231DDBB2A51D053456
:10E16000F35CE4B24AEA036A335D4FF47A725343D4
:10E170000AAC1B122046ADF81C3006F019FF454BC7
:10E1800053440693DBF83C3300930DF1180A9AE8E8
:10E190000600DBF8383308A806F0C7FE099B009399
:10E1A00094E80600089B504606F0A4FE9AE8030097
:10E1B00006F0D6FE01F00AFF0123EDB28BF83834E9
:10E1C00013E68BF8380410E60C2002F0A5F80028BE
:10E1D0003FF40BAE0C21002002F064F82C4B93F8B6
:10E1E0009034043B012B7FF600AE01F0EBFEFCE522
:10E1F000A31CDBB2725DF15CE31CDBB2651DF35C5A
:10E200000434E4B21B04305D43EA01231343642168
:10E21000594300F00F0001F0D6FEEDB28DF810006A
:10E22000012204A91120B1E60D2002F075F80028A2
:10E230003FF4DBAD0D21002002F034F8A31CDBB26B
:10E24000154AF05C735D1268251D0334E4B243EA9D
:10E250000020315DEDB201F0B8FEC6E5725DA31C91
:10E26000251D0334DBB2E4B2F15C335D1B0443EAE9
:10E27000012313436420584301F0A9FEEDB28DF849
:10E280001000012204A9132080E600BF042300200F
:10E29000C8280020803DD512981C00200E4B93F812
:10E2A0009124920703D593F88F24012A08D90B49AA
:10E2B00091F81A2122B18A6A501C18BF01328A6271
:10E2C0000022A3F8182483F81A24D3F8402322F05C
:10E2D0000202C3F840237047C8280020042300200E
:10E2E00070B5184C1848194D06F052FFD4F8403359
:10E2F000D4F89804D5F8906023F02003C4F8403394
:10E3000038B106F00BFF864203D2002385F83A307D
:10E3100070BD0120FFF766F90028F9D00B28F7D06F
:10E3200095F8393084F84234092094F8183484F888
:10E33000453484F8410401F0D7FFBDE87040FFF791
:10E34000ADBF00BFC8280020302C002004230020CF
:10E35000094BD3F84023012A0AD008490978C90794
:10E3600008D43AB993F89204013818BF01207047D5
:10E370000020704701207047C8280020AC1C0020F6
:10E38000034BD3F84003431E58425841704700BF27
:10E39000C82800202DE9F04FA9B0EFF3108272B623
:10E3A000DFF8F0B20021DBF80030CBF8001082F388
:10E3B0001088B94C002B00F0E180DAB29B06039282
:10E3C00064D5B64D95F81831022B02D0B44BDB6AF8
:10E3D0009847EFF3108872B6B24F06F095FE3E688C
:10E3E000D4F8B013361A3144AF4806F059FFAE489E
:10E3F00006F01CFFD4F8B413AC48314406F050FFCB
:10E40000AA4806F013FF88F3108894F81A34002BFA
:10E4100000F06B81152312A995F848008DF848305B
:10E4200002F038FCD4F8B4130F900144A04806F071
:10E4300037FF9F4806F0FAFE3B6894F81B24EB6216
:10E440000DAF38468DF870201D9306F0D7FDD5F836
:10E450002831009306AE97E80600D5F824313046FF
:10E4600006F063FD96E803001FAB83E80300D4F8D1
:10E470001C341E9395F8303195F84800003B18BFC6
:10E4800001231CA98DF8713002F00DFC039BDF06FF
:10E4900048D5824DDFF81CA2D5F8E42004929BF801
:10E4A0000020BAF90A809AF90C90A4F88C84002311
:10E4B00063F300020A9384F84434A4F8223484F805
:10E4C0002534C4F82834A4F82C3484F82E34C4F845
:10E4D000303484F82034C4F8343484F83834C4F840
:10E4E0003C346F4B8BF8002094F89024DB6A84F85E
:10E4F0008E9484F88F24DAF80470BAF8086098478C
:10E5000094F88F3413B9694806F042FE3146384614
:10E5100001F045FD8346002800F0EA80A4F87E84DF
:10E5200084F88094039B19071AD55C4B93F8183133
:10E53000022B02D05A4BDB6A98470220FEF712FFEB
:10E5400084F8410401F0D0FE94F81A3413B1012389
:10E5500084F8193494F8913443F0100384F891341A
:10E56000039B5A0703D506210520FEF765FF039B91
:10E570009B0703D504210320FEF75EFF01F02DFD6C
:10E5800094F89124D7065FD5002384F89234D4F808
:10E5900040331E0644BF23F08203C4F8403312F018
:10E5A000050F00F0FB820B2001F0B6FE002800F002
:10E5B000F58294F89134DD0700F1F082580740F1BC
:10E5C0000783D4F8403323F00203C4F84033D4F86F
:10E5D000402382BB94F8915415F001011EBF2B46D5
:10E5E00062F3000384F8913494F891345E0744BFD9
:10E5F0006FF3820384F89134012384F8923421B1BB
:10E60000D4F844332C481B6898476D070BD52B482A
:10E6100001F08EFE01F0BCFE28B194F8913443F075
:10E62000040384F8913401F0C6FC94F891346FF33C
:10E63000041384F89134012384F8923494F89134CB
:10E6400043F0200384F8913494F8913418070AD5E4
:10E650006FF3C3031A4984F89134D4F84433A1F119
:10E660002400DB68984794F8913499070AD56FF332
:10E670004103134984F89134D4F84433A1F16C0078
:10E680005B68984794F89034022B1BD1FFF722F96E
:10E6900018E000BFAC1C0020C82800200423002084
:10E6A000907E0308A81C0020482C0020602C00202D
:10E6B000C82C0020981C0020082D00201C2D0020B4
:10E6C000542D002094F891349A0640F1C4826FF3DF
:10E6D000451384F89134D4F84033002B40F0BB82CA
:10E6E00029B0BDE8F04FFFF7ABBA84F84134A3E698
:10E6F00095F81831012B0CD101F055FC804668B11A
:10E70000584601F045FC584601F047FC042384F8C4
:10E710008F347EB9012384F821344FE101F045FCA8
:10E720000028F6D0404601F034FC404601F036FCAB
:10E730000523ECE73B7805935B09013B062B00F2D0
:10E740001782DFE813F0070015029500150292000A
:10E7500015020602102EDDD995F830311297F6B267
:10E760008DF84C60002BD5D11CA804F021F912AA19
:10E770001CA9FF2002F09EF89DF85830C3F3030354
:10E7800007468DF82C3095F8480095F87D308DF8C7
:10E790002D3007220BA902F090FA002F5DD100283E
:10E7A0005BD09DF853309DF852201599C5F8E410C0
:10E7B0001B0443EA02239DF8512002201343C5F8AD
:10E7C000E03004F003F99DF8583095F8480085F8DA
:10E7D0002E71C3F30212C3F3030385F8703085F87A
:10E7E00078309DF8593085F86920012B38BF012316
:10E7F0004FF47A725343AB651344EB650DF15A0342
:10E800004FF001081093113E94F81B348DF83C3002
:10E810000FA985F868808DF8446002F056FA02234B
:10E82000404685F8303101F077FD18B14146384651
:10E8300001F038FD94F88F34012B00F2A78194F891
:10E840001A34002B40F09A8194F8913443F010036D
:10E8500084F89134FEF786FD64E6012001F05CFD4A
:10E860000028E7D001210720E2E7012384F82034C3
:10E8700095F87D308DF82E3094F824348DF82D30B5
:10E8800095F88C3095F848000D330BA98DF82C3095
:10E8900002F000FAA6F10D031BB2099023EAE3731C
:10E8A00000B283423FF736AF0B2E7FF633AFBA4B41
:10E8B00025931CA8FF231C978DF874608DF8983061
:10E8C00002F0C4F8074600287FF424AF95F8183109
:10E8D000012B13D101F067FB002872D0384601F0FC
:10E8E00057FB384601F059FB04239DF87C101E9815
:10E8F00084F88F34C1F3001101F06EFB9DF87C3079
:10E900001E99C4F8341413F00F0203D09DF8900040
:10E91000002862D19DF89800002861D0002A7FF479
:10E92000F9AE9DF89020002A14BF4FF003084FF075
:10E93000020800220A92D5F8EC2095F8E9009142ED
:10E9400051D100284FD0D5F80C1195F8EAB00968DC
:10E950000A9195F81811022902D1032184F88F1425
:10E96000B8F1030F7FF4D6AE13F0600F7FF4D2AE90
:10E970000492012795F82E31BBF1000F36D0BBF180
:10E98000010F13D1012B33D16FF0090646FA08F6B7
:10E9900006F00106C6F10206F6B2BDF87E100AAA1C
:10E9A000304601F011FE38B3072823D0012384F844
:10E9B00021340A9BC4F83034C4F86C34FEF720FDCF
:10E9C000B0E501F0F2FA002898D0384601F0E1FAFB
:10E9D000384601F0E3FA052387E74FF00008A8E77F
:10E9E0004FF00108A5E74FF0010BC3E70426D4E779
:10E9F0000326D2E70823DAE71CAB009304990A9BAD
:10EA00003246584601F0A2FE20B1022814BF0B2363
:10EA10000A2380E60A9BC4F83034C4F86C349DF8AD
:10EA20007C3084F82104C3F3401384F82E3484F836
:10EA3000443494F88F3484F82274012B9EBF012251
:10EA4000A86285F81E21012FC4F8280484F82C043C
:10EA500084F8410438D1022284F8202495F83A2021
:10EA6000002A4AD19DF87C20D60646D4012B94F882
:10EA700040149DF87C2005D8012901D1900601D5CC
:10EA800001F04CFBB8F1020F94F88F3443D0B8F189
:10EA9000030F0AD09DF87C10B8F1010F4A4601F02F
:10EAA0000F0120A83BD0FFF745F99DF8903084F87E
:10EAB0002334259BC4F828349DF8983084F82C34EE
:10EAC000012384F82D3430E0059A02F0E002A02AF8
:10EAD0001BD195F82E11012285F83A2009B9279902
:10EAE0006963012B84F8202407D9D5F89020C4F855
:10EAF0003C24DAF80020C4F8982495F81821002A5C
:10EB0000B4D1012284F82524B0E7002285F83A2008
:10EB100084F82024A6E79DF8981025984A46FFF728
:10EB200009F99DF8903084F823349DF89020E02A6C
:10EB300008D195F81F312BB984F82324C4F8283460
:10EB4000A4F82C3494F8913443F0020384F89134FF
:10EB500070E6114D013EB2B2791C284604F000F86F
:10EB60000323A4F82034C4F8285484F82C64E9E77B
:10EB7000012384F82134FEF743FC5BE694F8443427
:10EB8000002B3FF461AE0020FEF726FC94F88F3492
:10EB9000022B3FF45FAE57E6002B002094F891342F
:10EBA000590715D5012001F0B7FB60B1012001F034
:10EBB0008BFB08B984F81804D4F8403323F002031F
:10EBC000C4F8403304E0062001F0A6FB0028F3D18E
:10EBD00094F89134DA077FF5FAAC94F840240AB13E
:10EBE000032A18D11D4A94F8181492F8682091420B
:10EBF00005D29B0723D594F88F34012B1FD81848D2
:10EC000006F0C6FAD4F8403323F02003C4F84033AA
:10EC1000FFF744FBDBE4012A11D194F81924002A00
:10EC20003FF4D5AC0D4A94F8181492F8682091423C
:10EC3000E5D29F0703D594F84434002BDFD194F834
:10EC4000913400206FF3041384F8913484F819048C
:10EC5000FFF746FBBBE429B0BDE8F08F042300209A
:10EC6000302C00202DE9F04F89468DB090460746A4
:10EC7000002800F08F81002900F08C810368002BB0
:10EC800000F088814368002B00F084818368002BAA
:10EC900000F08081C368002B00F07C81104601F0F9
:10ECA000F5FF002800F07881BD4CBE4D384601F0DC
:10ECB000AFFA40F2C4520021204603F065FF40F253
:10ECC0001C520021284603F05FFFB74BC4F82C31DB
:10ECD00004F50973089304F50A7300264046099366
:10ECE00008A9B24B84F848800A9384F8186184F824
:10ECF0008C608DF82C6001F0DBFF0F2306A994F8DF
:10ED000048008DF8183001F0C5FF801B18BF0120A6
:10ED10004FF00A0B84F81C0106A994F848008DF8FE
:10ED200018B001F0B7FF4FF0060A84F8DC0006A91E
:10ED300094F848008DF818A001F0ACFF102384F877
:10ED4000DD0006A994F848008DF8183001F0A2FF04
:10ED50001123C4F89C0006A994F848008DF81830D7
:10ED600001F098FF1223C4F8A00006A994F8480007
:10ED70008DF8183001F08EFF1323C4F8A40006A903
:10ED800094F848008DF8183001F084FF1423C4F87B
:10ED9000A80006A994F848008DF8183001F07AFF11
:10EDA0001623C4F8AC0006A994F848008DF8183072
:10EDB00001F070FF172384F8B10006A994F8480009
:10EDC0008DF8183001F066FF18230DEB0301C4F82D
:10EDD000B400C4F8BC0094F848008DF8183001F075
:10EDE00059FFC0B21D2384F8B80084F8C00006A9FA
:10EDF00094F848008DF8183001F04CFF1E2384F879
:10EE0000C40006A994F848008DF8183001F042FFBC
:10EE10001F2384F8C50006A994F848008DF818301F
:10EE200001F038FF2023C4F8C80006A994F8480070
:10EE30008DF8183001F02EFF0B23C4F8CC0006A982
:10EE400094F848008DF8183001F024FF0C2306A92F
:10EE5000A4F8D00094F848008DF8183001F01AFF9B
:10EE6000D4F89C306365D4F8A030A365D4F8A430FE
:10EE7000E365D4F8A83023664FF00108D4F8AC302D
:10EE80000590A4F8D200636684F8B080C4F894B00A
:10EE900084F898A0C4F84CB084F850A084F8688036
:10EEA00084F81F81C5F84893FEF7AEFDC5F844739A
:10EEB000C4E90B663E4B84F8198185F89164C5F866
:10EEC000408332464FF0FF31009605F55A7006F048
:10EED00001F9384B009632464FF0FF3105F560706E
:10EEE00006F0F8F8344B009632464FF0FF3105F546
:10EEF000667006F0EFF802AF304B009632464FF0E6
:10EF0000FF3105F5806006F0E5F8384606F076F842
:10EF100097E8030004F5927383E80300284B294F18
:10EF20001E60294BC5F84C33284BC5F85433284B89
:10EF3000C5F85C33274BC5F85033274BC5F8583319
:10EF400005F553703B68984704F5A67003F04CFB39
:10EF500020B1112630460DB0BDE8F08F204601F0FB
:10EF600003FB0028F5D101F039F8B8B91B4801F0CE
:10EF70004DFB06460028ECD17B69984703F0CEFD97
:10EF8000BB6D94F819019847FB6A9847012385F8EF
:10EF90009234DFE70326DDE70926DBE71326D9E70E
:10EFA00004230020C828002000040001B01C002019
:10EFB000E1E20008A9DB0008F1DB0008D9D3000872
:10EFC000AC1C0020907E030899D500084DD50008A0
:10EFD00095D3000825D50008FDD40008EC230020B7
:10EFE00008B5034B0020C3F84003FEF7BBF908BD8A
:10EFF000C828002010B5FFF7ABF90A4C60B90A4BDE
:10F0000093F81831022B02D1084BDB6A9847012391
:10F01000C4F84033002010BDD4F84003013818BFB5
:10F020000120F8E7C828002004230020907E030870
:10F0300038B5124C204606F0ABF804F1180006F083
:10F04000A7F804F1300006F0A3F804F1980006F0E8
:10F050009FF800F0AFFF0A4B0025DB6A984744F8A1
:10F06000285CFEF7EDFD0749074840F2C45203F063
:10F0700077FD012344F8283C284638BD302C002079
:10F08000907E030804230020401D002070B52E4B05
:10F090008AB0054693F8DD008DF8090093F8DC008E
:10F0A0008DF80A0029489A6A90F8180403920026FD
:10F0B0008DF80B0004960C46002940D00692D3F838
:10F0C000882007921A8F93F81A118DF8151052BAEA
:10F0D000ADF8202093F87C2093F848308DF8243048
:10F0E00003AB8DF822008DF8232000930DF10A0266
:10F0F0000DF10B030DF1090105A88DF8146000F066
:10F10000D7FE9DF90900FEF74FF9607004A801F0E1
:10F110001BF8B0B9049A0F2A0DD863789A420AD81E
:10F120001544AB42A3EB02012CBF0020012021704B
:10F13000C0000AB070BD002323700820F9E7032047
:10F14000F7E71320F5E700BF04230020C8280020BC
:10F150001FB50446002800F010810378412B00F20F
:10F160000781DFE813F0420049004D0051005500CF
:10F1700059005E00050105010501050105010501B4
:10F1800005010501650069006D0078007F008200BF
:10F1900085008A0088008C009000930096009900FA
:10F1A0009C009F00AE00B200BA00B600BE00C100D5
:10F1B000C500CE00CA00CC000501D2000501050142
:10F1C000050105010501050105010501050105010F
:10F1D00005010501050105010501DA00DE00E20077
:10F1E000E700EB00EF00F300FC00664B93F81831EA
:10F1F0002371002004B010BD624B93F83031F7E763
:10F20000406803F08FFBF4E7406803F0D1FBF0E7C0
:10F210005C4B93F81A31EBE75A4BD3F8E03063605C
:10F22000E7E7584B011D93F8300103F0D9FBE0E705
:10F23000544B93F81931DBE7524B93F88C30D7E7F6
:10F240001C238DF808304F4B02A993F8480001F0B9
:10F2500021FD6060CDE74C4B043493E8030084E863
:10F260000300C6E7494B0434F7E7494B0434F4E79D
:10F27000484B0434F1E71A23E3E71923E1E7414B54
:10F2800093F86830B4E73F4B5B6DC8E73D4B9B6D2F
:10F29000C5E73C4BDB6DC2E73A4B1B6EBFE7394B12
:10F2A0005B6EBCE702238DF80830364B02A993F859
:10F2B0007C2093F848008DF80A2001F0EBFC2071C7
:10F2C00097E7304B93F8DD3092E72E4B93F83930C7
:10F2D0008EE72C4B93F8DC308AE72A4B93F83830D2
:10F2E00086E7284BDB6C9AE7264B93F850307FE794
:10F2F000244BD3F8843063607BE7224B8FE7264BA7
:10F300008DE7204BD3F8CC30F5E71E4BD3F82C31EA
:10F31000436001F04DFDA0606BE71A4BD3F89030CD
:10F320007DE7184B93F81F3162E7164BB3F888302E
:10F33000A3805EE7134BB3F88A30F9E7114BB3F8BB
:10F34000D030F5E70F4BB3F8D230F1E70D4B93F81F
:10F3500048200AB1062A12D1B3F8A035E8E7094BD4
:10F3600093F848200AB1062A09D1D3F8A43556E704
:10F3700004B0BDE8104000F021BE03203AE7182099
:10F3800038E700BF0423002070230020B8230020AA
:10F3900078230020C0230020401D00207FB50446B4
:10F3A00010B9032004B070BDA34DD5F840339A07BF
:10F3B00000F16F820278412A00F26882DFE812F0E1
:10F3C0004200470055005B005F0064006900760062
:10F3D000810087008D00930099009F00A500AB007D
:10F3E000B5006602BA00DC00EF0016013801290101
:10F3F00042014B014F01530157015B0166025F015E
:10F40000710199018701AB01B101B801BD01C201D0
:10F4100066022802660266026602660266026602EA
:10F42000660266026602660266026602660266029C
:10F4300066026602340239023E02430248024D026D
:10F4400052025C020079FEF773FA30B1AAE7037941
:10F45000022BA6D0794A82F8303195F8913443F0E6
:10F46000200385F8913400209CE7406803F04CFAB3
:10F470000028F2D095E7406803F08AFAF8E76F4B6E
:10F48000027983F81A21E8E76C4B4268C3F8E02060
:10F49000E3E76A4E416896F8300103F097FA0028D6
:10F4A0007FF47FAF6368C6F8E430D6E7416800298F
:10F4B0003FF477AF002001F0DDF90028CDD0112016
:10F4C00070E7416800293FF46CAF0120F3E7416821
:10F4D00000293FF466AF0820EDE7416800293FF4BA
:10F4E00060AF0920E7E7416800293FF45AAF0C20DC
:10F4F000E1E7416800293FF454AF0D20DBE74168A4
:10F5000000293FF44EAF0E20D5E7416800293FF4B3
:10F5100048AF0F20CFE74A4C484B007983F81901D8
:10F52000A36D9847E36A984797E7444B027983F8BD
:10F530008C2092E7414E037A8DF8043096F848000B
:10F5400096F87D308DF80530072201A901F0B5FB52
:10F5500000283FF426AF636896F848000193002224
:10F5600001A901F0AAFB00283FF41BAF6C36D4E9D7
:10F57000010186E8030070E7304E037A8DF804300D
:10F5800096F8480096F87D308DF80530072201A9DD
:10F5900001F093FB00283FF404AFB436E7E7274EB1
:10F5A000037A8DF8043096F8480096F87D308DF88F
:10F5B0000530072201A901F080FB00283FF4F1AEDD
:10F5C000D4E9010106F1740383E8030096F81831C9
:10F5D000022B7FF442AF96F83031002B3FF43DAF61
:10F5E000174BDB6A9847FEF775F936E7134E037A37
:10F5F0008DF8043096F8480096F87D308DF8053087
:10F60000072201A901F059FB00283FF4CAAEBC361D
:10F61000ADE74368029301238DF80C30074B02A934
:10F6200093F8480001F056FB00287FF416AFB8E6C7
:10F63000436802930023EFE7C8280020042300203A
:10F64000907E030803795A1E0E2A3FF6AAAE934A0B
:10F6500082F8683001E7914B42685A65FDE68F4BAE
:10F6600042689A65F9E68D4B4268DA65F5E68B4BA0
:10F6700042681A66F1E6894B42685A66EDE6874CA5
:10F68000037994F848008DF80430062201A901F0AE
:10F6900014FB00283FF485AE9DF8043084F8DD307B
:10F6A000DBE67E4C03798DF8043094F8480094F83A
:10F6B0007C308DF80630052201A901F0FEFA002801
:10F6C0003FF46FAE9DF8043084F83930C5E6734CD2
:10F6D000037994F848008DF804300A2201A901F05A
:10F6E000ECFA00283FF45DAE9DF8043084F8DC307D
:10F6F000B3E66A4C037994F848008DF80430092287
:10F7000001A901F0DAFA00283FF44BAE9DF804306D
:10F7100084F83830A1E6614B4268C3F89420DA647B
:10F720009BE65E4B027983F8982083F8502094E69C
:10F730005A4B4268C3F884208FE6584B4268C3F89E
:10F74000CC208AE6012B40F0A480554C2421204691
:10F7500003F01CFA636A984201D0172022E61C21AC
:10F7600004F1280003F012FA636C9842F5D14FF4CB
:10F77000807104F1480003F009FAD4F84831984246
:10F78000EBD1D42104F5A67003F000FAD4F82032AE
:10F790009842E2D1002104F5097003F0F7F9D4F89A
:10F7A00024329842D9D14FF4607104F50A7003F005
:10F7B000EDF9D4F8A8359842CFD1142104F2AC5019
:10F7C00003F0E4F9D4F8C0359842C6D1334E21464F
:10F7D000304640F2C45203F0C3F9204640F2C4520E
:10F7E000002103F0D1F995F81B3485F8E833736FE5
:10F7F000C5F8EC3396F87D3085F8F83340F20123F4
:10F80000A5F8FA33274B96F819019B6D984724E623
:10F810008379012B3FF6C5AD204B42684068C3F8A1
:10F820002C2100F0BDFE48E61C4B4268C3F8902036
:10F8300013E61A4B027983F81F210EE6174B8288D4
:10F84000A3F8882009E6154B8288A3F88A2004E6ED
:10F85000124B8288A3F8D020FFE5104B8288A3F8D2
:10F86000D220FAE50D4B93F848200AB1062A12D1AE
:10F87000A288A3F8A025F0E5084B93F848200AB128
:10F88000062A08D16268C3F8A425E6E500F098FBD3
:10F89000DBE5012086E5182084E500BF0423002075
:10F8A000401D0020907E03082DE9F04387B000231F
:10F8B000ADF800300646002800F0EE800361FEF748
:10F8C00047FD20B10124204607B0BDE8F08300F0D9
:10F8D00065FD0028F6D100F05BFD014618B96F48C0
:10F8E000142203F051F96E4D95F89134012243F042
:10F8F000040385F8552485F8913433788DF8043065
:10F900000021013B8DF80520ADF806100C2B00F20C
:10F91000BB80DFE803F007B9B9B97982B9B990B90A
:10F92000AD9AA900D5F8407317F02007CAD196F810
:10F930000480B8F1020F46D1DFF868815A4CFEF717
:10F9400063F896F9051098F848003A4601F00FFA66
:10F9500088F83900B37988F83830384607238DF8AD
:10F960000530FDF7E5FFFF2304F58670A5F80C319F
:10F97000C5F8084185F8047103F01AF804F58A7097
:10F9800002F0D0FF3846FDF72DFE0446002839D09E
:10F9900096F9051098F84800012201F0E8F988F876
:10F9A0003900D5F894343361002C71D000F0F0FCAC
:10F9B000002888D195F8913485F81A0460F3820301
:10F9C00085F891347FE7B8F1010F4FF00204E8D1D8
:10F9D000DFF8D0908DF8144099F8480089F81D712F
:10F9E00002A901F065F9337989F830318DF8057095
:10F9F0008DF80680FDF7C4FC95F8913443F01003B0
:10FA000085F891340024CCE700226946022000F0FA
:10FA1000F3FA0028F6D01324C3E7244BB288DB6B3B
:10FA200096F90C10B0689847D5F8403343F00203BC
:10FA3000C5F84033E6E702A90D2000F053FB00288B
:10FA4000E0D0002269460D20E1E7164B93F818310B
:10FA5000D3B9347904F0070000F0ABFA8DF8004018
:10FA6000012269461020D2E7002269461220CEE723
:10FA70008DF8072000F08EFA044638B900F087FAB6
:10FA8000204600F089FABDE702248AE7012488E7CE
:10FA900001A800F0D1FB16E7032414E71C2D002079
:10FAA000C828002004230020CA280020907E0308D4
:10FAB0002DE9F04F99B08046059118B9032019B08F
:10FAC000BDE8F08F00230361FEF742FC04460028E6
:10FAD00040F0A58046460FCE0EAD0FC51422524809
:10FAE00098F800A0B8F80C7098F90EB04F4E214667
:10FAF00003F04AF84E4B012283F8412496F8302156
:10FB0000022A25460BD196F81821022A07D196F829
:10FB10001E2122B9BAF1010F38BF4FF0010ABAF124
:10FB2000010F2BD0BAF1030F2AD0BAF1000F33D155
:10FB300002229DF83C30DDF84090029362F34715B5
:10FB4000012496F87C108DF8321002220CA996F848
:10FB500048008DF8302001F09DF896F81A3196F89B
:10FB600030C196F81D1140B2002B63D0BCF1010FDB
:10FB700057D1002955D1002C61D153E00422D8E798
:10FB80000023DDF83C90BDF840709DF942B002932F
:10FB900065F01F050124D4E74FF0000BD946CDF8DE
:10FBA00008B0CEE74FF0010084F81A04D2E005F265
:10FBB0009A420BA900F0D4FA002800F01581132016
:10FBC000049B33871A4B002283F81A2423E105F2A1
:10FBD0009A452A460BA900F0C3FA0028EFD10B9BE7
:10FBE00084F82801C4F82C5184F83031FCE0B9F1D4
:10FBF000000F00F0F980002A00F0F6804946E01C72
:10FC000002F0AEFF94F8373201332380ECE012208B
:10FC1000D6E70220D4E70720D4E71320D2E701205B
:10FC20004DE7FCB90220F6E0082D00200423002057
:10FC3000C8280020002CF5D05845B8BF584696F883
:10FC40007C308DF82000052296F848008DF822308F
:10FC500008A901F032F800283FF430AF9DF82030B9
:10FC600086F839306F4A704BD2F89804D3F8904038
:10FC700038B105F053FA6C4B84423CBF002283F844
:10FC80003A20198F1A8F93F830010491996A0991DB
:10FC900052BA0028BFD093F81B0100B9186393F83B
:10FCA0001801ADF85820013893F87C2093F81A41D8
:10FCB0001491D0F1000BD3F888108DF85B204BEB3A
:10FCC000000B93F8482093F83A0093F868308DF8C9
:10FCD0005A3009AB0093554B03904FF001008DF85B
:10FCE0004C0015918DF85C20A3F12F01A3F1300297
:10FCF00013A88DF84D4000F0DBF8039B4FEA0B1B77
:10FD00004BEA431B00264BEA801B4BEAC413B14568
:10FD1000444C039308BF37463A46494604F59C7065
:10FD2000CDE90A669B46268084F81A6402F018FF23
:10FD3000E9B2A570C5F34215FAB2042D3A4E039B01
:10FD400084F837223FF42EAF072D3FF450AF022D39
:10FD50007FF45FAF364D84F80D110420029984F8CA
:10FD60000401FF2084F80C0184F8281184F8143170
:10FD7000D6F8E410C4F8085105F59B730AA8C4F836
:10FD8000101184F83021C4F82C3100F011FC002847
:10FD90007FF43DAF0A9BA4F844040BA8A4F81631E5
:10FDA000C4F84C3400F0D0F900287FF408AF0B9B66
:10FDB000D3B196F93900FDF7F7FA94F83732002BF2
:10FDC0003FF405AF0B9B0F2B3FF6F1AE05F58B72A1
:10FDD0000BA90F2000F0C4F900287FF4F0AE0B9BB4
:10FDE00063F3030B84F814B10598FDF7FBFB0028BF
:10FDF0007FF4E6AE099B86F83A00B36200F080F922
:10FE000000287FF40AAF94F8913484F840A443F0BA
:10FE1000010384F89134034BD3F89434C8F81030BC
:10FE20004DE600BFC8280020042300206C230020DA
:10FE3000CA28002037B50B4D8DF8040004460F2268
:10FE400095F8480001A900F038FF40B1064A85F84E
:10FE50001C4192F8913443F0200382F8913403B0AE
:10FE600030BD00BF04230020C828002010B5FFF7D4
:10FE7000C1F8044688B90A4805F08AF9094805F02E
:10FE800087F9094805F084F900F094F8FDF7BCFD06
:10FE9000064BDB6A9847204610BD0124FBE700BFF4
:10FEA000302C0020482C0020602C0020907E03087D
:10FEB0002DE9F04F8BB047780093149B90F90C809C
:10FEC00090F90D6090F80EB08A46416819600446BA
:10FED0009146002F58D002238DF8103004A9C37B1F
:10FEE000007C8DF8123000F0D5FEB4F808C06189AE
:10FEF00043B26068984545466144B8BF1D466045B9
:10FF000034BF00270127884209D30A218DF8101039
:10FF1000207C019304A900F0BDFE019B46B2B4F819
:10FF200008C0608961680CEB400E714519D3A1EBE4
:10FF30000C01B1FBF0FC00FB1C1191B9984503DCEE
:10FF40002378CBB94FF0010B21238DF81030207CA2
:10FF5000E37B8DF8115004A98DF8123000F09AFE61
:10FF600045B2009B8AF80050384689F8006083F853
:10FF700000B00BB0BDE8F08F0223207C8DF8243058
:10FF800006A900F095FEDDE74546EAE770477047B1
:10FF900070477047002070477047704770470020D7
:10FFA00070470020704700207047002070470020F5
:10FFB00070477047704770470220704702207047B3
:10FFC000022070477047002070477047704700203C
:10FFD00070470020704770477047704710B5054C58
:10FFE0004FF403722046002102F0CEFD0020C4E948
:10FFF000000010BDE42D00202DE9F8438146904615
:020000040801F1
:1000000000293CD01F4C2023224604F1100012F896
:10001000017F6FBB8242FAD11B4E3368013403B9B2
:100020003460736803B11C6000252560C4F8088043
:1000300074601FFA88F284F80490601D02F090FD4D
:10004000B9F1110F4FF0000398BF104D6373D6F84C
:10005000083298BF25FA09F503F1010398BF05F0AE
:10006000010543442573C6F808323846BDE8F883D5
:10007000013B13F0FF030446C6D10227F5E7012731
:10008000F3E700BFEB2D0020E42D00202007020045
:1000900010B518B3124A1368984204D1036813606C
:1000A000002305E00B46002BFAD019688842F9D1ED
:1000B0005168884208BF53600BB101681960D2F8DB
:1000C00008328168013B00245B1A04602146C2F8B3
:1000D0000832102202F058FD204610BD0120FCE736
:1000E000E42D0020054B1B6813B11A798242FAD126
:1000F000002B0B600CBF032000207047E42D002074
:1001000010B5054B186800B910BD037B04680BB926
:10011000FFF7BEFF2046F6E7E42D002038B5084B78
:10012000084C186800B938BD03790568112B05D84B
:1001300024FA03F3DB0701D5FFF7AAFF2846F1E70E
:10014000E42D00202007020028B1044BD3F8083228
:100150000360002070470120704700BFE42D00209D
:100160002DE9F04107460E46154642B339B3154B0B
:100170001C6800232CB93046FFF7E6FF0020BDE8DD
:10018000F081A268F91A0132914215D32279EA541A
:10019000581C22895FFA80F8611D55FA80F002F040
:1001A000DFFCA368246898445FFA88F3E2E72046FE
:1001B0002568FFF76DFF2C46002CF8D1DBE7012006
:1001C000DDE700BFE42D00200238C0B211289ABF3D
:1001D000014B185C00207047AB77030830B50B4B20
:1001E00093F820200446084672B100211C3305789C
:1001F000A54208D001319842CDB214BF0430103866
:10020000AA42F4D8002030BD1046FCE7F02F0020B1
:1002100010B5084C00232060142204F10C00FF21CB
:1002200084F82030C4E9010002F0AEFC012384F818
:10023000213010BDF02F002010B50E4A92F820108A
:10024000042915D8936804781C7044785C70C478CD
:10025000807898700131DC7082F8201002F11C0166
:100260008B4214BF043302F10C039360012010BDD4
:100270000020FCE7F02F0020094B93F8200068B124
:100280005A6803F11C018A4200F1FF3014BF0432A6
:1002900003F10C0283F820005A600120704700BF70
:1002A000F02F002010B5074B93F820200446084695
:1002B00032B15968FFF792FF10B101234470837087
:1002C00010BD00BFF02F002008B5064B93F820208A
:1002D0002AB15968FFF782FF08B1407808BD0120B4
:1002E000FCE700BFF02F002030B50A4A92F820103A
:1002F000536882F8210061B1916801241C32DD78D5
:10030000587005B99C70934214BF0433103B994256
:10031000F5D130BDF02F002008B5044B5968FFF728
:100320005DFF003818BF012008BD00BFF02F00207E
:10033000F7B50422154E044600210DEB020096F895
:10034000207002F021FC0025EBB29F4201D803B0DF
:10035000F0BD7368197821705A786270987838B156
:10036000336820469B689847FFF786FF0135EBE727
:10037000DB788DF804108DF805208DF80730FFF735
:100380007BFF01A8FFF758FFF0E700BFF02F002028
:10039000014B93F820007047F02F0020034B93F897
:1003A0002000042894BF002001207047F02F002077
:1003B0001FB50024CDE90244C41F8DF800408DF81C
:1003C00001100C0AADF80420090C120C8DF8031072
:1003D0008DF806208DF8073002461B0A0121684679
:1003E0008DF802408DF8083002F029FA002818BF75
:1003F0000E2004B010BD2DE9F04188B090460D46A6
:100400000F9A0746002847D000240121CDE9044473
:100410008DF810109DF838108DF81510ADF81630C5
:10042000190CCDE900441B0ECDE902448DF81930BA
:10043000ADF81A20130C120E07948DF818108DF8D1
:100440001C308DF81D20E3B21E01002DF6B203DC36
:10045000002008B0BDE8F081013310218DF81F3075
:1004600042466B460DEB010002F07FF90346A8B946
:10047000102D28463E44A8BF10206946327811F856
:1004800001CB013382EA0C02984206F8012BF5DC1D
:10049000103D2DB20134D6E70920DAE70E20D8E767
:1004A0000138032815D8DFE800F002080C100A4BC9
:1004B0001B681B690B6000207047074B1B685B695A
:1004C000F8E7054B1B689B69F4E7034B1B68DB6986
:1004D000F0E70520704700BF143000202DE9F041FF
:1004E000C4B00C464A9E17461D468046B8B3B1F5C7
:1004F000807F36D84FF488720021684602F044FBB2
:10050000492300934FF48073ADF804302B0C8DF821
:100510000830330CADF80650ADF80A608DF80C3099
:1005200022460023414604A82D0E360E8DF80E30CB
:100530008DF809508DF80D608DF80F4002F010FB1A
:1005400004F110014B9A3B4689B2684602F0F7F875
:1005500010B1012818BF0E2044B0BDE8F081092079
:10056000FAE70D20F8E7000010B590B10A4C2822F8
:100570000021206002F008FB2368084A1A6000206E
:100580004FF0FF32C3E90302C3E90522C3E90722A2
:1005900010BD0820FCE700BF14300020000101015D
:1005A000024B1B6818600020704700BF1430002009
:1005B00030B1044B1B68DB680133036000207047D7
:1005C000092070471430002013B500230C46019316
:1005D000CAB101A9FFF764FF18B9019B591C02D1E8
:1005E000146002B010BD99B2611A002901DD5C18D7
:1005F000F6E702D113600720F3E71B0C1B0403F599
:1006000080331C44ECE70920EBE7000028B1044BE1
:100610001B681C334362002070470920704700BFED
:10062000143000201FB5044600B3002303A8039331
:1006300002F05CF9104ABDF80C3012682046938035
:10064000E38200F05EFA98B904F118030093216880
:100650000123132202F068F860B9204600F051FA35
:10066000003818BF0120000104B010BD0920FBE7CD
:100670001020F9E70E20F7E714300020F0B505460A
:1006800087B01C4613B9092007B0F0BD2E4E336861
:10069000DB68834255D894F82020002A0CBF08223A
:1006A0000922834205D3204600F05FFA68B110208A
:1006B000EAE7002301900093A36894F82810606A89
:1006C000FFF799FE0028EED0DEE723792168B4F821
:1006D00008C0A768043B9AB20029D4D0B2F5807F45
:1006E0002DD8ADF80EC08DF817304FEA174C04F135
:1006F0002C033F0E8DF8117000932F0C08234FF040
:10070000490EADF80C008DF814708DF816002F0E00
:100710000DEB0300CDF808E08DF810C0ADF81250D5
:100720008DF8157002F000F808B10E20ACE72046F5
:1007300000F01BFA0028BAD13368DD60A4E70D2071
:10074000A2E70620A0E700BF143000202DE9FF41FA
:100750000A9D80460F4616461C46002D5AD000239F
:1007600003A910460393FFF79BFE18B1062004B0BF
:10077000BDE8F081039B9C4201D80133F6D12846A5
:1007800000F064F9002847D1264B1A78424503D07F
:100790001A79424542D10120AA68BA4240D103EBFE
:1007A0008002EB6A92F801802979CDE9004304398F
:1007B000927828683B4689B2FFF790FE0028D6D190
:1007C00095F820300194002B4FF00103009314BFE3
:1007D0004246082295F82810686A3B46FFF70BFE50
:1007E0000028C4D1013E032EC1D8DFE806F002077D
:1007F0000B0F0D4B1B681C611C62B8E70A4B1B6892
:100800005C61F9E7084B1B689C61F5E7064B1B68C8
:10081000DC61ACE70920AAE70F20A8E70B20A6E7D8
:100820000220A4E754030020143000201FB50B2938
:100830004FF00003CDE90033CDE902330A4607D07B
:100840000C2914D00A2910D00A2005B05DF804FB49
:10085000012802D120238DF800300021684601F0E4
:10086000EEFF002818BF0E20EFE73023F3E70B213F
:10087000F4E7000038B5054601F0DCFF044610B18E
:100880000E24204638BD002DFBD1094B1B680B21DF
:100890009878FFF7CBFF0028F2D10C21FFF7C6FFB5
:1008A0000028EDD10A21FFF7C1FF0028E9D0E7E7D2
:1008B000143000202DE9F04380468FB00C461746D7
:1008C000002A6BD0002969D0002529461D2206A8E0
:1008D00005951DF091FF8DF81350344D2B680DF1E7
:1008E00014099E88CDF804900DF1130302933B790F
:1008F00000933B6832462146404601F0BCFF002889
:100900004ED138683A79494602F02AF9384600F063
:100910004FF8002846D13C7AFA79BB79240444EA9E
:1009200002241C432B689A6894423DD99C609DF830
:1009300013000B21FFF77AFF034658BB0C21FFF78A
:1009400075FF034630BB0A21FFF770FF034608BB63
:100950007B7ABA7AFF7A3F0447EA02271F433A4676
:10096000334621460920FFF723FD034690B933465D
:100970003A4621460820FFF71BFD034650B92A6876
:100980009DF8131091700021D1604FF0FF31C2E942
:100990000411916118460FB0BDE8F0830923F9E70F
:1009A0000E23F7E70F23F5E70323F3E714300020C6
:1009B00010B50446002845D00168002942D011F83E
:1009C000013B43710322063002F0CAF8204603229D
:1009D00050F8091B043102F0C3F82168CB79E360B9
:1009E0000A7A43EA0223E3604A7A43EA0243E36075
:1009F0008A7A43EA0263E360CB7A23740B7B6374E5
:100A00002379212B1AD110220D3104F1120002F0AA
:100A1000A7F81D222168501C8B5C6362085C43EAC6
:100A20000023901C6362085C033243EA0043636264
:100A30008A5C43EA02636362002010BD112B03DC71
:100A40000D22E7E70220F8E70120F6E710B504469B
:100A5000002854D00168002951D00B7843714B789D
:100A600083608A7843EA02238360CA7843EA0243B8
:100A700083600A7943EA026383604B7903738B795D
:100A8000C381CA7943EA0223027BC38102F00F02C9
:100A90000831103002F064F8237B002203F00F03CA
:100AA00084F8202084F82820227903F10800111A04
:100AB00004290DDD21680933043AD21A085C84F850
:100AC0002000D2B2606A84F82820194402F048F865
:100AD000237922681A44002012F8043CE36212F8D9
:100AE000031C43EA0123E36212F8021C43EA0143B8
:100AF000E36212F8012C43EA0263E36210BD0220B4
:100B0000FCE710B5044660B3036853B30279162AB4
:100B100029D942791A700146082251F8060B013092
:100B200002F028F82146082251F80E0B093002F095
:100B300021F82368E28A5A74E38A22681B0A9374B4
:100B40002368A269DA74A36922681B0A13752368F3
:100B5000628B5A752368E27E9A75172323710020F1
:100B600010BD0120FCE70220FAE738B50446002852
:100B700063D00168002960D0037B90F8282003F03F
:100B80000F03002A57D108332079043213449842C6
:100B900055D363790B702368A2685A70A3682268E2
:100BA0001B0A937023686289DA702368E27A1A71EB
:100BB0002368227B5A712368E2899A71E38922684B
:100BC0001B0A2146D371227B51F8100B02F00F0251
:100BD000083001F0C5FF237B94F8282003F00F03B1
:100BE00003F108052AB1226894F82010515503F149
:100BF0000905206894F82820616A284401F0B0FFB4
:100C000094F828302268E16A2B44D1545A1CE16AD6
:100C1000206892B2090A81549A1C2168E08D92B230
:100C20008854DA1C216894F82F0092B20433885457
:100C30002371002038BD0933A6E70120FAE702201E
:100C4000F8E70000024B1A8810431880704700BF75
:100C50001830002008B5074B1B883BB1FEF7CAF9D6
:100C6000002814BF6FF00200002008BD6FF00100E3
:100C7000FBE700BF1830002010B5034B00241C8098
:100C8000FEF7AEF9204610BD18300020B0FA80F013
:100C90004009704782B018B9084602B000F0CAB8DF
:100CA000002002B0704710B9084600F079B97047CB
:100CB00010B9084600F090B970470346084611463F
:100CC0000BB900F0DDB90020704710B9084600F0FC
:100CD00039BD704710B9084600F0FEB900207047D2
:100CE00010B40446084611461A46019B14B910BCBC
:100CF00000F00CBA10BC70470346084611460BB909
:100D000000F036BA0020704710B404460846114679
:100D10001A4614B910BC00F0A3BA002010BC7047EA
:100D200030B40546084611461A46DDE902341DB9BD
:100D3000029430BC00F022BB002030BC704710B9D8
:100D4000084600F0D3BB0020704710B9084600F0F9
:100D500037BD0020704710B9084600F0E2BB002004
:100D6000704710B9084600F0DFBB0020704703460B
:100D7000084611460BB900F0F9BB0020704710B4CB
:100D80000446084611461A46019B14B910BC00F0EF
:100D9000EFBB092010BC704710B40446084611464A
:100DA0001A4614B910BC00F02DBDC8B210BC704773
:100DB0000048704701000102064B10B51B6A04464B
:100DC000984730B10448054B204498428CBF00201E
:100DD000012010BD907E0308403576C9405DC600F5
:100DE000F0B5114B85B00C4610491F56054601F071
:100DF00017F80F4BE4B25E6A072D4FF00103CDE9FF
:100E0000024301460AD105220023CDE900234FF415
:100E10007A727A431846B04705B0F0BD0822002028
:100E2000CDE900203A46F5E77878030858780308BA
:100E3000907E03081FB5002300930378013B372BF6
:100E400021D8DFE803F01C242020201E20202020B1
:100E50004143454E2055585B5E6164206C1E6E73A5
:100E6000787A7D207F8326202020202020202020AB
:100E70002020202085878C2020858C208E92C3788E
:100E80000BB102230093009805B05DF804FB837852
:100E9000F6E743788DF8043007238DF80530837822
:100EA000003B18BF01235B008DF8063010238DF83E
:100EB0000730314B1B6801A803F55872CDE90223B6
:100EC00000F08EFF0090DEE74023DBE72023D9E728
:100ED000827890F9013012B9284AD35CD2E7284AC7
:100EE000FBE7827890F90130002AF8D1254AF4E72F
:100EF00040F6B833C6E74FF47A73C3E74FF4FA63AA
:100F0000C0E741F28833BDE741F27073BAE71E488B
:100F10004FF47A7101F008FE00F5FA60D2E71B4B3E
:100F2000B0E7154B1B6803F55873ABE7124B1B6812
:100F300003F55B73A6E71023A4E70F4B1B68A1E73B
:100F400001239FE74FF0834300939CE7104BFBE79F
:100F5000104B97E740F21113ADF8003093E70323ED
:100F600090E790F901300C4AB7E70C4990F901007D
:100F700000F056FFA6E700BF203000204D780308A0
:100F80003D7803084578030818FCFFFF00EA0637A0
:100F90009A99094040F70937787803085878030888
:100FA00037B50B4B02781B680C2101FB02335B7ACF
:100FB00003EB4304074B1D6803690093C368427841
:100FC000816805EBC40000F0A7FC03B030BD00BF92
:100FD000203000201C30002030B587B0027B642315
:100FE000ADF80030012A4FF00003CDE90133CDE91F
:100FF00003338DF802308DF8143028D0022A2FD018
:101000001ABB03680BB34368FBB11A4C80682360BA
:10101000194B18226946186001F0A2FD174B24688D
:1010200093E807000C3384E8070093E8070004F115
:101030000C05032385E80700A4F86C33012204F5AE
:101040005B7104F5587000F058FC07B030BD0949D9
:1010500008684360036100F55B7100F55870F2E7C2
:10106000044B1B68B3F86023B3F86C130A43A3F86E
:101070006023EAE7203000201C300020A81E03086F
:1010800008B503460A2924D8DFE801F00623232304
:10109000230B161B23212100BDE808400068FFF741
:1010A0008BBE90F900009978072271B900F0E5FB3A
:1010B000003818BF012008BD052293F90000002167
:1010C000F4E790F900005978EEE70221EEE70722F5
:1010D000F3E70020EFE7000008B502791AB1012A12
:1010E0000BD0002008BD084B01681B68012203F5E6
:1010F000587000F002FC0120F4E7034B01681B6804
:1011000003F55B70F5E700BF20300020F7B5072836
:10111000144D1C46A8BF072058700E462946174696
:1011200000F07EFE94F90130A070072B13D132201D
:1011300000F076FD0C4BDB6D0546984704F10C0280
:1011400008340346019200943A463146284600F09E
:101150006CFD03B0F0BD054A55F82310D05C00F0DB
:1011600057FDE7E758780308907E0308787803086E
:101170002DE9F04F344F90F901607B68D0F804906E
:101180008BB00446884698470546002859D1E37C31
:1011900073B92E4A2378126803EB4303990002EBDC
:1011A0008303D3F80490B9F1000F01D152F80190F4
:1011B000274B484613F906B0FB689847A37C228961
:1011C000D7F818A00993072E28D100230121CDE9D3
:1011D0000223204A0693CDE90431CDE907330521E6
:1011E000CDE900214FF47A7202FB0BF24CF2503140
:1011F0001846D047637C13B3174B995D7B6D0D3157
:10120000C9B228469847E07C3246494600F01AFEAB
:1012100088F8006001200BB0BDE8F08F00210125A7
:101220000823CDE90013CDE90715CDE90511CDE976
:1012300003110292A1782B465A462846D9E7074B5C
:10124000DBE70020E7E700BF907E030820300020A6
:101250007878030885450100457803084D78030830
:101260002DE9F04F8DB090F90130DFF8FCA0DFF8E8
:10127000FC90CDE90A123E4A12F903B00278DAF87E
:1012800000300C2505FB02333A4A5B7A126803EB07
:10129000430302EBC303044693F9021090F90200E2
:1012A00000F0B9FD3449064694F9010000F0B8FD9C
:1012B000A26861688046304600F0DFFC2178DAF8E9
:1012C0000020D9F80C306943074650589847D9F8A0
:1012D0001C309C4694F901300025072B4FF47A63AB
:1012E000CDE90753CDE905552DD10123CDE90353B0
:1012F0000523CDE901534FF47A7303FB0BF30093FD
:101300003946434646F2A81228466746B84723782E
:10131000DAF800200C214B4394F90110D05800F06A
:10132000B3FDA18994F90100FFF75AFD0B9B217BC6
:101330001860D9F85430284698470A9B01201E703F
:101340000DB0BDE8F08F01200823CDE90350CDE9B1
:1013500001032A46CDF800B0654643463946A84702
:1013600001200546D3E700BF20300020907E03080F
:10137000787803081C300020587803082DE9F04FD6
:101380008FB0002405468A46914698460494ADF8ED
:101390001440ADF8024007264FF0010B2B7AA34210
:1013A00006D9686804A9204400F0CAFB00285DD172
:1013B00002238DF8083002A86B7A8DF80A30FFF707
:1013C00039FDAB7A8DF81D309DF811308DF81E3047
:1013D0009DF812308DF81F309DF810308DF82030B8
:1013E000EB7A8DF821302B7B8DF822306B7B8DF8DA
:1013F000233010238DF81C608DF824303A4E8DF880
:101400002C000DF102030A93072332688DF82D306A
:10141000ADF834302B680C9206930DF1120204AB38
:101420000DF1110106A800F0A5FB072805460BD118
:1014300030680C22002100F5587001F0A5FB3368DC
:10144000BDF80220A3F860239DF811308AF800301F
:101450009DF8123089F800309DF8103088F800307F
:10146000189B28461C700FB0BDE8F08F9DF8133014
:10147000BDF81470ADF802702044C4B2F3B917B3CC
:10148000194A00201168072602464FF00C0C062B63
:101490001BD10CFB00FE51F80EE0BEF1000F04D092
:1014A0000BFA00F23A4397B2012201301028EED134
:1014B000002A3FF473AFADF802706FE75A1E042A9A
:1014C00001D9062BDCD0062668E747FA00FE1EF09D
:1014D000010FEAD00CFB00FE51F80EE0BEF1000F48
:1014E00008BF0626E1E700BF2030002038B50546DA
:1014F0004068FFF761FC0722841D002195F9000078
:10150000E4B200F0BAF908B904F0FD0495F901005D
:101510000722002100F0B1F908B904F0FB042046CD
:1015200038BD00207047000010B503780F2B04462B
:1015300018D84068FFF740FC22780B4902EB4202C2
:101540000968831C01EB820051F82220DBB21AB932
:1015500003F0FD0358B210BD032B06BF6268426062
:101560000223F7E70020F6E7203000200220704732
:101570002DE9F0413A4D0446286896B00E46904653
:1015800000211F460122032300F55870CDE9041104
:10159000CDE906118DF80C108DF80D10ADF80E3058
:1015A00000F08DF930B92A68B2F8603343F00303D4
:1015B000A2F860332A68637A8DF8203002F55871FA
:1015C000CDE90912274A94F9083012680B921022CB
:1015D000ADF830200DF10E020D9222680E92626875
:1015E0000F92D4E90301A27A8DF8402001228DF8F0
:1015F000412011AA82E80300227DE18A8DF8213082
:1016000018468DF84C20FFF7EBFB08AB15930DF156
:101610000D0314900093CDF8048003AB04AA39465F
:101620000EA800F099FB044678B99DF80C1001391A
:1016300001F07AFA00F158030DEB030010F8483C72
:101640003370204616B0BDE8F0810C2801BF2A682F
:10165000B2F8603343F00303A2F86033F1E700BF50
:10166000203000201C300020F8B50679012E0546F8
:1016700048D90F2E48D80368187A40F30300072290
:10168000002140B200F0F9F82B680446187A40F3C4
:1016900003100722002140B200F0EFF8B8B1B4FA0D
:1016A00084F4640929680B7A086843F3030243F35E
:1016B00003135BB252B29A42C8BF0124FFF77CFB0E
:1016C00080F00103DBB224B10533D8B2F8BD0124A8
:1016D000E8E7DBB90E4F29683B6806EB460003EBF1
:1016E00080000C2201F03CFA3A680C2303FB06232D
:1016F00020465C72B2F860130123B3400B43A2F89A
:101700006033E3E70620E1E70320DFE70420DDE7BD
:101710002030002010B4017801290ED9084B186838
:101720000C234B43C4180022C250C4E9012200F527
:10173000587010BC102200F0A9B8002010BC7047EF
:10174000203000202DE9F04186B050238DF8143070
:10175000037A102B074630D14368DD7B6DBB022432
:10176000A8466426062C14D87A68535D03932A444D
:10177000517843EA01230393927843EA0243734387
:10178000CDE9033863B968468DF80040FFF7C2FF22
:101790000DE0CDF80C808DF81480CDF81080F2E7C4
:1017A00003AB01A801938DF80840FFF75DFF0134FA
:1017B000E4B2102C05F10305D4D106B0BDE8F081E8
:1017C0001FB502680379116849B901A88DF8043082
:1017D000FFF7A0FF78B1032005B05DF804FB02A875
:1017E00002928DF80C30FFF73FFF042805D0052842
:1017F00005D00028EFD00020EEE70220ECE7012022
:10180000EAE70000C90020B9034B0B449856C0B268
:101810007047024BF9E700BFFD770308BD77030867
:10182000F0B59A42069D03DB9DF914309A4220DD03
:101830000020F0BD03EB430331F814C005EB830334
:1018400000264CFA06F7FF0707D51F7A07F00F0EA0
:10185000964502DCB2EB171F0DDD0136102E03F1A9
:101860000C03EED10134E4B22301DBB29842E1D89B
:10187000DEE70024F8E70120DBE7884204DB904242
:10188000CCBF0020012070470020704710B514091C
:10189000B4EB111F03464FEA11100ED391420CD244
:1018A00002B201F00F0133F81240012000FA01F1F9
:1018B00024EA010123F8121010BD0020FCE7F0B566
:1018C00028B100EB410501270020914200D3F0BD73
:1018D000002435F802CB234607FA04F636EA0C0654
:1018E00008BF013304F1010408BFDBB2102CF3D1AF
:1018F00018440131C0B2C9B2E7E710B500B149B927
:1019000010BD31F8134020F813400133DCB2A2427D
:10191000F7D8F5E70023F9E782B030B504880493DF
:10192000D2B9B3F5616F15D349F6AF2542F2107203
:10193000AB4298BF4FF47A72944238BF1446614369
:10194000BDE83040C3688B428CBF5B1A0023C36084
:1019500002B070476422EFE7012C38BF0124EEE7A4
:101960002DE9F04F8FB01546199F03939DF8603015
:1019700007930C46804603F0C7FB6A4A0590A7F51B
:10198000F633303BB3FBF2F3534303F5F63B0493DA
:10199000182313FB05430BF1300B069300254FF082
:1019A000FF3A069B9C4207D1002D14BF50464FF0D2
:1019B000FF300FB0BDE8F08FBDF96830ADF82430CE
:1019C000099919973846089703F02EFB2688B8F135
:1019D000000F5FD1B7F5616F5AD349F6AF2242F2DB
:1019E0001073974298BF4FF47A739E4238BF1E46D9
:1019F000642E59D1DFF83091A060A1680CA803F0E3
:101A000035FB0D9B0093DDE908120C9B0AA803F03F
:101A10008CFA039A0A9B0AB9079A2AB122694A45A5
:101A200002D1424A93420ED9414BC4F80C909F42D6
:101A300009D90023ADF82C300B99CDF828B05846C1
:101A400003F0F2FAA060606808B9C4F80C90C4F81A
:101A50001090B8F1000F04D003F060FBE36803447A
:101A6000E360D4E903329342059B88BFE260636080
:101A70001B9BE1687343994204D20398E8B9B8F11B
:101A8000000F1AD001231D442375EDB2183488E7E6
:101A90006423AAE7039B0BB9234BE360012EDFF815
:101AA000889038BF0126CEE7B6F57A7F0ABFDFF807
:101AB0008490DFF88490A0609FE700209342207517
:101AC00006D85B1A9A4505F1010528BF9A46EDB282
:101AD000B8F1000FDAD1642E184AADF82C801DD071
:101AE00049F6B023B6F57A7F18BF1346974281BFF7
:101AF000049A02F5A83202F5C0729B180A931A9B49
:101B000000930AAE96E80600199B304603F00DFAE2
:101B100096E8030003F088FA8246B7E74FF4616362
:101B2000E4E700BF8051010040771B007F510100B6
:101B30002FEC010080A81201002E930230EC01006E
:101B40000378032B14D1437803F00F021B098A702A
:101B50004B7083788B80C27843EA02238B800379B1
:101B6000C3F3021203F00F03CA700B700520704715
:101B7000002070472DE9F3479A464379057990F99B
:101B800007609146044690F906208846D3B190F943
:101B90000870002D37D00F2A1BD194F909200F2E81
:101BA00027D194F90A00072D02D1002F08BF012781
:101BB00088F8002089F8000028468AF8007002B0F2
:101BC000BDE8F08790F90B7090F9092090F90A6050
:101BD000DFE7A369019394F91530009394F9143069
:101BE0002169207BFFF71CFE0028D8D105F0FD05F8
:101BF000D5E794F91D00B042D5DC94F91C30B3420E
:101C000003DA05F0FB053046D2E73046CBE70000AB
